:1000000000800020BD01000099DA000051DA0000F4
:1000100051DA000051DA000051DA000051DA000034
:1000200051DA000051DA000051DA000099DA0000DC
:1000300099DA000051DA00009104010095040100F2
:1000400099DA000099DA000099DA000099DA0000E4
:1000500099DA000099DA000099DA000099DA0000D4
:1000600099DA000099DA000099DA000099DA0000C4
:1000700099DA000099DA000099DA000099DA0000B4
:1000800099DA000099DA000099DA000099DA0000A4
:1000900099DA000099DA000099DA000099DA000094
:1000A00029B1000035B1000099DA000099DA0000AA
:1000B00099DA000099DA000099DA000099DA000074
:1000C00099DA000099DA000099DA000099DA000064
:1000D00099DA000099DA000099DA000099DA000054
:1000E00099DA000099DA000099DA000099DA000044
:1000F00099DA000099DA000099DA0000E1E80000DE
:1001000099DA000065EE000099DA000099DA000043
:1001100099DA000099DA000099DA000099DA000013
:1001200099DA000099DA000099DA000099DA000003
:1001300099DA000099DA000099DA000099DA0000F3
:1001400099DA000099DA000099DA000099DA0000E3
:100150004108010055080100690801007D080100FF
:1001600099DA000081F1000099DA000099DA0000C4
:1001700099DA000099DA000099DA000099DA0000B3
:1001800099DA000099DA000099DA000099DA0000A3
:1001900099DA000099DA000099DA000099DA000093
:1001A00099DA000099DA000099DA000099DA000083
:1001B00099DA000099DA000099DA0000564B4CF207
:1001C000205210B51A804DF628121A8000BF00BFC9
:1001D0000DF066FC514B4FF010621A60504A9A6065
:1001E000504ADA60504A136813F4807304D14F49BF
:1001F0000B604FF4A85313604D4B1A78110703D5C9
:100200001A7842F008021A704A4B4B492A221A7097
:100210004A4A4B4B8B4204D252F8040F43F8040B6A
:10022000F8E7484B484900228B4202D243F8042B9E
:10023000FAE74649464A002352F8230041F82300D2
:1002400001336F2BF8D1434B434A802103F8011B44
:100250009342FBD1414B3D4A1A60414B8A221A70AE
:10026000A3F5805324225A70A0221A709A7992071B
:10027000FCD59A79D406FCD43A4A937903F00C035E
:10028000082B384BF9D103221A7140225A719A79FE
:100290009006FCD5334A9179324B4906FBD5324A58
:1002A000324911600221516020221A709A7902F0BD
:1002B0000C020C2AFAD12E4B2E4A1A602E4B2F4AD2
:1002C0001A6000225A60072243F8042C2C4AC3F813
:1002D0000C2D62B60DF06EFF144B1B68DA0705D5C6
:1002E00028480DF03BFD284B284A1A60284B1B7804
:1002F0005B0609D5244C254B22689A4204D121483B
:100300000DF02CFD0023236011F026FE0DF0CEFB36
:1003100010F02CFBFEE700BF0E20054030800440AB
:10032000823F04000100002B10D0034014D0034092
:1003300002D0074000E00740049CFF1FA4590100C1
:100340004088FF1F049CFF1F98A3FF1F0082FF1F10
:100350000000000000E400E05FE400E008ED00E0E1
:100360000050064000400640448004400000030165
:1003700004800440C010050014E000E0FF76010096
:1003800000002020611EEF5F1CE00340A5C3945ACB
:1003900000F00740FFFFFFFFFFFFFFFFFFFFFFFF32
:1003A000FFFFFFFFFFFFFFFFFFFFFFFFFFFFFFFF5D
:1003B000FFFFFFFFFFFFFFFFFFFFFFFFFFFFFFFF4D
:1003C000FFFFFFFFFFFFFFFFFFFFFFFFFFFFFFFF3D
:1003D000FFFFFFFFFFFFFFFFFFFFFFFFFFFFFFFF2D
:1003E000FFFFFFFFFFFFFFFFFFFFFFFFFFFFFFFF1D
:1003F000FFFFFFFFFFFFFFFFFFFFFFFFFFFFFFFF0D
:10040000FFFFFFFFFFFFFFFFFFFFFFFFDEF9FFFF23
:1004100010B5054C237833B9044B13B10448AFF33E
:1004200000800123237010BD049CFF1F000000000A
:10043000A0590100084B10B51BB108490848AFF39B
:1004400000800848036803B910BD074B002BFBD0A0
:10045000BDE81040184700BF00000000089CFF1FC7
:10046000A0590100049CFF1F0000000038B504469D
:10047000104621700A491D4611F056FB01464FF007
:100480007E5011F005FC074911F04EFBE5606060FD
:10049000256165610DF01EFEE061204638BD00BF9C
:1004A000DB0FC9400024744938B50446104621705A
:1004B00009491D4611F038FB01464FF07E5011F0FE
:1004C000E7FB064911F030FBE5606060256165617E
:1004D0000DF000FEE06138BDDB0FC9400024744917
:1004E00038B503780446032B20D8DFE803F01A1848
:1004F0001002C168406911F00DFA0D4905466068A7
:1005000011F0C6FB0146284611F0C2FB38BD084970
:10051000406811F0BDFBE16811F006FB38BDC06812
:1005200038BDC168406911F0F5F938BD002038BD0B
:100530000024744970B504460E460DF0CBFD054607
:10054000E069281A11F09CFAE3682361E5616661AD
:10055000A0610146606811F09BFB0146A060104855
:1005600011F096FB10F06CFE10F006FB11F07EF916
:10057000054601464FF07E5011F0CCF9616911F04B
:10058000D3FA21690646284611F0CEFA01463046D4
:1005900011F0C2F9E0602046BDE87040FFF7A0BF4F
:1005A000000080BF08B50E200DF02CF9114B1B8800
:1005B000012B19D0104B1B88984213DB40F6FF71BA
:1005C0008842D4BFC3EB0001C3EB0101C1EB013191
:1005D000C3F57F630F33282091FBF3F1BDE808409A
:1005E0000DF0CEBB0021F3E70146BDE80840142022
:1005F0000DF0C6BB609EFF1FF49CFF1F10B50446A4
:1006000010F0FCF8204610BD70B44C88A04220D9F0
:1006100001230133DBB21CB2660031F8144084427E
:100620001D46F6D3A04211D005F10045013D965B71
:1006300031F8151032F81530401AF21A00FB02F0AA
:10064000641A90FBF4F4E01870BC7047905B70BCC7
:10065000704702260125E5E700280CDA064A4342E6
:1006600082FB0320DA17C2EB600000EB4000A3EB33
:100670008000C0F10C007047ABAAAA2A38B5234B02
:100680001B78002B2CD015200DF0BCF8204B1860E7
:10069000204B1B88984203DA1F4C237863BB38BD7C
:1006A0001E4A1488A042A4EB0302A8BF20467F2A5A
:1006B0001CDDC01AC001541C90FBF4F4002CEBD0DC
:1006C000154B1A780AB901221A70154D2B689C42F5
:1006D00004D0144BE1B2187808F002FE2C6038BD4B
:1006E00011200EF02BFC0A4B1860D1E7C01AC0EBAA
:1006F000C01090FBF2F4E1E70A4B0021187808F0F3
:10070000EFFD0023064A2370136038BD729EFF1F61
:10071000309CFF1FAA9CFF1FE09EFF1F8C9EFF1FA7
:10072000DC9EFF1F809CFF1F38B50F200EF006FCDB
:100730001B4A1C4B12881860C0F53B600830904281
:1007400020DB194B1B889842A3EB0204A8BF184674
:10075000801A7F2CC6BFC0010134C0EBC01090FBD3
:10076000F4F47CB1114B1A780AB901221A70104DB9
:100770002B689C4204D00F4BE1B2187808F0B0FD12
:100780002C6038BD094C237803B938BD094B0021D2
:10079000187808F0A5FD0023054A2370136038BDC2
:1007A000F89CFF1F449CFF1F789EFF1F9C9EFF1F0D
:1007B000B49CFF1FA29CFF1FF0B40E8886420DD28E
:1007C00003F10043013B31F81350854202D9F0BCDC
:1007D000FFF71ABF32F81300F0BC70471088F0BC66
:1007E000704700BF094B1B880C2B09D8084A80B200
:1007F00052F8232028B143F6FE73984203D9108C97
:100800007047108870470349FFF7FEBE5A9CFF1FD0
:1008100060330100FC3401004B4B4C4A2DE9F0479A
:100820001E8814684A4BB442B3F80080494B33DB4E
:100830004445A8BF4446A6421C60C8BF00202DDD29
:10084000C6EB0807B7F5804F33DB80037B1C90FBBA
:10085000F3F0FFF7C7FF404A404B15881B88C0F3F1
:10086000C61909FB05F57F2D8246A8BF7F252BB34E
:10087000A64253DC4445D4BFC6EB0404C6EB0804CF
:100880009F42CCBF03FB04445C43354BC8BF0137D8
:1008900094FBF7F71F6013E034461E60C6EB0807B1
:1008A000A045D4BFC6EB0800C6EB0400B7F5804FE7
:1008B000CBDAC0EB803090FBF7F0CAE7284A136030
:1008C000284C2368994508D0274B1B88002B34D12E
:1008D000264B1B886BBBC4F80090254C23689A45B7
:1008E00006D0214B1B885A1F032A19D9C4F800A02F
:1008F000204C23689D420FD01F4B188848B11A4BDB
:100900001E4A1B88D35C834203D0C0B2E9B208F010
:10091000E7FC2560BDE8F087BDE8F0870024AFE77D
:10092000164AD05C2030C0B20AF07F0108F0D8FC33
:10093000DCE7484608F074FDCDE7104A4946D05C34
:1009400008F0CEFCC4E700BFF49CFF1F5C9EFF1FB5
:10095000BC9EFF1F289CFF1F389CFF1F3A9CFF1F57
:10096000C09EFF1F9C9CFF1F429EFF1FEA9CFF1F13
:10097000549CFF1FEC9CFF1F529EFF1FB089FF1F5E
:100980002DE9F04F17208BB00EF0D8FADFF870B3D6
:10099000DFF870A3CBF8000016200EF0CFFABA4BA8
:1009A000CAF800001B880C2B00F05E82B74EB84AD4
:1009B0003188B84B52F8214000221A70B64BB74A22
:1009C0001B88B7491288013B012A31F9133005937E
:1009D00000F0AE81B34B0193B34B0293B34FDFF8FA
:1009E000288300230093B24B1B88012B00F0F48175
:1009F000DFF81893AF4B0393D9F80050AE4B049334
:100A00000023AE4A1288013A032A00F24982DFE845
:100A100012F0A500ED000400C9002846059311F06E
:100A20002FF8A74911F080F8059B0546184611F0EC
:100A300027F8A44911F078F80146284610F06CFF19
:100A400011F038FA0546C9F80050386811F018F866
:100A50009B4911F069F88146009811F011F8994905
:100A600011F062F80146484610F056FF11F022FAE4
:100A70003860954A954B17881988954BDBF800200C
:100A80001B88DFF88CE2C7EB050C3D44039FC7F8D9
:100A900000C0471A084404990D6001990F6002993B
:100AA000BEF8007008609A4280F2E7800025C3EB30
:100AB000070E7445DAF8000080F2D380611C98427A
:100AC00005FB01F50EF1010E95FBFEF5C0F25F830B
:100AD0008742A8BF0746FF1A01FB07F494FBFEF408
:100AE0009A4200F3A780984200F3A480794C2068D2
:100AF00010F0C6FF784911F017F8784910F00CFF94
:100B000011F0D8F9A0F5FF531C3B082B98BF4FF408
:100B10000050D8F80030184400282060C0F29F80B0
:100B2000B0F5804F80F2F6806D4B1B781BB1B0F5AD
:100B3000005F40F0F7806B4D2B78002B40F0AB81CD
:100B4000694D20682B68634C984204D080B208F04D
:100B500097FB23682B600BB0BDE8F08F2846059308
:100B600010F08EFF614910F0DFFF059B0546184627
:100B700010F086FF5E4910F0D7FF0146284610F0BE
:100B8000CBFE11F097F90546C9F80050386810F00F
:100B900077FF564910F0C8FF8146009810F070FFAB
:100BA00053495DE72846059310F06AFF4A4910F063
:100BB000BBFF059B0546184610F062FF4D4910F03B
:100BC000B3FF0146284610F0A7FE11F073F9054661
:100BD000C9F80050386810F053FF3F4910F0A4FFE7
:100BE0008146009810F04CFF424939E728460593AA
:100BF00010F046FF404910F097FF059B0546184648
:100C000010F03EFF3D4910F08FFF0146284610F0DE
:100C100083FE11F04FF90546C9F80050386810F00E
:100C20002FFF354910F080FF8146009810F028FF13
:100C3000324915E73388002B3FF458AF2B1B002BAC
:100C4000B8BF5B42092B00F32D81D8F80030214C4E
:100C50004FF40050184400282060BFF661AF002216
:100C60005AE0984205FB04F5B8BF002195FBFEF55C
:100C700080F2848291FBFEF432E7BA42D4BFC3EB28
:100C80000205C3EB070512E78E9EFF1F909CFF1F16
:100C90006C89FF1F2E9CFF1F3689FF1F629EFF1F5E
:100CA00068370100849CFF1FC49CFF1F209CFF1F0E
:100CB000F09DFF1F809EFF1FF49DFF1F4289FF1FB5
:100CC000CDCC4C3FCDCC4C3EBC89FF1F4089FF1F93
:100CD000589EFF1FA489FF1F9A99193FCDCC4C4500
:100CE000969FFF1FE89CFF1F3889FF1F3333733F18
:100CF000CDCC4C3DCDCCCC3E6666663FCDCCCC3D1C
:100D00008C9CFF1F509CFF1F989EFF1F7C9EFF1F07
:100D10006C9CFF1F43F6FF72C04B22601B78002BB8
:100D20003FF409AF05F024FCBD4B01221A7007E720
:100D3000BC4BBD4A1B88BD491278013B31F91350A9
:100D4000002A40F0C78011200EF0F8F80090B84B50
:100D50000193D3F80080009B984540F3C080B54BC9
:100D6000B54F1B88B54A012B3B68B2F80090B44AD6
:100D700002922046A3EB050500F0E28010F080FE11
:100D8000029A52F8291010F0CFFE0146002010F010
:100D9000C1FD11F08FF8009BC8EB05029D42B8BF62
:100DA0001D469042C8EB050580F2DE8000FB05552C
:100DB000013295FBF2F5A34BDFF8B4820293D8F829
:100DC00000302B4403EBD3735B10C8F800309E4B0C
:100DD0001B88012B7FF40CAE9C4B03931D460F2008
:100DE0000EF0ACF82A6804929042034680F2CC8060
:100DF000904A1288012A00F03F81904A0790128899
:100E00008F4D0692204610F03BFE069ADFF8649262
:100E100055F82210D9F8005010F086FE0146002047
:100E200010F078FD059BEA1A059211F043F8059A37
:100E3000079B04999A42C1EB020EB8BF1A4670454F
:100E400080F24481521A00FB02220EF1010192FB52
:100E5000F1F2D8F800107E4804900A4402EBD272F6
:100E60005210C8F80020CCE57A4B1B78002B3FF4D9
:100E70009DAD794E794A3188794B52F82100012293
:100E80001A7010F0FDFD4FF07C5110F04DFE11F086
:100E900011F8044692E505F067FB00232B704FE63E
:100EA0003868E6E505F500500130001B10F0E8FD5C
:100EB0006C496D4C10F038FE0546206810F0E0FDDE
:100EC0006A4910F031FE0146284610F025FD10F069
:100ED000F1FF1EE615200CF095FC009037E7594B0A
:100EE0000293D3F80080009B984542DA514B524F51
:100EF0001B88524A012B3B68B2F80090504A03927B
:100F000020461D4400F0E98010F0BAFD039A52F823
:100F1000291010F009FE10F0CDFF009B9D42C8EB98
:100F20000502A8BF1D46C8EB05059042BABF00FBED
:100F300005550132454395FBF2F5DFF834813EE774
:100F400010F09EFD029A52F8291010F0EDFD10F0FD
:100F5000B1FF009BC8EB05029D42B8BF1D4682420F
:100F6000C8EB05053FF722AF00FB05F595FBF2F551
:100F700021E7DFF8FC80304FD8F8003003EBD37363
:100F80005B10C8F800302EE5314A049212680692D0
:100F9000904237DD274A1288012A00F0BC80274A98
:100FA00009901188264A08912046079210F068FDA2
:100FB000079A0899DFF8BC9052F82110D9F8005030
:100FC00010F0B2FD059B2B44059310F073FF0599BB
:100FD000099B069A9942C2EB010EA8BF19467045BB
:100FE00080F2BE80891A00FB01110EF1010291FB13
:100FF000F2F2D8F800100A4402EBD2725210C8F88C
:101000000020FEE4D8F80020DFF8689002EBD272EE
:101010005210D9F80050C8F80020F2E4969FFF1F44
:10102000E89CFF1FC089FF1F729EFF1FB4340100A0
:10103000849CFF1FCA9CFF1F209CFF1F749CFF1FE6
:1010400080370100C49CFF1FF09DFF1F809EFF1F83
:10105000F49DFF1F409EFF1F909CFF1F6C89FF1F88
:101060002E9CFF1FCDCCCC3EA489FF1F9A99193F1F
:10107000989EFF1F7C9EFF1F464A08901188464A93
:1010800007912046069210F0FBFC069A0799DFF8BC
:101090000C9152F82110D9F8005010F045FD059B35
:1010A000E91A059110F006FF0599089B049A9942E8
:1010B000C2EB010EB8BF1946704558DA891A00FB19
:1010C00001110EF1010291FBF2F2C2E60499521AEB
:1010D00000FB02F292FBFEF2BBE610F0D1FC039A99
:1010E00052F8291010F020FD0146002010F012FCEB
:1010F00010F0E0FE009A9542C8EB0503A8BF154624
:10110000C8EB05059842BABF00FB055501334543BE
:1011100095FBF3F511E71F491F4A089020460D88FB
:10112000079210F0ADFC079ADFF8709052F8251086
:10113000D9F8005010F0F8FC0146002010F0EAFB4E
:10114000059B2B44059310F0B5FE0599089B069A64
:101150009942C2EB010EA8BF19467045FFF642AF97
:10116000069A891A00FB01F191FBFEF241E7049A0D
:10117000891A00FB01F191FBFEF26AE6B842D4BF86
:10118000C3EB0001C3EB070104FB01F172E51F464D
:10119000A1E400BF749CFF1F803701007C9EFF1FED
:1011A00008B5244B1B88FBB1234B1B78FBB1234BA9
:1011B0001B78E3B1224B1B78CBB1224B1B78B3B128
:1011C000214B22481A78C2B9214A22490088128844
:1011D00009680244B1EB620F09DD01221A70642034
:1011E000BDE8084005F0D8B9174A117801B908BD23
:1011F0001370BDE8084008F0E7B8154A16490088A2
:10120000128809680244B1EB620FF0DD00221A7007
:1012100008F0DAF8642005F0BFF9642005F0BCF9A5
:10122000642005F0B9F94FF41670BDE808400CF0E1
:1012300073BF00BF009EFF1FE49EFF1FB69EFF1FEF
:10124000B79EFF1FB89EFF1F589CFF1F6C9CFF1F7F
:10125000589EFF1F8C9CFF1F509CFF1F38B5114CE0
:10126000232025780CF0CEFA0F4A42F82500131FF0
:1012700002F1C400002253F8041F83420A44FAD149
:1012800023780A4907480A4C0133DBB2322B81FB31
:10129000025108BF0023D217C2EB21120370226053
:1012A00038BD00BF3C9CFF1F049DFF1F1F85EB51F5
:1012B000549EFF1F2DE9F04FB84CB94D2068B94F2F
:1012C00083B010F0DDFBB84910F02EFC064610206C
:1012D0000DF034FE10F0D4FBB44910F025FC31467B
:1012E00010F01AFB10F0E6FD2988206088423B8848
:1012F00043DA9E465B1A7F2B4FF0000247DDD20196
:101300005E1C92FBF6F2AA4EDFF8C882B6F800C067
:10131000C8F80020BCF1190F00F0DF80BCF11A0FF3
:1013200000F01781BCF11E0F00F020810126B146AC
:10133000A04A1288002A00F09D808842C0F20781EE
:101340007045D4BFC1EB0000C1EB0E009A42BABF9A
:1013500002FB00000133504390FBF3F3964A136005
:10136000964B1888C0B9964A1288AAB9954B197835
:1013700001B11A7003B0BDE8F08F9842D4BFC1EB41
:101380000002C1EB03029E465B1A7F2BB7DCC2EB67
:10139000C21292FBF3F2B6E72988D4F800E0DFF836
:1013A0000082DFF8F8A171456CDCDFF818C29CF808
:1013B0000020002A2ED14FF0010B04288CF800B039
:1013C00028D1002E40F094817D4B18880028D1D080
:1013D000B9F1000FCED023682C883A88A34280F25E
:1013E00065810023141B7E2C774DD5BFC3EB83137F
:1013F000C3EBC3135B00013493FBF4F42B6801349B
:10140000A34203D0C0B2E1B207F06AFF2C6003B080
:10141000BDE8F08F012800F0F680022800F0EB8094
:101420000328D1D1694B1B88092BCDD0002ECBD0FE
:1014300023682E883A88B34280F27B810023961B72
:101440007E2EDFF88CA1D5BFC3EB8313C3EBC31390
:101450005B00013693FBF6F6DAF800300136B34252
:1014600003D0F1B24A2007F03BFFCAF80060ABE7B7
:1014700016469146BCF11E0F7FF472AF0022DFF8D2
:1014800058817EE04F4B1A78002A3FF473AF002456
:1014900001281C7000F0A480022840F00E81002E6C
:1014A00000F0A3804A4D2B68002B00F09E800420A2
:1014B000214607F015FF424B2C60188800283FF4A6
:1014C00059AFB9F1000F3FF455AFC0B2002107F09A
:1014D00007FF3D4B00221A604CE7DFF8FC8098F8CC
:1014E0000020C2B1DFF8D890B9F800A0BAF1000F1F
:1014F00011D0DFF8E89099F800B0934578D05FFA02
:101500008AF07F2107F0ECFE98F80030B6F800C0B2
:1015100089F8003010E0DFF8C49099F800A09245F7
:1015200066D0274B0021187807F0DAFE98F80030D3
:10153000B6F800C089F800301E4B1A88002A97D0F0
:10154000BCF11E0F40F006810026B14619E00020D4
:10155000FCE6DFF8848098F80020002A0BBF012603
:1015600000264FF000094FF00109E1E6DFF868803E
:10157000104B98F800601A88B6FA86F676094FF094
:10158000000998F80030002B3FF4E8AE2988B7F83E
:1015900000E02068C1EB0E03CFE600BF7C9CFF1F7C
:1015A000069EFF1F029EFF1F9A99193FCDCCCC3E8D
:1015B0008E9EFF1FC49EFF1FFC9CFF1F8A9CFF1F67
:1015C000A09EFF1F959EFF1F609CFF1F429EFF1F56
:1015D000009DFF1F749EFF1F409EFF1F409CFF1F2A
:1015E0001EB1614D2B68002B7BD1604B188865E7DD
:1015F0000026B1469CE6002E3FF4E6AEDFF868A177
:10160000DAF800202EE0002E3FF4DEAEB7F80080BE
:10161000F045D4BFC1EB0802C1EB0E02C1EB0808D4
:10162000B8F17E0FDFF840A1D5BFC2EB8212C2EB4A
:10163000C212520008F1010892FBF8F8DAF8002013
:1016400008F10108424506D05FFA88F101200093B5
:1016500007F046FE009B1888CAF8008002287FF435
:10166000DFAE42462168B5F800803888414559DA36
:101670000021C8EB0008B8F17E0FD3BFC1EB811188
:10168000C1EBC11108F10108490091FBF8F808F11C
:101690000108904506D05FFA88F10420009307F016
:1016A0001FFE009B1888CAF80080B9E69342D4BF99
:1016B000C4EB0303C4EB020394E6032827D12C4BAD
:1016C0001B88092B91D0002E8FD0274D2B68002B23
:1016D0008BD04A20214607F003FE244B2C6018884B
:1016E000ECE6214607F0FCFD204B2C601888E5E66F
:1016F00040207F218DE80C0007F0F2FD019B009A4D
:10170000188858451CD002287FF48AAE76E7042852
:101710007FF46BAF002E3FF468AF2146402007F006
:10172000DFFD62E78142D4BFC8EB0101C8EB0001D5
:101730009FE79342D4BFC6EB0303C6EB02037EE6EA
:10174000B8F80010DAF800E0B7F800808E45FFF630
:1017500065AF5DE72988B7F800E020680026C1EB97
:101760000E03B146E9E500BF009DFF1FA09EFF1FCD
:10177000429EFF1F08B5114B1B88022B09D0052B79
:1017800007D0032B15D0042B0BD00D4B01221A7060
:1017900008BD7F21412007F0A3FD094B01221A70EB
:1017A00008BD7F21092007F09BFD054B01221A701F
:1017B00008BD4021092007F093FDE6E7FA9CFF1FD2
:1017C000AC9CFF1F38B5074B074D1B88052B044603
:1017D00006D02B68834203D0C1B2052007F080FDFC
:1017E0002C6038BDFA9CFF1FA49EFF1F38B5124D18
:1017F000124C2B88052B12D022684AB9022B0ED02E
:10180000033B012B13D90E4A00231370236038BD0C
:101810000021052007F064FD2B88022B04D1002154
:10182000412007F05DFDEEE7052BE9D1F7E7002148
:10183000092007F055FDE6E7FA9CFF1FA49EFF1F55
:10184000AC9CFF1F464B1B881D2B70B541D0454DEE
:101850000024454B1B88022B16D0444B1B88022BBF
:1018600054D02888424B002C1B780ADB8442A8BF46
:10187000044634B1002B3AD02046BDE87040FFF753
:10188000A1BF002B2FD170BD3A4B1B78002B37D056
:1018900015200BF0B7FF384B1860384A1288002A21
:1018A000DBD0374A186811888142D6DC354B2A884C
:1018B0001B888342A3EB0106A8BF03465B1AB24212
:1018C000BABF02FB03330136534393FBF6F31C44C8
:1018D000C3E72A4B1C888CB12B4B224D1C78002C63
:1018E000B7D02C88B5E7BDE87040FFF77FBFFFF7A2
:1018F00041FF2046BDE87040FFF764BF194DA8E7DF
:1019000011200DF01BFB1C4B1860C6E70F200DF0DB
:1019100015FB1A4B1D4A1B881060002BA1D01C4AD6
:10192000C0F53B63118808338B429ADB194A28883B
:1019300012889342A2EB0105A8BF1346A842A3EB6D
:10194000010306DA00FB0333013593FBF5F31C4476
:1019500088E700FB03F292FBF5F31C4482E700BF2B
:101960008E9EFF1F929EFF1F629EFF1FF09DFF1F16
:10197000AC9CFF1F729EFF1F309CFF1FFA9CFF1F35
:10198000AA9CFF1F8C9EFF1F409EFF1F449CFF1FB1
:10199000F89CFF1F789EFF1F38B510200DF0CEFA7F
:1019A000C830B0F5FA7FC0F2EE80B0F57A6F01462C
:1019B000A8BF4FF47A6101F51673B3F57A6FA8BF2B
:1019C0004FF47A639BB289B28E4A8F4C11802220E9
:1019D000238007F007FE21888C4D8D4C242007F0D2
:1019E00001FE0E200BF00EFF40F6FF71C83088425A
:1019F000A8BF084620EAE07000F2DC5283B28A42B7
:101A0000A8BF0A460220194622802B8007F0EAFD73
:101A10002188042007F0E6FD17200DF08FFA044618
:101A200016200DF08BFAA042B8BF204600F1C80185
:101A3000B1F5FA7FC0F2A280B1F57A6FA8BF4FF47A
:101A40007A6101F54873B3F57A6FA8BF4FF47A63F2
:101A50009BB289B26F4A704C11800A20238007F034
:101A6000C1FD21880C2007F0BDFD0F200DF066FAA6
:101A7000C0F53F610431B1F5AF6F7CDBB1F5FA6FB2
:101A8000A8BF4FF4FA6189B2644BC0F54360B0F56A
:101A9000AF6F19806CDBB0F5FA6FA8BF4FF4FA6036
:101AA00083B25F4CA420238007F09CFDA6202188F0
:101AB00007F098FD0B200CF0F9FA002868D01120EF
:101AC0000DF03CFA00F1C801B1F52F7F6EDA40F25B
:101AD00014534FF42F71534A1180534C0620238026
:101AE00007F080FD2188082007F07CFD00244FF4DA
:101AF000AF75E1B24D4809F04DFB01348542A8BFF6
:101B000005460C2CF5D101200DF018FA04460020F2
:101B10000DF014FA323CA0F1320345496FF4957090
:101B200000FB03F300FB04F081FB034281FB004157
:101B3000DB17C017C3EB6223C0EB612003F5AF7264
:101B400000F5AF739342A8BF13469D42A8BF1D4640
:101B5000A5F11401312938DC40F26C73322135488B
:101B6000354A018013602A20BDE8384007F03ABDAD
:101B70004FF4AF6395E74FF4AF6185E740F214533C
:101B80004FF4FA7166E740F24C434FF4FA711BE7E9
:101B900015200BF037FE00F59671B1F52F7F96DB1F
:101BA00041F25C2399421FDD194694E741F25C2320
:101BB0009942F9DC1B4A00F5487089B2B0F52F7FD5
:101BC000118019DA4FF42F7387E740F23A72A5F5C6
:101BD000B9751A4B02FB05F583FB0523ED17A5EB41
:101BE000631389B23233BAE70E4A00F5617089B2E5
:101BF000B0F52F7F1180E5DB8342A8BF03469BB27F
:101C00006BE700BF069EFF1F029EFF1FF49CFF1F95
:101C1000BC9EFF1F589EFF1F6C9CFF1FF89CFF1F60
:101C2000789EFF1FAA9CFF1F8C9EFF1FE49CFF1F36
:101C300067BBCF46B49EFF1FAC89FF1FB5814E1B0B
:101C40002DE9F04F0C2083B00BF0A8FD0C200CF018
:101C500095F9C149DFF888A314200CF09FF9BF491A
:101C6000BF4808F067FF022103200CF02DFA022183
:101C700004200CF029FA022105200CF025FA02219B
:101C800006200CF021FA01210A200CF01DFA012196
:101C900009200CF019FA01210D200CF015FA012190
:101CA00028200CF011FA012114200CF00DFA022169
:101CB0000B200CF009FA01210C200CF005FA002190
:101CC0000C200CF0EDF9012121200CF0FDF902218E
:101CD0001C200CF0F9F901211B200CF0F5F9002172
:101CE0001B200CF0DDF91C200CF0E0F9B0FA80F3B9
:101CF0005B091A208AF800300CF026FC1F20002116
:101D00000CF0E8FB04200CF0D1F9002800F0F08082
:101D100005200CF0CBF9002800F068810023914CDD
:101D2000062023700CF0C2F9B0FA80F35B094FF083
:101D3000000B8D4A137005F0EFFF2378002B40F065
:101D4000D280584607F078FC884B894A1B88148853
:101D500088498948894DA3F5AF7240F23A7303FB75
:101D600002F381FB0321DB17A3EB61113231062360
:101D700000937B4A01600C235A2181482C7009F0A2
:101D800071FA002800F039817E4A7F481268DFF836
:101D9000549200230121FEF787FB0B200CF086F9FB
:101DA000011E0CBF0123002389F8003000F0B98028
:101DB000764F774D774EDFF8308200233B602B6003
:101DC000336004240F200DF0B9F8336803440E206B
:101DD00033600BF017FD3B6899F800201844386019
:101DE000002A79D015200BF00DFD2B6818442860CF
:101DF00004F0010080F0010004F0BEFBB8F80030F0
:101E0000002B14BF4B20DC200CF086F9013CD9D10B
:101E1000336839685D4A28685F4F002BB8BF0333C9
:101E20000029B8BF0331891011605C495C4A0988F8
:101E300014889B1000283360B8BF0330594E8210BD
:101E4000581A19442A6031603860574D574858492C
:101E5000161B22442E6002600B60BBF1000F64D1A0
:101E6000B8F80030002B4FD0524B012404201C60E6
:101E70000CF01CF918B9504B404A1C7010704F4BB5
:101E80001B881C2B58D04E4C04F1C80523200BF0A6
:101E9000B9FC44F8040F01200CF03EF9AC42F5D136
:101EA0009AF800301BB1474B1B78002B4ED1002114
:101EB00021200CF0F5F8444A444B1078187007F0D4
:101EC00057FB04F051FB4249424845F6BF5203B06C
:101ED000BDE8F04F0EF048BC11200DF02FF82B6834
:101EE0001844286084E703B0BDE8F04F08F036BD21
:101EF00006200CF0DBF800287FF40AAF194C0346EB
:101F000020704FF0010B14E74FF4FA7004F044FB1B
:101F100004F02EFB06F036FA4FF4AF600CF0FCF83C
:101F2000A2E711200CF0D0F842E7FFF735FDB8F832
:101F30000030002B98D1E7E7274B18880028A2D063
:101F4000264BC0B2197807F0CBF99CE7012121207C
:101F50000CF0A6F8AFE700BF001B374640420F0069
:101F6000E090FF1F5E9CFF1FF89DFF1FB49EFF1FA8
:101F7000909EFF1FB5814E1BAC89FF1FC09CFF1FA9
:101F8000E49CFF1F3C89FF1F209EFF1F349CFF1F06
:101F9000209CFF1F7C9EFF1F809EFF1FBC89FF1F90
:101FA0004089FF1FF49DFF1F849CFF1FC49CFF1FDF
:101FB000CC9EFF1F889EFF1F489CFF1F8E9EFF1F09
:101FC000009DFF1F089EFF1F0A9EFF1FEE9DFF1F23
:101FD000A5050000AC9EFF1FC89CFF1F789CFF1F3B
:101FE000F29DFF1F729EFF1F4E9EFF1F03200CF0ED
:101FF0005DF8B0FA80F35B0991E603200CF056F827
:102000000028FAD104200CF051F80028F5D1052061
:102010000CF04CF80028F0D106200CF047F800280E
:10202000EBD10DF0ABF800BF2DE9F04F89B005AD55
:10203000A14F2C4608AE611BC9B2A04809F0AAF80E
:102040003B88834294BF0020012004F8010BA64284
:10205000F1D19B489B4A9DF814E09B4980F800E031
:102060009DF81600994D10709DF818209DF81C30B1
:10207000974E984C0A709DF81A10297000253370FD
:10208000257073B9002940F00F81934F1AB13B7846
:10209000002B40F01F82002800F0F2810222227003
:1020A00005E0002A40F0B08005228B4F22708B4B58
:1020B000DFF888929DF815109DF81900DFF880A2CE
:1020C000DFF880B2864DDFF88082864E3A709DF848
:1020D0001EE019709DF81F209DF81D109DF817C077
:1020E0009DF81B7089F80000012000938BF800E038
:1020F00088F8001032708AF800C02F700CF01EFFB4
:1021000079497A4AD1F800E0009B7045CCBF0121A3
:10211000002111707CDD764A1288182A78D875491A
:102120000F880C3A002F78D1734993F800C00B78D0
:1021300099F800909AF800109BF8007095F800B09C
:102140002478A3EB4C03A9EB890A5B1A5344C7EB31
:10215000877AC7EB8A07DFF8A8A11F4498F80030F8
:10216000BAF800A007EB4B0796F800B03B440BFB16
:102170000A33624F4FF00C0A1AFB043AC7F800A06A
:10218000B9F1000F0BD033784BB15D4B1B88042B9A
:102190000CBF0AF1020A0AF1040AC7F800A0594B61
:1021A000594CDFF8A8B11B882488DBF800B0574FE2
:1021B000574E3F883688033BC4EBC4045C4403EBB2
:1021C0004303DFF88CB10AEB83033B44DBF800B038
:1021D000504FC6EBC60657F824404F4F5E440C3BA9
:1021E000134457F826601A193244BCF1000F27D067
:1021F0002B782BB300295BD1B9FA89F9474B4FEA09
:10220000591983F8009023E006222270324F4EE7DE
:1022100038490F880022002F86D0012F00F0CF8090
:10222000022F00F0FB80032F00F09480334F9AF8C8
:10223000001093F800C099F80090D7F800A09FE72D
:10224000364B00241C7011B198F8003023BB0021DC
:10225000334B70451970C8BF324B3349C8BFC3F800
:1022600000A00B689A4213D0304B314C1868039091
:10227000039820601B6804932E4C049B24880A60FA
:102280001B1AA34284BF2C4B1A6009B0BDE8F08F23
:102290002748264B0068EDE7BCF1000FD7D1B9F114
:1022A000000FD4D10121D3E7042222700A4FFEE6A9
:1022B0001A4B00211970CAE7B49EFF1FE49CFF1F50
:1022C000B69EFF1FB79EFF1FB89EFF1FB99EFF1F40
:1022D000BA9EFF1FFA9DFF1F049EFF1FE19EFF1F76
:1022E000E59EFF1F949EFF1FAC89FF1F409EFF1FAE
:1022F0008E9EFF1F2C9CFF1FBE89FF1F489EFF1F45
:10230000989CFF1F669EFF1F849EFF1F3E9CFF1F21
:10231000AE9CFF1F4435010020300100C69EFF1F08
:10232000C79EFF1FD09EFF1FA49CFF1FB49FFF1FCF
:10233000949CFF1F9E9EFF1FD89EFF1FE39EFF1FC2
:10234000E29EFF1FE49EFF1FE69EFF1FFC9CFF1FF7
:10235000C09EFF1F664993F800C00B7899F8009063
:102360009AF800109BF8007094F800A02C78A3EB6A
:102370004C03A9EB890B5B1A5B444FF0050B1BFB6D
:102380000733009398F800300193009BDFF86CB19D
:10239000C7EBC707BA440533019FBBF800B003EB96
:1023A000440334783B4404FB0B33524C524F54F8F3
:1023B0002A400C3303EB040AC7F800A0E0E64C49BE
:1023C00093F800C00B7899F800909AF800109BF8E9
:1023D000007095F800A02478A3EB4C03A9EB890BBF
:1023E0005B1A5B44C7EB877BC7EB8B07DFF80CB14D
:1023F0003B4498F80070BBF800B003EB4A0A33780E
:10240000BA44C4F1060403FB0BA3E4B24FF00C0A78
:10241000394F1AFB043AC7F800A0B1E6344993F8E3
:1024200000C00B7801932B780093019B9AF8001061
:1024300099F800909BF800A02478A3EB4C03A9EB3B
:10244000890B5B1A5B44A3F1020B2C4BCAEBCA0A43
:1024500054441B88DFF8C8A00193BDF800305AF837
:1024600024A098F8004017FB03BB3778019B5C441D
:1024700007FB03431833204F9A44C7F800A07FE6B8
:10248000BEF1000F29D13A78012A2FD91C4B2270B6
:102490001B882BB31B4B1B88013B9BB2062B1FD801
:1024A000194B1B78E3B1194B1B68012B7FF4FFAD6F
:1024B0001749184B0968184D83FB0130CB17C3EB44
:1024C000600303EB4303A1EB83032B80134B032136
:1024D0001970ECE503222270E9E501222270E6E59D
:1024E0000A4B1B68012B7FF4E2ADEFE77246DEE595
:1024F000BE89FF1FC8380100489EFF1F989CFF1F20
:10250000709EFF1F0C9EFF1FF69CFF1F889EFF1FE3
:10251000D89EFF1FABAAAA2A4C9EFF1FA089FF1FAF
:10252000303701002DE9F04F3A4B1B788BB0002B70
:102530006BD10E200BF066F90FF0A2FA0146364877
:10254000364E374DFDF7F6FF3348FDF7C9FF0FF064
:10255000B1FC80F30C003060FFF766FD2C68012CA5
:102560007AD0022C00F0BD82032C00F0CF832D4ED8
:102570002D4C33682D4A2E4E0993099B31681288E1
:102580002360591A013A9142274F00F2A582294E41
:1025900032689A1A0D2A00F28E82274E32689A1AF1
:1025A000132A00F28382254E32689A1A252A1AD9F4
:1025B000234B1B88002B40F06481224B1B78002B9F
:1025C00040F05F81FEF74AFE1F4B1B881B3B9BB20E
:1025D000022B04D81D4B1B78002B40F0558103F0D3
:1025E000EDFF236833601A4D2A689B1A502B00F2C6
:1025F0001982184B1B88012B00F0318206F016FE61
:1026000006F0FAFC0BB0BDE8F08F08F033F80BB021
:10261000BDE8F08F5E9CFF1F209EFF1F5C9EFF1F8A
:10262000889EFF1FB49FFF1F1C9EFF1FA889FF1FCE
:10263000F09CFF1FD89CFF1FB89CFF1FBC9CFF1F76
:10264000009EFF1F589CFF1F8E9EFF1F409EFF1F76
:10265000109EFF1F609EFF1FDFF83893A44AB9F851
:1026600000001378834204D0C3B21846137006F0FA
:10267000CFFDDFF81C839F4AB8F8003011789942EB
:1026800004D09D4F3978002940F0FC869B4A33687E
:1026900012889B4E9A42C0F201819A4A1278002A0F
:1026A00040F0FC80DFF8F0A2BAF8003023B9964B76
:1026B0001B88002B00F01285944A954B11881B88CB
:1026C000944A0B4412685B109342934A126880F25A
:1026D000B48400219342B4BF01230B4604910093BC
:1026E000ACBF4FF0010B8B4605910E200BF08AF822
:1026F0008A4B8B4A1B68176803930133A7F2523247
:10270000002B8446029240F3CE86802BA8BF802304
:10271000844A854912780191002A00F0C98009781D
:10272000914200F0C580B8F80010DFF864E29942E9
:1027300001F0B7807049AEF800307C4B4FF0010ECD
:1027400081F800E01978DFF854E2019B8EF8001060
:102750001A70009B002B00F02381BAF80030002B88
:1027600000F01E81724B1B685A1C002A40F39F86A2
:10277000802A00F39B866F4C6F4970482488098833
:1027800000682144B0EB610FC1F2FF82A3F148025F
:102790000F2A02D8473BA9F800300E200BF032F880
:1027A0006FF454731F44874202DC654B00221A7099
:1027B00000200CF0C3FB634A634B1168634C1B8819
:1027C0008842D4BF002201222270002B00F02C840A
:1027D0005F4B1C78944243D0884241DD5D490C78C0
:1027E000002C00F028875C4991F800C0BCF1000F74
:1027F00040F01F87594F0097594F5A480297574F3B
:10280000007887F800C0564F4FF0010E87F800C0DF
:1028100081F800E0002841F09480534909780029AC
:1028200000F0E887514903910C460978002940F0EF
:10283000DE874F484A4F0078397001210297217096
:1028400070B14648444900904A4803270770002069
:1028500008700099029F0870039901243C70087069
:102860001A70454B1B88A3F11B02012A40F2CE854A
:102870001D2B7FF47DAE3E4A404B12781A70404CBF
:1028800077E6FEF78DFC9DE63E4B1B78002B3FF470
:10289000A6AE2B68012B7FF4A2AEA2E631683A4ABD
:1028A000069106983949106002220B602A60F9E609
:1028B0001E49DFF8E8E0097800293FF446AF9EF8AA
:1028C000000081423FF441AF03984B2840F3B087AA
:1028D0001833802BB8F80000A8BF802398423FF43B
:1028E00034AF2B4803800448012303702DE700BF59
:1028F000EE9DFF1FC09CFF1F489CFF1FF49CFF1F05
:10290000B49FFF1F589CFF1FDE9CFF1F6C9CFF1F86
:10291000589EFF1F8C9CFF1F509CFF1FD09EFF1FC7
:10292000349CFF1FC69EFF1FA09CFF1FC79EFF1F5A
:10293000489EFF1F069EFF1F029EFF1F7C9CFF1FDD
:10294000F99DFF1FAC89FF1F0C9EFF1F729CFF1F8C
:10295000249CFF1FE49EFF1F509EFF1FA29EFF1F8F
:10296000F69CFF1FE59EFF1FE19EFF1F259CFF1F9A
:10297000409EFF1FA089FF1F8E9EFF1F409CFF1FD0
:102980001C9EFF1F949EFF1FB09CFF1F189EFF1FE1
:10299000909EFF1F0A9EFF1FA89CFF1FA19CFF1F68
:1029A000029B9C45BFF6F9AE8B4B1B88002B3FF476
:1029B000F4AEBBF1000F7FF4D5AE884B1B881BB182
:1029C000059B002B7FF4CEAE049B002B3FF4E5AEBD
:1029D000834B1A78002A7FF4E0AEDFF8809299F8F2
:1029E000004001221A70002C40F045837D4B1B787B
:1029F000002B02F060807C4B1B78002B02F03E83A2
:102A00007A4B1B78002B7FF4C8AE794B1B78002BD8
:102A10003FF4C3AEB8F8003076490A3BA8F800305E
:102A20000A70BAE605F0C0F9734B1B7873B9734BA3
:102A30001B785BB9724B1B7843B9724B1B782BB96F
:102A4000714B1B7813B903F08FFD01E003F098FD83
:102A500023682B606D4B1B88012B7FF4CFAD6C4A34
:102A60006C4B11686C481A78A1F118032A2101FBFC
:102A700003F10160002A00F0C182684C236899428A
:102A800000F36A8310DA66480278002A40F046872D
:102A9000644A1068D0F17F0048BF033080100130D5
:102AA0001B1A994242F34E862160A9E2FEF7CAFE44
:102AB0002368336077E5FDF763FFFEF7FBFB5A4BB6
:102AC0001B88032B00F01385584B1B88032B00F049
:102AD0000A852368336060E5FDF79EFE3B6833603E
:102AE00055E5534A34681188A14204DB464B1B78F4
:102AF000002B00F061834F4E4F48336807934F4BD4
:102B0000079A00681B88121A9A4200F2AD80002BC7
:102B100000F0AA804A4B1A88002A3FF429AD494B9D
:102B200049481B680088A342B8BF2346994241F335
:102B30002281464B1960DFF8288188F80020344F45
:102B4000FDF76AFE38687F2840F36F85404B7F3879
:102B500083FB0032C317C3EB620303EB4303A0EB19
:102B6000830073303B4B01931B883860002B40F08F
:102B70009186234B00931B78002B00F0C883364CC2
:102B80002378002B00F0C383DFF8D890DFF8C0A0D3
:102B90004FF0000B0CE003F17300C0B298F8001086
:102BA00006F0CEFB23780BF1010B5B4540F3AF83BE
:102BB0003B6859F8040F1844A0F17F038AFB0321F6
:102BC000DA17C2EB610202EB42027F28A3EB820319
:102BD000E1DCFDF741FDE0E7DE9CFF1F149EFF1FD7
:102BE000F99DFF1FE19EFF1FE29EFF1FE39EFF1F57
:102BF000E49EFF1F489CFF1FF69CFF1F509EFF1F77
:102C0000A29EFF1F259CFF1F589CFF1F609EFF1F59
:102C1000D89EFF1FAC9CFF1FD09CFF1FE09CFF1F96
:102C2000A89EFF1FA49EFF1F629EFF1FF09DFF1F17
:102C3000F49CFF1FB49FFF1FB09CFF1FDC9CFF1F75
:102C4000429CFF1F189EFF1FBC9EFF1F289CFF1F5A
:102C5000ABAAAA2A889CFF1F6889FF1FFA9DFF1F45
:102C6000CC9CFF1F4089FF1F554B564A1B6810889C
:102C7000554AA342B8BF2346994200F38482534C7D
:102C800012888342A8BF03462360002A7FF453AF13
:102C90009942C8BF134640F37D82401AB0F5804F79
:102CA000AABF9B03C3EB8333013093FBF0F0FDF726
:102CB00099FDC0F3C6100EF0E3FE454B044618889C
:102CC0000EF0DEFE4349074620460EF02DFF01467A
:102CD00038460EF029FF21460EF01EFE4FF07E51C1
:102CE00004460FF0BFF8002841F03A803A492046E8
:102CF0000FF0D6F8002840F01E8620460FF000F9AD
:102D0000C0B2DFF8F48088F8000018E7334B34686D
:102D10001988A14274DD324B1B78002B70D1DFF88B
:102D2000DC9099F800007F2840F3F485A3F1553337
:102D30007F3803F1004383FB0032C317C3EB620308
:102D400003EB4303A0EB83007330264B01931B88F6
:102D5000C0B289F80000002B40F0E387224B0093BB
:102D60001B78002B00F09484204C2378002B00F07B
:102D70008F841F4FDFF87C804FF0000A0AE003F1D8
:102D80007300C0B206F000FB23780AF1010A534534
:102D900040F37E8457F8043F99F800001844A0F1EE
:102DA0007F0388FB0321DA17C2EB610202EB4202C8
:102DB0007F28A3EB8203E2DCFDF74EFCE1E700BFD6
:102DC000189EFF1FBC9EFF1F429CFF1F289CFF1FD9
:102DD000C89EFF1FCDCCCC3D0000FE42F49CFF1FDF
:102DE000589CFF1F889CFF1FA29EFF1F6889FF1F22
:102DF0004089FF1FABAAAA2ACC9CFF1F449EFF1F3D
:102E0000B84F38687F2840F3CC81B74B7F3883FBBD
:102E10000032C317C3EB620303EB4303A0EB830051
:102E20007330DFF8249399F800A0824500F01582F2
:102E3000AE4B1B88002B43D1AD4AAE4812680088C8
:102E4000914205DC8242D4BFC1EB0203C1EB000317
:102E5000411AB1F5804FA6BF9B030131C3EB833309
:102E600093FBF1F0FDF7BEFCC0F3C6100EF008FEB8
:102E7000A14B044618880EF003FEA0498046204668
:102E80000EF052FE014640460EF04EFE21460EF078
:102E900043FD4FF07E5104460EF0E4FF002840F061
:102EA000BA86974920460EF0FBFF002840F0408587
:102EB00020460FF025F8C0B2DFF8908288F80000B5
:102EC000BAF17F0F40F3A3838748AAF17F0A80FB02
:102ED0000A304FEAEA73C3EB600000EB4000AAEB54
:102EE00080007330874B00931B78C0B289F80000D4
:102EF000002B40F00383844B03931B78002B40F09E
:102F0000EC84824B02931B78002B40F02C87804B83
:102F10000193029B1B78FBB17E4B1B88012B00F0B9
:102F2000F885022B00F08087032B01F02181042B10
:102F300001F02183052B01F0C183062B01F0878569
:102F4000072B01F04387082B02F04980092B02F080
:102F500010810A2B02F01083009B1B78002B00F0DD
:102F60005984019B6A4C1988002900F0AF843868A5
:102F70007F2840F3C0825C4B7F3883FB0032C3174D
:102F8000C3EB620303EB4303A0EB830073303860B1
:102F9000002940F05E84009B1B78002B00F06981C3
:102FA0005D4C2378002B00F06481DFF8A4A1DFF8EA
:102FB0009C814FF0000B0CE003F17300C0B298F855
:102FC000001006F0BDF923780BF1010B5B4540F3CF
:102FD00050813B685AF8040F434A1844A0F17F031C
:102FE00082FB0321DA17C2EB610202EB42027F2867
:102FF000A3EB8203E0DCFDF72FFBDFE7474B196013
:10300000474B1B68A92202FB03F3002BBCBF03F54F
:103010007F533F339B13543B194481F30C01282009
:103020000AF0AEFEFFF7EABA384C3E483549364A58
:10303000237003700B70137013E493424FF0000B76
:1030400080F2B2800123CDF800B0CDF814B0049323
:10305000FFF74BBB344B1B78002B7FF49EAB039BDD
:10306000324A243B83F34703D9B25B20136006F056
:1030700037F999F80040032C30D1DFF8D88098F860
:103080000030002B42F0E381294F3B78002B42F0C7
:10309000D181254C2378002B42F0BF81254B1B7832
:1030A000002B42F0AD81244A1380244B1B78002B67
:1030B00042F0FF800D4B7F221A8098F800306BB9E8
:1030C0003B785BB923784BB91D4A7F2107201380D9
:1030D00006F006F97F210B2006F002F9194B1F6854
:1030E000FFF75BBBD89EFF1FABAAAA2A429CFF1F1B
:1030F000289CFF1FBC9EFF1FC89EFF1FCDCCCC3D50
:103100000000FE42A29EFF1F259CFF1FF69CFF1F92
:10311000889CFF1F0C9EFF1F6889FF1FE09CFF1FFC
:10312000A489FF1F509EFF1FE49EFF1F689CFF1F86
:10313000E39EFF1FE29EFF1FEA9CFF1FE59EFF1F0D
:10314000429EFF1F349CFF1F449EFF1FCC9CFF1F0D
:103150004089FF1FE19EFF1FB54A1078002840F00C
:103160003D83B44A1268D2F17F0248BF033203EBB9
:10317000A202531CB04A23609942B8BF1160FFF607
:103180003FAF19463CE7AD4B12881960002A7FF427
:10319000D2AC0B469842D4BFC1EB0003C1EB030392
:1031A0007BE5FDF759FA3CE60123CDF810B0CDF8E8
:1031B00000B00593FFF799BA01232B60FFF7D7B949
:1031C000029B1B78FBB19E4B1B88012B00F01A84DD
:1031D000022B00F0A786032B01F04080042B01F0A6
:1031E000EF81052B01F0E082062B01F03984072BDB
:1031F00001F03985082B01F0A386092B02F022800B
:103200000A2B02F07F81019B1B88002B00F02A8390
:10321000009B1B783BB9039B1B7823B9029B1B784F
:10322000002B00F09B87874B1B78002B00F0FE8063
:1032300085490B78082B00F2F98084483A680068C9
:10324000834C0133DBB25F1E101A44F827000B7069
:10325000804B3468198889F800208C427E4E7FF7B5
:1032600087A932687D4B0892089A7D4C1A60FFF757
:1032700080B9039B1B78002BA2D03B68A3F10C0004
:103280007F2840F3338377488B3B80FB0320DA179A
:10329000C2EB600000EB4000A3EB800303F173007E
:1032A000DFF8D481C0B298F8001006F049F8009B0E
:1032B0001B78002B84D0644C2378002B80D0DFF85F
:1032C000BCA14FF0000B0CE003F17300C0B298F802
:1032D000001006F035F823780BF1010B5B457FF702
:1032E0006FAF3B685AF8040F5E4A1844A0F18B0395
:1032F00082FB0321DA17C2EB61020C3802EB4202B7
:103300007F28A3EB8203DFDCFDF7A6F9DEE74D4B58
:103310001B78002B40F0AC823B68534A1278002A9D
:1033200045D0A3F10C007F2840F3F1824D4A8B3B3E
:1033300082FB0321DA17C2EB610202EB4202A3EB2C
:10334000820303F17300C0B298F8001005F0F8FF93
:10335000009B1B7853B33C4C23783BB3DFF81C91A4
:10336000DFF800A14FF0000B0BE003F17300C0B2D7
:1033700098F8001005F0E4FF23780BF1010B5B4592
:1033800014DD3B6859F8040F1844A0F18B038AFB45
:103390000321DA17C2EB61020C3802EB42027F28EC
:1033A000A3EB8203E1DCFDF757F9E0E73B682F4A26
:1033B0001278FAB1224A1288012A00F02F84022AD8
:1033C00000F03186032A00F0C687042A01F01F812D
:1033D000052A01F05C82062A01F06683072A01F0C3
:1033E0009D83082A01F05D86092A01F0F9860A2AE0
:1033F00002F05480019A1288002A00F044821C4A8C
:10340000174C137003232B60FFF7B3B8DFF87080FD
:1034100098F80030002B40F0FE80164F3B78002BD0
:1034200040F0C6840E4C3B70FFF7A3B83A680FE734
:10343000A89EFF1FA49EFF1FE09CFF1F289CFF1F4C
:103440000C9EFF1F509EFF1F6889FF1F4C9CFF1F93
:103450004489FF1FF49CFF1FB49FFF1F809FFF1F25
:103460001C9EFF1FABAAAA2A259CFF1FF69CFF1FCC
:10347000449EFF1F409CFF1FCC9CFF1F4089FF1FE5
:10348000409EFF1FDBB21846137005F0E7FFA54B07
:10349000A5491A46A54B184600230B703B701370C4
:1034A0000370FFF7F3B80123FFF732B98024A04976
:1034B000A04BA14A09881B8812680B44B2EB630F2A
:1034C000BFF66BA99D4B1B78002B40F0F081B8F83C
:1034D00000309B4AA3423FF460A99A4B148001221A
:1034E0001A70FFF75AB9FDF71FF9FFF7F2BAFDF7A7
:1034F000C5F8FFF7E9BAFDF7AFF848E5924B01933D
:103500001B8863BB894B0393904B0293904C2378A9
:103510007BB3DFF85882DFF83CA24FF0000B09E0E4
:1035200003F17300C0B205F02FFF23780BF1010BFC
:103530005B451EDD58F8043F99F800001844A0F1DF
:103540007F038AFB0321DA17C2EB610202EB42021E
:103550007F28A3EB8203E3DCFDF77EF8E2E7734B01
:1035600003937A4B029305F00FFF009B1B78002B0F
:10357000CCD1039B1B78002B3FF4CBAC99F80030E7
:10358000A3F10C007F2840F3BF8172488B3B80FB86
:103590000320DA17C2EB600000EB4000A3EB8003CE
:1035A00003F17300C0B205F0EFFE009B1B78002B07
:1035B00000F09F81664C2378002B01F05D82DFF8DC
:1035C000AC81DFF890A14FF0000B0AE003F173002B
:1035D000C0B205F0D9FE23780BF1010B5B457FF7F4
:1035E00098AC58F8043F99F800001844A0F18B03F8
:1035F0008AFB0321DA17C2EB61020C3802EB4202AC
:103600007F28A3EB8203E1DCFDF726F8E0E75046D4
:10361000FDF722F866E4504A1278002A40F09E81B5
:103620004E4F4F4C3B70FEF7A4BFFDF715F8FFF768
:1036300099BA002008704B49087840B13949009187
:103640000978002900F07A81009F002139704649ED
:10365000097800297FF4E6A8002C40F0CB800028F0
:1036600040F0C880354C2F4F94F800E02F4C039465
:10367000364C02942D4C2C492070344C0097087025
:1036800038702070BEF1000F7FF4DEA8FFF7E8B8B5
:10369000264B1B78002B6BD099F80030A3F10C005F
:1036A0007F2840F390832B4A8B3B82FB0321DA1760
:1036B000C2EB610202EB4202A3EB820303F173004F
:1036C000C0B205F061FE009B1B78002B50D0204C4F
:1036D0002378002B4CD0254FDFF878804FF0000A7C
:1036E00009E003F17300C0B205F04EFE23780AF141
:1036F000010A53453CDD57F8043F99F8000018448F
:10370000A0F18B0388FB0321DA17C2EB61020C38AE
:1037100002EB42027F28A3EB8203E2DCFCF79CFF72
:10372000E1E700BFA29EFF1F509EFF1F259CFF1FC9
:10373000069EFF1F029EFF1F7C9CFF1F409EFF1FD7
:10374000909EFF1F489CFF1F889CFF1FF69CFF1F39
:103750006889FF1FABAAAA2A949EFF1F409CFF1FE7
:103760001C9EFF1FE59EFF1FE19EFF1F4089FF1F5C
:10377000904B1B78FBB1904B1B88012B00F074869B
:10378000022B00F06E87032B01F0E480042B01F084
:103790007E81052B01F0B983062B01F05484072BA1
:1037A00001F09485082B01F01087092B01F07E872A
:1037B0000A2B01F05C87019B1B88002B00F0BA826A
:1037C0007E4B1B78002B40F0B0827D4B7D4A1988E0
:1037D00034680020012310602B603EE50130C0B248
:1037E000022886BF002111701070194608E4039862
:1037F000002101707449097800293FF431A86D490E
:1038000002910978002900F0528702980021017086
:10381000FFF726B8039B1B78002B7FF4A2AB029B1B
:103820001B78002B7FF49DAB019B1988FFF79FBB92
:10383000243B002BB8F8000040F3748498423EF417
:1038400084AF9BB26148A8F8003001230370FEF7F3
:103850007CBFDFF87C81C0B298F8001005F070FDE5
:10386000FFF799BB5A4B3878197805F069FDCFE41A
:103870007F21402005F034FD5649574A3B680B60D4
:103880000021117049E5D8B298F8001005F058FDF4
:103890003B68B4E5C0B298F8001005F051FDFFF7A1
:1038A00068B94E4BDFF854E11978FEF74EBF4B2C48
:1038B00040F345821834802CB8F80030484AA8BF3D
:1038C0008024A3427FF409AEFEF767BF99F8000099
:1038D00005F05AFD2188FFF74ABB424B01931B8834
:1038E000002B41F03387334B029347E6FCF7B4FEDD
:1038F000D6E4029B1B78002B7FF40EAB039B1B7856
:10390000002B7FF42EAB8FE7FCF7A6FE4AE6FCF710
:10391000A3FE18E5FCF7A0FEFFF717BA0132D2B2FA
:10392000022A40F25682002202701946FFF768BB55
:103930007F20FFF7C1BA7F20FFF7E3B91D4F1F4972
:1039400002974FF0000C81F800C0009F02994FF0E1
:10395000010E87F800E081F800C078E6224F387841
:1039600002F07CFE214B1B78002B00F040823B884C
:103970007E2B00F23C821E4CDFF884902268D9F83E
:103980000010521A0F2A40F229821A4A0133108875
:1039900099B23980002800F04382C9B2C0B205F064
:1039A0009FFC154F226898F80030C9F800203B7042
:1039B000FEF7DFBDF69CFF1F0C9EFF1F509EFF1FF2
:1039C000F49CFF1F289CFF1F409EFF1F489CFF1F69
:1039D000CC9CFF1F4C9CFF1F6889FF1FC79EFF1FC9
:1039E000909EFF1F889CFF1F789CFF1FE69EFF1F75
:1039F0001C9EFF1FC89CFF1F409CFF1FA19CFF1F18
:103A0000D49EFF1FDFF89CA33868BAF80030E04A64
:103A1000E04CC31A82FB031ED917C1EB6E0101EB08
:103A20004101A3EB810303EB430354F82330184413
:103A30007F2840F307857F3882FB0032C317C3EB32
:103A4000620303EB4303A0EB83007330DFF858837A
:103A5000DFF858B398F80010C0B205F071FCBBF85D
:103A60000030022B7FF6CFAB3968BAF80030C84A75
:103A7000CB1A82FB030ED817C0EB6E0000EB4000A0
:103A8000A3EB800303EB430304EB83035868084470
:103A90007F2840F3EE867F3882FB0032C317C3EBEA
:103AA000620202EB4202A0EB82007330C0B298F8CF
:103AB000001005F045FCBBF80030032B7FF6A3ABEC
:103AC0003968BAF80030B24ACB1A82FB030ED81715
:103AD000C0EB6E0000EB4000A3EB800303EB43035D
:103AE00004EB8304A06808447F2840F37D817F387D
:103AF00082FB0032C317C3EB620202EB4202A0EB6F
:103B00008200733098F80010C0B205F019FCFFF77E
:103B10007ABBDFF890A299F80000BAF800309C4A0E
:103B20009C4CC31A82FB031ED917C1EB6E0101EB3B
:103B30004101A3EB810303EB430354F82330184402
:103B40007F2840F305847F3882FB0032C317C3EB24
:103B5000620303EB4303A0EB83007330DFF84CB246
:103B6000C0B205F011FCBBF80030022B7FF6F4A9BF
:103B700099F80010BAF80030854ACB1A82FB030E80
:103B8000D817C0EB6E0000EB4000A3EB800303EB03
:103B9000430304EB8303586808447F2840F36D8691
:103BA0007F3882FB0032C317C3EB620202EB420292
:103BB000A0EB82007330C0B205F0E6FBBBF800302A
:103BC000032B7FF6C9A999F80010BAF80030704AA3
:103BD000CB1A82FB030ED817C0EB6E0000EB40003F
:103BE000A3EB800303EB430304EB8304A0680844C6
:103BF0007F2840F3C7807F3882FB0032C317C3EBB6
:103C0000620202EB4202A0EB82007330C0B205F008
:103C1000BBFBFFF7A1B90120FFF74EB9DFF884A184
:103C20005B49BAF800205B4C9A1A81FB020ED01750
:103C3000C0EB6E0000EB4000A2EB800202EB420200
:103C400054F8220018447F2840F30084A0F17F0339
:103C500081FB0321DA17C2EB610000EB4000A3EB0C
:103C600080007330DFF844B198F80010C0B205F05E
:103C700067FBBBF80030022B50D93968BAF8003026
:103C8000434ACB1A82FB030ED817C0EB6E0000EB41
:103C90004000A3EB800303EB430304EB830358686A
:103CA00008447F2840F3B9867F3882FB0032C3176F
:103CB000C3EB620202EB4202A0EB82007330C0B29F
:103CC00098F8001005F03CFBBBF80030032B25D919
:103CD0003868BAF800302E4AC31A82FB031ED9177F
:103CE000C1EB6E0101EB4101A3EB810303EB430345
:103CF00004EB8304A36818447F2867DD7F3882FBC8
:103D00000032C317C3EB620202EB4202A0EB820057
:103D10007330C0B298F8001005F012FB3B68FFF753
:103D200069BB05F031FBFFF719B80021402005F011
:103D3000D7FA4AE599F8000005F026FB40E5243C57
:103D4000002CB8F8003040F39C85A3423EF425AD2A
:103D5000A4B2114BA8F8004001221A70FEF71DBD55
:103D60000120FEF7CEBF0D4B01931B88002B3FF4C3
:103D7000D0A8FFF7F8BB0A498342A8BF03460B60EF
:103D8000FEF7D9BEFCF768FC40E71446FFF79ABB84
:103D9000ABAAAA2A24340100489CFF1F889CFF1F5D
:103DA000289CFF1F4C9EFF1FCC9CFF1F5C9CFF1F8D
:103DB000DF4BE04C19886A2005F014FC98F80030BD
:103DC0003B70FEF7D6BBFCF747FC79E4FCF744FCFC
:103DD0009FE702701946FFF713B9D64CD64F98F8F3
:103DE00000303B70FEF7C5BBFCF736FC8AE6D34BD0
:103DF0001B78002BF1D03B88CD4F002BEDD0CD4C64
:103E0000DFF848932268D9F80010521A0F2AE5D932
:103E1000CB4A013B108899B2398000287FF4BDADB0
:103E2000C8B205F0FDFABCE5DFF824A399F800005C
:103E3000BAF80030C34AC44CC31A82FB031ED91718
:103E4000C1EB6E0101EB4101A3EB810303EB4303E3
:103E500054F8233018447F2840F3FD837F3882FBD9
:103E60000032C317C3EB620303EB4303A0EB8300F1
:103E70007330DFF8E0B2C0B205F086FABBF800306C
:103E8000022B7FF669A899F80010BAF80030AD4A05
:103E9000CB1A82FB030ED817C0EB6E0000EB40007C
:103EA000A3EB800303EB430304EB8303586808444C
:103EB0007F2840F3DD857F3882FB0032C317C3EBD8
:103EC000620303EB4303A0EB83007330C0B205F041
:103ED0005BFABBF80030032B7FF63EA899F8001080
:103EE000BAF80030974ACB1A82FB030ED817C0EB02
:103EF0006E0000EB4000A3EB800303EB430304EBF5
:103F00008304A06808447F287FF73CAF7F3882FB9A
:103F10000032C317C3EB620303EB4303A0EB830040
:103F2000733073E6DFF828A23868BAF80030854AA3
:103F3000854CC31A82FB031ED917C1EB6E0101EB3E
:103F40004101A3EB810303EB430354F823301844EE
:103F50007F2840F359837F3882FB0032C317C3EBBD
:103F6000620303EB4303A0EB83007330DFF8E881C7
:103F7000DFF8E0B198F80010C0B205F0E1F9BBF845
:103F80000030022B7FF63FA93968BAF800306D4A3D
:103F9000CB1A82FB030ED817C0EB6E0000EB40007B
:103FA000A3EB800303EB430304EB8303586808444B
:103FB0007F2840F368857F3882FB0032C317C3EB4C
:103FC000620303EB4303A0EB83007330C0B298F8A5
:103FD000001005F0B5F9BBF80030032B7FF613A9EC
:103FE0003868BAF80030574AC31A82FB031ED91743
:103FF000C1EB6E0101EB4101A3EB810303EB430332
:1040000004EB8304A36818447F287FF7EDAE7F3864
:1040100082FB0032C317C3EB620303EB4303A0EB45
:10402000830073306EE5DFF828A14649BAF8002016
:10403000454C9A1A81FB020ED017C0EB6E0000EBC4
:104040004000A2EB800202EB420254F82200184426
:104050007F2840F30383A0F17F0381FB0321DA175C
:10406000C2EB610000EB4000A3EB80007330DFF88F
:10407000E4B098F80010C0B205F062F9BBF8003067
:10408000022B7FF64BAE3968BAF800302D4ACB1AB6
:1040900082FB030ED817C0EB6E0000EB4000A3EBD1
:1040A000800303EB430304EB8303586808447F2831
:1040B00040F3F6847F3882FB0032C317C3EB620300
:1040C00003EB4303A0EB83007330C0B298F80010F9
:1040D00005F036F9BBF80030032B7FF61FAE3868C9
:1040E000BAF80030174AC31A82FB031ED917C1EB76
:1040F0006E0101EB4101A3EB810303EB430304EBEE
:104100008304A36818447F287FF760AE7F3882FB62
:104110000032C317C3EB620303EB4303A0EB83003E
:104120007330F6E501283EF410AB0123FFF78ABB9C
:10413000789CFF1F1C9EFF1F409CFF1FE59EFF1FDA
:10414000C89CFF1FABAAAA2AEC350100D49EFF1F12
:104150004C9EFF1F5C9CFF1FCC9CFF1F4FF47A43BB
:10416000013BFDD199F8000005F00EF9FFF75BB8AF
:10417000DFF8E8A299F80000BAF80030B54AB64C6A
:10418000C31A82FB031ED917C1EB6E0101EB41017B
:10419000A3EB810303EB430354F8233018447F2837
:1041A00040F3DD817F3882FB0032C317C3EB62022C
:1041B00002EB4202A0EB82007330DFF8A4B2C0B27F
:1041C00005F0E2F8BBF80030022B7EF6C5AE99F898
:1041D0000000BAF800309F4AC31A82FB0321DA17A5
:1041E000C2EB610202EB4202A3EB820303EB430347
:1041F00004EB83035B6818447F2840F312847F3804
:104200000C2290FBF2F302FB13007330C0B205F0F6
:10421000BBF8BBF80030032B7EF69EAE99F8000089
:10422000BAF800308B4AC31A82FB0321DA17C2EBBB
:10423000610202EB4202A3EB820303EB430304EBB4
:104240008304A36818447F287FF79CAD7F380C2235
:1042500090FBF2F302FB13007330D7E4DFF8FCA10C
:104260003868BAF800307B4A7B4CC31A82FB031EC5
:10427000D917C1EB6E0101EB4101A3EB810303EB05
:10428000430354F8233018447F2840F365817F3876
:1042900082FB0032C317C3EB620202EB4202A0EBC7
:1042A00082007330DFF8BC81DFF8B4B198F80010F9
:1042B000C0B205F045F8BBF80030022B7EF6A3AF84
:1042C0003868BAF80030634AC31A82FB0321DA1750
:1042D000C2EB610202EB4202A3EB820303EB430356
:1042E00004EB83035B6818447F2840F3A7837F387F
:1042F0000C2290FBF2F302FB13007330C0B298F86B
:10430000001005F01DF8BBF80030032B7EF67BAFE4
:104310003868BAF800304F4AC31A82FB0321DA1713
:10432000C2EB610202EB4202A3EB820303EB430305
:1043300004EB8304A36818447F287FF755AD7F38CA
:104340000C2290FBF2F302FB13007330FFF7DABB91
:10435000FCF782F902E4DFF804A13E49BAF8002034
:104360003D4C9A1A81FB020ED017C0EB6E0000EB99
:104370004000A2EB800202EB420254F822001844F3
:104380007F2840F3EF80A0F17F0381FB0321DA1740
:10439000C2EB610101EB4101A3EB81007330DFF857
:1043A000C0B098F80010C0B204F0CAFFBBF80030EB
:1043B000022B7FF6B3AC3868BAF80030254AC31A2E
:1043C00082FB0321DA17C2EB610202EB4202A3EB8C
:1043D000820303EB430304EB83035B6818447F28E9
:1043E00040F32F837F380C2290FBF2F302FB130083
:1043F0007330C0B298F8001004F0A2FFBBF8003090
:10440000032B7FF68BAC3868BAF80030114AC31A18
:1044100082FB0321DA17C2EB610202EB4202A3EB3B
:10442000820303EB430304EB8304A36818447F284F
:104430007FF7CCAC7F380C2290FBF2F302FB130029
:10444000733066E4FCF708F9FFF700BBFCF704F9EA
:1044500008E400BFABAAAA2A7C3601004C9EFF1FCD
:104460005C9CFF1FCC9CFF1FDFF834A399F8000071
:10447000BAF80030C24AC34CC31A82FB0317D917DB
:10448000C1EB670101EB4101A3EB810303EB4303A4
:1044900054F8233018447F286ADD7F3882FB0032CD
:1044A000C317C3EB620202EB4202A0EB820073303F
:1044B000DFF8F0B2C0B204F067FFBBF80030022BA7
:1044C0007FF679A999F80000BAF80030AC4AC31A0F
:1044D00082FB0321DA17C2EB610202EB4202A3EB7B
:1044E000820303EB430304EB83035B6818447F28D8
:1044F00040F3AA827F380C2290FBF2F302FB1300F8
:104500007330C0B204F040FFBBF80030032B7FF6DD
:1045100052A999F80000BAF80030994AC31A82FBF0
:104520000321DA17C2EB610202EB4202A3EB820322
:1045300003EB430304EB8304A36818447F2814DDD2
:104540007F380C2290FBF2F302FB13007330C0B2F1
:1045500004F01AFFFFF72FB9FCF77EF8A2E6FCF78C
:104560007BF82AE6FCF778F819E7FCF775F8EEE730
:10457000FCF772F89CE7DFF828A299F80000BAF877
:1045800000307F4A804CC31A82FB031ED917C1EB4F
:104590006E0101EB4101A3EB810303EB430354F8EC
:1045A000233018447F28DADD7F3882FB0032C317BE
:1045B000C3EB620303EB4303A0EB83007330FCE522
:1045C000DFF8DCA13868BAF800306D4A6E4CC31AC7
:1045D00082FB031ED917C1EB6E0101EB4101A3EB76
:1045E000810303EB430354F8233018447F28B3DDE1
:1045F0007F3882FB0032C317C3EB620303EB430334
:10460000A0EB830073304DE6FCF726F8AEE4DFF84C
:1046100090A15B49BAF800205B4C9A1A81FB020E0C
:10462000D017C0EB6E0000EB4000A2EB800202EB63
:10463000420254F8220018447F2893DDA0F17F0342
:1046400081FB0321DA17C2EB610000EB4000A3EB12
:1046500080007330A3E6FBF7FFFF0AE4FBF7FCFFE3
:1046600005E5DFF83CA199F80000BAF80030444AAB
:10467000464CC31A82FB0317D917C1EB670101EB44
:104680004101A3EB810303EB430354F823301844A7
:104690007F287FF76DAF7F3882FB0032C317C3EBF3
:1046A000620303EB4303A0EB8300733000E7384859
:1046B0000090384838490390FEF7C6B8DFF8E0A00C
:1046C00099F80000BAF800302D4A344CC31A82FB26
:1046D0000321DA17C2EB610202EB4202A3EB820371
:1046E00003EB430354F8233018447F2840F3A081A0
:1046F0007F380C2290FBF2F302FB13007330DFF8DB
:10470000A4B0C0B204F040FEBBF80030022B19D9AF
:1047100099F80000BAF800300C22C11A91FBF2F3AC
:1047200002FB131302FB03435B6818447F2840F32A
:1047300052847F3890FBF2F302FB13007330C0B257
:1047400004F022FEBBF80030032B7EF605ACBAF86D
:10475000003099F800000C22C11A91FBF2F302FB21
:10476000131302FB0344A36818447F287FF70AABA6
:104770007F3890FBF2F302FB13007330FFF746BA69
:10478000ABAAAA2A2434010090300100EC350100C4
:10479000A29EFF1F259CFF1F509EFF1F0039010096
:1047A0004C9EFF1F5C9CFF1FDFF864A33868BAF8BB
:1047B0000030CE4ACE4CC31A82FB0321DA17C2EB7B
:1047C000610202EB4202A3EB820303EB430354F8C2
:1047D000233018447F2840F328817F380C2290FB37
:1047E000F2F302FB13007330DFF82883DFF828B3FD
:1047F00098F80010C0B204F0A3FDBBF80030022B03
:104800001AD93868BAF800300C22C11A91FBF2F3B9
:1048100002FB131302FB03435B6818447F2840F339
:10482000D4837F3890FBF2F302FB13007330C0B2E5
:1048300098F8001004F084FDBBF80030032B7EF6DE
:10484000E2ACBAF8003038680C22C11A91FBF2F3DE
:1048500002FB131302FB0344A36818447F287FF76D
:10486000C3AA7F3890FBF2F302FB13007330FFF70B
:1048700049B9FBF7F1FEFFF719B9FBF7EDFEFFF7BA
:104880009AB9012B3DF489AF0124FFF762BADFF832
:1048900080A29649BAF80020954C9A1A81FB021022
:1048A000D117C1EB600101EB4101A2EB810202EBE8
:1048B000420254F8220018447F2840F3BC80A0F143
:1048C0007F030C2093FBF0F200FB12307330DFF813
:1048D00048B298F80010C0B204F032FDBBF80030C6
:1048E000022B1AD93868BAF800300C22C11A91FB91
:1048F000F2F302FB131302FB03435B6818447F28A7
:1049000040F366837F3890FBF2F302FB13007330B1
:10491000C0B298F8001004F013FDBBF80030032B70
:104920007FF6FCA9BAF8003038680C22C11A91FB56
:10493000F2F302FB131302FB0344A36818447F281D
:104940007FF744AA7F3890FBF2F302FB1300733029
:10495000FFF7DFB9DFF8B8A199F80000BAF8003026
:10496000624A644CC31A82FB0321DA17C2EB61026C
:1049700002EB4202A3EB820303EB430354F8233020
:1049800018447F2846DD7F380C2290FBF2F302FBAF
:1049900013007330DFF880B1C0B204F0F5FCBBF84F
:1049A0000030022B19D999F80000BAF800300C2217
:1049B000C11A91FBF2F302FB131302FB03435B6882
:1049C00018447F2840F38F807F3890FBF2F302FB7E
:1049D00013007330C0B204F0D7FCBBF80030032BD7
:1049E0007EF6E9AEBAF8003099F800000C22C11A40
:1049F00091FBF2F302FB131302FB0344A368184478
:104A00007F287FF7B2AD7F3890FBF2F302FB1300F3
:104A100073309CE5FBF720FEBCE7FBF71DFEFFF7BC
:104A20004EB9FBF719FEFFF7F1BBFBF715FEDBE60E
:104A3000FBF712FE63E6FBF70FFE48E7FBF70CFE01
:104A40005CE4FBF709FED4E4FBF706FE59E5DFF86A
:104A5000C0A099F80000BAF80030244A264C35E688
:104A6000DFF8ACA03868BAF80030204A224CA2E641
:104A7000FBF7F2FDFFF72ABA029B1B78002B7EF4AE
:104A80004BAAFEF76EBAFBF7E7FDFFF79FBADFF818
:104A900080A099F80000BAF80030144A174C61E77A
:104AA000FBF7DAFDFFF711BBDFF864A00F49BAF896
:104AB0000020114CF1E6124B1B78002B00F0CB824A
:104AC000104B1B78002B7DF468AE0F4B1B78002B2E
:104AD0003DF463AEB8F800300C490A33A8F8003052
:104AE0000A70FDF75ABEFBF7B7FD73E7ABAAAA2A17
:104AF000003901007C360100A83701009030010028
:104B0000E29EFF1FE39EFF1FE49EFF1F489CFF1FC6
:104B10004C9EFF1FCC9CFF1F5C9CFF1FA44C228857
:104B2000002A00F02383A349DFF89CB20988BBF870
:104B300000000331884227DD9F48A0490088B1F872
:104B400000E0DFF87CC2181A0C2190FBF1F901FBA0
:104B500019004FF0900909FB0EFE01FB00E06FF019
:104B60000B0E5CF8000003440EFB02307F2840F37C
:104B700028857F3890FBF1F301FB13007330C0B23E
:104B800098F8001004F0DCFBBBF8002023881344E5
:104B9000022B23DD884B894A38681B88B2F800C095
:104BA000DFF81CE2C31A0C2193FBF1F201FB123275
:104BB000902303FB0CF301FB023373445B6818443E
:104BC0007F2840F3A3857F3890FBF1F301FB1300AE
:104BD0007330C0B298F8001004F0B2FBBBF80020AC
:104BE00023881344032B23DD734B744A38681B88D6
:104BF000B2F800C0DFF8C8E1C31A0C2193FBF1F250
:104C000001FB1232902303FB0CF301FB02337344CC
:104C10009B6818447F2840F326857F3890FBF1F38A
:104C200001FB13007330C0B298F8001004F088FB49
:104C3000BBF8002023881344042B7FF76FA85D4B3B
:104C40001B88012B7FF46AA83A68A2F10C007F2828
:104C50007FF7BCA88B3A0C2092FBF0F300FB1320EB
:104C60007330FFF756B8524C2388002B40F0A282D5
:104C7000DFF854B15049514A0988D7F80080B2F89A
:104C800000E04F48C1EB080C0C229CFBF2F102FB48
:104C900011C14FF0900C0CFB0EFE02FB01E16FF016
:104CA0000B0E405880440EFB03807F2840F3858420
:104CB000A0F17F0393FBF2F002FB10307330414B05
:104CC000C0B2197804F03CFBBBF8002023881344E1
:104CD000022B23DD384A394B11883868B3F800C0FD
:104CE000DFF8DCE0411A0C2291FBF2F302FB131116
:104CF000902303FB0CF302FB013373445B681844FD
:104D00007F2840F3A3847F3890FBF2F302FB13006B
:104D100073302C4BC0B2197804F012FBBBF80020A2
:104D200023881344032B23DD234A244B118838683E
:104D3000B3F800C0DFF888E0411A0C2291FBF2F3CF
:104D400002FB1311902303FB0CF302FB01337344AA
:104D50009B6818447F2840F36C847F3890FBF2F303
:104D600002FB13007330174BC0B2197804F0E8FA55
:104D7000BBF8002023881344042B7EF744AA0D4B74
:104D80001B88012B7EF43FAA3A68A2F10C007F2811
:104D900040F356818B3A0C2092FBF0F300FB13207A
:104DA0007330084BC0B2197804F0CAFAFEF72BBA78
:104DB000D49CFF1F769CFF1F4C9EFF1FFC9DFF1F76
:104DC00020310100CC9CFF1F5C9CFF1FCF4C23882F
:104DD000002B40F0FA81DFF868B3CD49CD4A09884D
:104DE00099F80000B2F800E0DFF85883C1EB000C3E
:104DF0000C229CFBF2F102FB11C14FF0900C0CFB5A
:104E00000EFE02FB01E16FF00B0E58F80110084492
:104E10000EFB03007F2840F3AC83A0F17F0393FBDC
:104E2000F2F002FB10307330C0B204F0ADFABBF800
:104E3000002023881344022B22DDB54AB54B11888C
:104E400099F80000B3F800C0DFF8F8E2411A0C222C
:104E500091FBF2F302FB1311902303FB0CF302FB13
:104E6000013373445B6818447F2840F3F3837F3831
:104E700090FBF2F302FB13007330C0B204F084FA2B
:104E8000BBF8002023881344032B22DDA04AA14B4A
:104E9000118899F80000B3F800C0DFF8A8E2411AC1
:104EA0000C2291FBF2F302FB1311902303FB0CF392
:104EB00002FB013373449B6818447F2840F3BD8391
:104EC0007F3890FBF2F302FB13007330C0B204F0A2
:104ED0005BFABBF8002023881344042B7EF73CA820
:104EE0008D4B1B88012B7EF437A899F80020A2F186
:104EF0000C007F287EF746AF8B3A0C2092FBF0F334
:104F000000FB13207330FEF781BEDFF804A299F88E
:104F10000000BAF80030814CC11A0C2291FBF2F368
:104F200002FB131302FB03F3E35818447F287FF7B7
:104F300071AD7F3890FBF2F302FB1300733029E56B
:104F4000774B1A88182A13D03B681344A3F1180032
:104F50007F2840F385830C20973B93FBF0F200FB06
:104F6000123303F173006F4BC0B2197804F0E8F903
:104F70006D4B6E491A78022A94BF013200221A70D2
:104F80001A7831F81200182810D10424022A02F1EC
:104F90000100C2B288BF002231F81200182804D1E3
:104FA000013CF3D11A70FEF72EB91A703B68034426
:104FB000A3F118007F2843DD0C20973B93FBF0F210
:104FC00000FB123303F17300EBE6FBF745FB2EE425
:104FD000FBF742FB9CE4FBF73FFBFFF7B0BB504BFA
:104FE0001B88182B12D099F800201344A3F1180045
:104FF0007F2840F31B830C20973B93FBF0F200FBD0
:10500000123303F17300C0B204F0BEF9464A474BB5
:10501000127833F81230182B3DF49EAF99F8002027
:105020001344A3F118007F287EF7ACAE0C20973B09
:1050300093FBF0F200FB123303F17300FEF7E6BDC1
:10504000FBF70AFBADE6DFF8C8A099F80000BAF854
:105050000030374C60E7374B1B78002B7DF4FAAFFC
:10506000354B1B78002B3DF498ABB8F80030334932
:105070000133A8F800300A70FDF78FBB2D4B1B7869
:10508000002B7DF48AAB2C4B1B78002B3DF485ABB9
:10509000B8F800302949013BA8F800300A70FDF744
:1050A0007CBB1F4A1288182A12D01344A3F118009F
:1050B0007F2840F3D2820C20973B93FBF0F200FB59
:1050C000123303F17300C0B298F8001004F038F9FD
:1050D000154B16491A78022A94BF013200221A7021
:1050E0001A7831F8120018282FD10424022A02F16C
:1050F0000100C2B288BF002231F81200182823D163
:10510000013CF3D11A703B68FEF774B9D49CFF1FC1
:105110004C9EFF1FFC9DFF1F769CFF1F0039010066
:10512000649CFF1FCC9CFF1FA089FF1F689EFF1F70
:10513000A8370100E39EFF1FE49EFF1F489CFF1F4E
:105140005C9CFF1F203101001A703B680344A3F1EF
:1051500018007F287EF73AAE0C20973B93FBF0F2C5
:1051600000FB123303F17300FEF7D3BDDFF828B361
:10517000E2E4BD4B1B88182B12D099F80020134491
:10518000A3F118007F2840F35B820C20973B93FB30
:10519000F0F200FB123303F17300C0B204F0F4F834
:1051A000B24AB34B127833F81230182B7FF436AF73
:1051B000FDF7D2BEAF4ADFF8E0B21288BBF80010AC
:1051C000033291427FF780AD54E5AA4ADFF8C8B2B6
:1051D0001288BBF80010033291427FF728AEFCE53D
:1051E000A14A1288182A12D01344A3F118007F286C
:1051F00040F37B820C20973B93FBF0F200FB1233D1
:1052000003F17300C0B298F8001004F099F8974BBE
:1052100097491A78022A94BF013200221A701A782C
:1052200031F81200182890D10424022A02F1010258
:1052300094BFD2B2002231F81200182884D1013C68
:10524000F3D15FE7884B1A88182A13D03B681344C0
:10525000A3F118007F2840F3F6810C20973B93FBC5
:10526000F0F200FB123303F17300834BC0B21978E4
:1052700004F066F87D4B7E491A78022A94BF013209
:1052800000221A701A7831F8120018287FF48EAEB6
:105290000424022A02F1010294BFD2B2002231F8A2
:1052A000120018287FF481AE013CF2D11A70FDF78C
:1052B000AABF724B00227F2107201A8004F010F849
:1052C0007F210B2004F00CF8FDF7F7BE6C4C23880F
:1052D000002B40F01082DFF8C0B16A4999F8000055
:1052E000694A09881788DFF8A4E1411A0C2291FB6A
:1052F000F2FC02FB1C114FF0900C0CFB07F702FBB9
:1053000001716FF00B075EF80110014407FB0310F9
:105310007F2840F3ED817F3890FBF2F302FB13000E
:105320007330C0B204F030F8BBF800202388134477
:10533000022B21DD534B544A99F800001B88B2F828
:1053400000E0524FC31A0C2193FBF1F201FB123221
:10535000902303FB0EF301FB02333B445B681844CC
:105360007F2840F3DA817F3890FBF1F301FB1300D3
:105370007330C0B204F008F8BBF80020238813444F
:10538000032B21DD3F4B404A99F800001B88B2F8FF
:1053900000E03E4FC31A0C2193FBF1F201FB1232E5
:1053A000902303FB0EF301FB02333B449B6818443C
:1053B0007F2840F3AF817F3890FBF1F301FB1300AE
:1053C0007330C0B203F0E0FFBBF800202388134421
:1053D000042B7EF7F0A9274B1B88012B7EF4EBA949
:1053E00099F80020A2F10C007F287FF7BEA88B3A25
:1053F0000C2092FBF0F300FB13207330FFF7A7B8EB
:10540000234B01227F2107201A8003F069FF7F21AF
:105410000B2003F065FFFDF748BE1E4B04227F21E1
:1054200007201A8003F05CFF00210B2003F058FFD7
:10543000FDF734BE174B02227F2107201A8003F0AC
:105440004FFF7F210B2003F04BFFFDF722BE114BD6
:10545000002107201C8003F043FF7F210B2003F075
:105460003FFFFDF711BE00BF6E9CFF1FA089FF1F0D
:10547000DC9DFF1F769CFF1FCC9CFF1F429CFF1FE3
:10548000D49CFF1F4C9EFF1FFC9DFF1F203101007D
:10549000EA9CFF1F429EFF1F5C9CFF1FAD4A1288C3
:1054A000182A12D01344A3F118007F2840F3478133
:1054B0000C20973B93FBF0F200FB123303F17300D7
:1054C000C0B298F8001003F03BFFA34BA3491A7831
:1054D000022A94BF013200221A701A7831F81200A1
:1054E00018287FF432AE0424022A02F1010294BF8C
:1054F000D2B2002231F8120018287FF425AE013C08
:10550000F2D1FFE5934B1A88182A13D03B68134455
:10551000A3F118007F2840F309810C20973B93FBEF
:10552000F0F200FB123303F173008D4BC0B2197817
:1055300003F006FF884B89491A78022A94BF01328A
:1055400000221A701A7831F8120018287FF42EAD54
:105550000424022A02F1010294BFD2B2002231F8DF
:10556000120018287FF421AD013CF2D11A70FDF72A
:105570004ABEFBF771F857E4764B1B88182B12D004
:1055800099F800201344A3F118007F2840F3CB8042
:105590000C20973B93FBF0F200FB123303F17300F6
:1055A000C0B203F0F1FE6C4A6C4B127833F8123043
:1055B000182B7FF433ADFDF7CFBCFBF74DF8FFF7A9
:1055C0007EBBFBF749F8FFF7DABA664B1B88182B4E
:1055D00012D099F800201344A3F118007F2840F35B
:1055E0009F800C20973B93FBF0F200FB123303F1FA
:1055F0007300C0B203F0C8FE574A5B4B127833F811
:105600001230182B3EF4D7A899F800201344A3F1C8
:1056100018007F287EF7A9AF0C20973B93FBF0F290
:1056200000FB123303F17300FEF791BFFBF714F890
:10563000E9E4FBF711F8FFF796BBFBF70DF845E43B
:10564000FBF70AF8A9E5FBF707F80EE6FBF704F805
:10565000FFF75FBBFBF700F80FE4FAF7FDFF32E559
:10566000FAF7FAFF7FE4FAF7F7FFFFF7DCBA394BF6
:105670001B88182B11D099F800201344A3F11800AF
:105680007F2856DD0C20973B93FBF0F200FB123392
:1056900003F17300C0B203F077FE2F4A2F4B12784C
:1056A00033F81230182BAFD1FEF785B82F4B1B887B
:1056B000182B11D099F800201344A3F118007F286B
:1056C0003ADD0C20973B93FBF0F200FB123303F121
:1056D0007300C0B203F058FE1F4A254B127833F80E
:1056E0001230182B90D1FEF766B8FAF7B5FF89E5AE
:1056F000FAF7B2FF15E61F4ADFF880B01288BBF850
:105700000010033291427FF70FAEE6E5FAF7A4FFEF
:10571000FFF75FBAFAF7A0FF53E6FAF79DFF28E616
:10572000FAF79AFF65E7FAF797FF39E7FAF794FF78
:10573000FBE6FAF791FFADE7FAF78EFFC9E7FAF754
:105740008BFFBDE623601946FDF75ABC0A4B029356
:10575000FDF709BF709CFF1FA089FF1FE49DFF1F7D
:10576000CC9CFF1F649CFF1F689EFF1F6E9CFF1F49
:10577000DC9DFF1F769CFF1FF69CFF1F5C9CFF1F9C
:1057800038B508F0DBF80B4805F0DAFC00234FF0E1
:105790007E5201210848FAF769FE084B084A094978
:1057A000802400251C7118461D60BDE838400BF0B0
:1057B000DDBB00BFE49CFF1F209EFF1FAC9EFF1FB0
:1057C0001C89FF1FFD05000010B50446A420636876
:1057D000198803F007FFE368A6201988BDE8104088
:1057E00003F000BF43682A20198803F0FBBE00BF06
:1057F00010B5044622206368198803F0F3FEE368BD
:1058000024201988BDE8104003F0ECBE10B5044612
:105810000A206368198803F0E5FEE3680C20198804
:10582000BDE8104003F0DEBE10B5044606206368F4
:10583000198803F0D7FEE36808201988BDE81040F6
:1058400003F0D0BE10B5044602206368198803F047
:10585000C9FEE36804201988BDE8104003F0C2BE09
:1058600070B50E4C84B01225042201230646039025
:10587000029320468DE824001423102107F00AFB30
:1058800006220923029303960195204600921423D1
:10589000102107F0FFFA04B070BD00BF149FFF1F76
:1058A00070B5AE4CB4F90030032B00F0E880002B4B
:1058B0004DD0022B6CD0052B00F09880012B00F00E
:1058C000C080042B00D070BD00244FF4AF75E1B24E
:1058D000A34805F05FFC01348542A8BF05460C2CA7
:1058E000F5D1012009F02AFB0446002009F026FB2F
:1058F000323CA0F132039B496FF4957000FB03F337
:1059000000FB04F081FB034281FB0041DB17C01761
:10591000C3EB6223C0EB612003F5AF7200F5AF73F8
:105920009342A8BF13469D42A8BF1D46A5F114018E
:10593000312900F3E28040F26C7332218A488B4AAD
:105940000180BDE870402A20136003F04BBE0E209A
:1059500007F058FF40F6FF71C8308842A8BF0846DC
:1059600020EAE07000F2DC5283B28A42804D814E20
:10597000A8BF0A460220194633802A8003F032FE6F
:105980002988042003F02EFEB4F90030022B92D1B6
:10599000172009F0D3FA0546162009F0CFFAA842DD
:1059A000B8BF284600F1C801B1F5FA7FC0F2BF8048
:1059B000B1F57A6FA8BF4FF47A6101F54873B3F57A
:1059C0007A6FA8BF4FF47A639BB289B26A4A6B4D73
:1059D00011800A202B8003F005FE29880C2003F09B
:1059E00001FEB4F90030052B7FF468AF0F2009F0F9
:1059F000A5FAC0F53F630433B3F5AF6FC0F28F80F3
:105A0000B3F5FA6FA8BF4FF4FA6399B25C4BC0F5D7
:105A10004360B0F5AF6F19807EDBB0F5FA6FA8BFB9
:105A20004FF4FA6083B2574DA4202B8003F0DAFDC7
:105A30002988A62003F0D6FDB4F90030012B7FF4AD
:105A400040AF0B2008F032FB00283CD0112009F0B9
:105A500075FA00F1C801B1F52F7F3CDB41F25C2300
:105A6000994278DC484A00F5487089B2B0F52F7F3A
:105A700011806DDB8342A8BF03469BB231E010204A
:105A800009F05CFAC830B0F5FA7F4BDBB0F57A6FFD
:105A90000146A8BF4FF47A6101F51673B3F57A6F2A
:105AA000A8BF4FF47A639BB289B2384A384D11804F
:105AB00022202B8003F096FD2988242003F092FDFC
:105AC000B4F90030F3E6152007F09CFE00F596715E
:105AD000B1F52F7F30DA40F214534FF42F712A4A78
:105AE00011802C4D06202B8003F07CFD2988082096
:105AF00003F078FDB4F90030E3E640F23A72A5F520
:105B0000B975254B02FB05F583FB0523ED17A5EBC6
:105B1000631389B2323311E74FF4AF6383E74FF475
:105B2000AF6173E740F24C434FF4FA71BDE740F2C6
:105B300014534FF4FA7149E741F25C2399420ADCAD
:105B4000114A00F5617089B2B0F52F7F118091DAAA
:105B50004FF42F73C5E71946C1E700BFF09EFF1F42
:105B6000E49CFF1F67BBCF46B49EFF1FAC89FF1F9D
:105B7000BC9EFF1FF49CFF1F589EFF1F6C9CFF1FC5
:105B8000F89CFF1F789EFF1FAA9CFF1F069EFF1F09
:105B9000029EFF1F8C9EFF1FB5814E1B2DE9F04119
:105BA000224D82B0012602B284B2009228460196AC
:105BB0007823192107F0B4F804F10C0212B28DE831
:105BC00044002846A7197823192104F1020807F098
:105BD000A7F83FB20FFA88F819233A462846194623
:105BE0000196CDF8008007F09BF878233A462846C6
:105BF0001946CDF80080019604F10A070B3407F02E
:105C00008FF83FB224B278233A46284619468DE8E9
:105C1000500007F085F8192300943A46019628466B
:105C2000194607F07DF802B0BDE8F081149FFF1F10
:105C300030B583B000230C4605B2009326225B23C7
:105C40001C210C4806F0BCFD2946012326220948E8
:105C500006F0D2F8002C24B205DB214601232622CF
:105C6000044806F0C9F8044A044B15801C8003B0B0
:105C700030BD00BF149FFF1FC289FF1FC489FF1FD3
:105C800070B5A54C237882B01BB1A44B4FF6FF72C0
:105C90001A80A34BB3F90030C3B9A24A9F4B1068D6
:105CA000B3F9002080F30C005B2303FB00F000132A
:105CB0001C3082424AD04FF0FF31FFF7B9FF9A48BB
:105CC00006F0E2FD0023237002B070BD012B1BD053
:105CD000022B5AD0032B3FD0042B00F09A80052BC7
:105CE000F0D10F2009F02AF9C0F53B600830B0F57B
:105CF000AF6F48DBB0F5FA6FA8BF4FF4FA60A0F5BC
:105D0000AF625B23894835E0894B1B78002B70D04C
:105D1000152007F077FD874B1860B0F52F7F32DB39
:105D200041F25C239842A8BF1846A0F52F735B226E
:105D3000814802FB03F380FB0320DB17C3EBA020A9
:105D40001C30764BB3F900308342B4D17B4BB3F9AE
:105D500000300133AFD1B5E7794B1B68B3F5FA7F5B
:105D600011DBB3F57A6FA8BF4FF47A637548A3F5DA
:105D7000FA725B2303FB02F380FB0320DB17C3EB08
:105D800020201C30DDE71C20DBE76F4B1B68B3F5E0
:105D9000FA7F36DBB3F57A6FA8BF4FF47A63A3F5C9
:105DA000FA7268485B2303FB02F380FB0320DB17D6
:105DB000C3EB20201C30654B1B68B3F5FA7F1EDB5C
:105DC000B3F57A6FA8BF4FF47A63A3F5FA725D4911
:105DD0005B2303FB02F381FB0321DB17C3EB2121D0
:105DE0001C314E4BB3F9003083420CD0FFF720FF3B
:105DF00065E7112009F0A2F84E4B18608DE71C21D1
:105E0000EFE71C20D7E74D4BB3F900308B42EDD1C3
:105E100058E7272200258DE8240076231C214248DC
:105E20004B4E06F07DFF16E0B0F5AF7FA8BF4FF4F4
:105E3000AF70323803FB00F386FB0321DB17C3EBA3
:105E400061111C3109B201231D442722364805F097
:105E5000D3FF0C2D09D0E9B23E4805F09BF931285B
:105E60004FF05B03E0DC1C21EDE7012009F066F850
:105E70006FF495733238384A03FB00F082FB00233D
:105E8000C017C0EB632303F5AF73312B42DDB3F5CD
:105E9000AF7FA8BF4FF4AF735B22323B2C4D02FBA8
:105EA00003F385FB0325DB17C3EB65151C350020C9
:105EB00009F044F86FF495733238274A03FB00F079
:105EC00082FB0023C017C0EB632303F5AF73312BB4
:105ED0001EDDB3F5AF7FA8BF4FF4AF735B22323B3B
:105EE0001B4902FB03F381FB0321DB17C3EB6111A9
:105EF0001C310A4BB3F90030AB4201D0284675E79C
:105F00000E4BB3F900308B423FF4D9AE28466DE713
:105F10001C21EEE71C25CAE7EA9EFF1FC289FF1F6E
:105F2000F09EFF1F5C9EFF1F149FFF1F37800B6DAD
:105F3000729EFF1F309CFF1FD3058541C489FF1F40
:105F40007C9CFF1F011FB8128C9CFF1F509CFF1FE1
:105F50004B48371BE49CFF1F67BBCF462DE9F0433E
:105F6000754C054683B02046D5F80080EE6806F0F3
:105F70007FFB1120FFF712FE012719234FF028099C
:105F80001946204601972422CDF8009006F0C8FE5D
:105F900078231946242201972046CDF8009006F078
:105FA000BFFE3946204607F045FA02231922404633
:105FB0002382E2810CF084FD4146024620460AF02D
:105FC00067FC20460AF07AFC0027142303225B4971
:105FD00023822046E7810AF05BFC20460AF06EFC33
:105FE0002323204603225649E78123820AF050FCEE
:105FF00020460AF063FC6EB12F20FFF7CFFD32235D
:1060000003225049E781204623820AF041FC2046C2
:106010000AF054FC01234C4A18461370FFF720FC89
:1060200029896A896B68521A1B885C2AA3EB0103D1
:1060300057DD03EB43030132C3EB431393FBF2F34E
:1060400003F11B023C4FDFF80CE113B21A214FF0B1
:1060500001088DE802013846AEF8002019461422E6
:1060600006F05EFE002E4ED0298A6B8AEA685B1A23
:106070005C2B12883DDC511A5C2202FB01F292FB80
:10608000F3F31B33314A2C48138001261BB238220C
:1060900019468DE84400322206F042FE00224023D9
:1060A00009218DE806002448194606F007FE31460E
:1060B000214807F0BFF96B681F4802224421228261
:1060C000E18119880AF04AFC324621491A480AF04F
:1060D000DFFBEB681848198803B0BDE8F0430AF00D
:1060E0003DBC5C2101FB03F393FBF2F303F11B02C4
:1060F000A8E7521A02EB4202C2EB4212434492FB5F
:10610000F3F31B33BEE740230921324600913846A2
:106110001946019606F0D2FD4146384607F08AF945
:106120006B6868210222F9813A821988384603B0E7
:10613000BDE8F0430AF012BC149FFF1FD8390100DC
:10614000DC390100E0390100959FFF1FEE9EFF1F23
:10615000E4390100EC9EFF1F2DE9F04F1F4685B08A
:106160001446002A4ED0052A0646D0F80C8000F0CE
:10617000AB800F9B8C4A00EBC305012CB5F80AE0FD
:1061800029896868C1EB0E0382FB03C21A444FEAF7
:10619000E373C3EBA213028851D0042C00F08D806E
:1061A000824D00220921402328468DE80600194629
:1061B00006F084FD2846012107F03CF9B8F1000FF4
:1061C00000F0E8807368022244212A82E98119885C
:1061D00028460AF0C3FB7649012228460AF058FBFC
:1061E000F368284619880AF0B9FB724B022CB3F900
:1061F000001000F0AD80082C00F0C980012005B02F
:10620000BDE8F08F6C4E6D4A33681268CB1A93422A
:106210000D4655D96A4A3B8811786448012918BF50
:10622000012414700E9A06321BB212B28DE81400CB
:106230001946BDF9382006F073FD3560DEE79BB2E4
:10624000D31A994203DC9E457146A8BF19460E9A9F
:106250000180B7F90030BDF938A0544802F10609B1
:106260004FF0000E0FFA89F919465246CDF800900A
:10627000CDF804E006F054FD29896A896868521A4D
:1062800003885C2AA3EB01037ADD03EB43030132AD
:10629000C3EB431393FBF2F303F11B0213B2012090
:1062A0003A80194652460190CDF800903F4806F0DA
:1062B00037FD434B00221A7072E712FA83F3C0E7EE
:1062C000204605B0BDE8F08F384D4FF0070A4FF07B
:1062D000000B28465A2323228DE8000C1A2106F0D1
:1062E000EDFC2846012107F0A5F84FF001094FF019
:1062F000350E2323A5F80EE052462B823149A5F82E
:1063000014902846A5F8129003930AF0C1FA284683
:106310000AF0D4FA284606F0B7FA4FF4FA6007F00C
:10632000FBFEFFF7BDFA039B1A211A4628465A23A3
:106330008DE8000C06F0C2FC284606F0A5FA3046AF
:10634000FFF70CFE204B83F80090FFF799FC27E73E
:106350004A1C12B21A8091423FF450AF0E9AB7F91C
:10636000003012480632012412B2009219460194FC
:10637000BDF9382006F0D4FC204605B0BDE8F08F0A
:106380005C2101FB03F393FBF2F21B3286E7002250
:106390001A80E0E7736868210222E9812A8219885D
:1063A00028460AF0DBFA20E7C94216B2149FFF1F05
:1063B000E4390100F49EFF1F809FFF1F8449010004
:1063C000959FFF1FE8390100EA9EFF1F2DE9F04F5E
:1063D0005A4E5B4DB6F900704C7855F8277085B071
:1063E0008146984604B10C78DFF874A11AB99AF87E
:1063F0000030002B39D0534D002338462B808AF8CB
:106400000030FFF7ABFD504A504BB5F900000121B9
:1064100011704FF6FF721A8060B301285ED0012020
:1064200032232246019000934946494B3846FFF7F4
:1064300093FE00240346B5F90020022A39DD00222C
:106440002A80B6F900203D49002A3BDB052AC4BF5B
:1064500000220A80B8F1000F39D1002C0CBF184679
:106460004FF0FF3005B0BDE8F08F364DB5F90000B4
:106470000028D2D1DFF8ECB0364ADBF800301268E1
:10648000C3EB0903934227D9334B1A78012A18BF6B
:1064900001201870FFF7E4F90123CBF80090012CDC
:1064A0002AD0042C35D0022C3AD0082C3ED000241F
:1064B000C1E7C6D1FA68002AC1D0B6F900201F4949
:1064C000002AC3DA05220A80B8F1000FC5D0039371
:1064D000FFF7D6FB039BC0E70346E0E74FF0000E53
:1064E000142322468DE8084049461C4B3846744622
:1064F000FFF732FE03469EE732888AF800400132F9
:1065000032807A6982B10024384603939047039B16
:1065100091E732880121013A32808AF80010F0E7D1
:1065200001222A8000248CE7144684E77A6900213E
:1065300029804FF0FF34002AE6D182E7F09EFF1F4A
:10654000C889FF1FF49EFF1FEA9EFF1FC289FF1F1D
:10655000EE9EFF1F84490100959FFF1FEC9EFF1FC9
:10656000F29EFF1F809FFF1F01210D2007F098BDA5
:1065700000210D2007F094BD01460D2007F090BDCD
:1065800008B50D2007F092FDB0FA80F149090D2001
:10659000BDE8084007F084BD10B5002144080D2077
:1065A00007F07EFD204607F0B7FD0D20012107F022
:1065B00077FD2046BDE8104007F0AEBD214A224BD2
:1065C00010881B68984210B535DA204A1288141AD0
:1065D0009A42A8BF1A46B4F5157F22DA121A40F281
:1065E000532303FB02F393FBF4F105310A2007F078
:1065F000C7FB174B197801B3164B17491B6840F2BC
:10660000271283F3070302FB03F381FB03211944E1
:10661000DB17C3EBA11105310920BDE8104007F0DD
:10662000AFBB131A4FF41572611C02FB03F393FB0B
:10663000F1F10531DAE70021D8E70920BDE8104083
:1066400007F09EBBF49CFF1F289CFF1FBC9EFF1FF2
:10665000AC9CFF1FA49EFF1F090402817F2838B550
:10666000A8BF7F200F4C4FF4167202FB00F284FB90
:1066700002311144D2170546C2EBA1110A2007F0DE
:106680007FFB7F3D4FF4967303FB05F384FB0321EF
:106690001944DB17A3EBA1110920BDE8384007F02E
:1066A0006FBB00BF09040281C368B3F9003030B585
:1066B00083EAE374A4EBE374002BA0B218DB01239C
:1066C00000E0134603EB830252009442F9DA0A4DCC
:1066D00090FBF3F285FB03E403FB1200DB1730327F
:1066E000D3EBA40380B201F8012BF1D10B7030BDC4
:1066F0002D230B700131E2E76766666638B5094DF8
:106700008224204602F088FF35F8021B00B288423E
:10671000204601D002F066FF0234A4B28A2CF0D1E8
:1067200038BD00BFE49DFF1F024B8020198802F096
:1067300059BF00BF709CFF1F38B5094D7824204613
:1067400002F06AFF35F8021B00B28842204601D0F1
:1067500002F048FF0234A4B2802CF0D138BD00BF53
:10676000DC9DFF1F024B7620198802F03BBF00BF63
:106770006E9CFF1F38B5094D4624204602F04CFFA1
:1067800035F8021B00B28842204601D002F02AFFF1
:106790000234A4B24E2CF0D138BD00BF689EFF1F5A
:1067A000024B4420198802F01DBF00BF649CFF1FEC
:1067B000024B4E20198802F015BF00BF889CFF1FB6
:1067C000024B9A20198802F00DBF00BFD49CFF1F16
:1067D000024B9820198802F005BF00BF769CFF1F6E
:1067E000024B8C20198802F0FDBE00BFFC9DFF1FEC
:1067F000024B9C20198802F0F5BE00BF5C9CFF1F75
:10680000024BA020198802F0EDBE00BF709EFF1F52
:10681000024B9620198802F0E5BE00BF4C9EFF1F78
:10682000024B8A20198802F0DDBE00BF0C9EFF1FBC
:10683000024B1020198802F0D5BE00BF0A9EFF1F30
:10684000024B2C20198802F0CDBE00BF5A9CFF1FBE
:10685000024B1E20198802F0C5BE00BF749CFF1FAA
:10686000C3680E20198802F0BDBE00BF024B28206D
:10687000198802F0B7BE00BF669EFF1F024B622060
:10688000198802F0AFBE00BF989CFF1F024B642026
:10689000198802F0A7BE00BF609EFF1F024B5A205E
:1068A000198802F09FBE00BF389CFF1F024B1620C4
:1068B000198802F097BE00BF429CFF1F024B2E209A
:1068C000198802F08FBE00BFDC9CFF1F024B3020F6
:1068D000198802F087BE00BFC89EFF1F024B9E2092
:1068E000198802F07FBE00BFA889FF1F024BAC20B1
:1068F000198802F077BE00BF629EFF1F024BAE20D8
:10690000198802F06FBE00BF809CFF1F024BB020B1
:10691000198802F067BE00BFF09DFF1F024BB22036
:10692000198802F05FBE00BFA29CFF1F024B182017
:10693000198802F057BE00BFFA9CFF1F024BA2202D
:10694000198802F04FBE00BF929EFF1F024B1A2013
:10695000198802F047BE00BF909CFF1F024B1C200D
:10696000198802F03FBE00BF8A9CFF1F024B6620C1
:10697000198802F037BE00BFA09EFF1F024B722095
:10698000198802F02FBE00BFC49EFF1F024B2020BB
:10699000198802F027BE00BF9E9EFF1F024B3220C7
:1069A000198802F01FBE00BF8E9EFF1F024B682099
:1069B000198802F017BE00BFC89CFF1F024B6C2055
:1069C000198802F00FBE00BF2C9CFF1F024B522003
:1069D000198802F007BE00BF4289FF1F024B5020FA
:1069E000198802F0FFBD00BF3689FF1F024B5420FB
:1069F000198802F0F7BD00BFBC89FF1F024B5C2065
:106A0000198802F0EFBD00BFC089FF1F024B5E2056
:106A1000198802F0E7BD00BF4089FF1F024B5620D6
:106A2000198802F0DFBD00BFCA9CFF1F244B1B88E2
:106A30000B2B43D8DFE803F00B10151A1F24292E67
:106A400033383D06084604221E490CF0F7B80846C4
:106A500004221D490CF0F2B8084604221B490CF030
:106A6000EDB8084604221A490CF0E8B8084604229A
:106A700018490CF0E3B80846042217490CF0DEB8B8
:106A80000846042215490CF0D9B8084604221449D6
:106A90000CF0D4B80846042212490CF0CFB80846CE
:106AA000042211490CF0CAB8084604220F490CF020
:106AB000C5B8084604220E490CF0C0B8704700BFA4
:106AC0004C9EFF1F204201008C3F0100F43D01005D
:106AD000D4420100F83D0100BC420100FC3D010030
:106AE000003E0100B4400100043E01002C420100C0
:106AF000083E0100064B074A10B41C88064B0846A6
:106B0000002C14BF11461946042210BC0CF096B894
:106B1000A89CFF1F0C3E0100103E0100064B074AD7
:106B200010B41C88064B0846002C14BF11461946A9
:106B3000042210BC0CF082B8DE9CFF1F0C3E01004A
:106B4000103E0100064B074A10B41C88064B08464D
:106B5000002C14BF11461946042210BC0CF06EB86C
:106B6000009EFF1F0C3E0100103E0100064B074A2D
:106B700010B41C88064B0846002C14BF1146194659
:106B8000042210BC0CF05AB8149EFF1F0C3E0100EA
:106B9000103E0100064B074A10B41C88064B0846FD
:106BA000002C14BF11461946042210BC0CF046B844
:106BB0004E9EFF1F0C3E0100103E0100064B074A8F
:106BC00010B41C88064B0846002C14BF1146194609
:106BD000042210BC0CF032B8EA9CFF1F0C3E0100EE
:106BE000103E01001B4B1B880A2B0AD8DFE803F07C
:106BF0000A0E12161A1E22262A2E0600164B186896
:106C000008607047154B186808607047144B186887
:106C100008607047134B186808607047124B18687B
:106C200008607047114B186808607047104B18686F
:106C3000086070470F4B1868086070470E4B186863
:106C4000086070470D4B1868086070470C4B186857
:106C5000086070470C9EFF1F383E0100103E010087
:106C6000143E0100183E01001C3E0100203E0100C0
:106C7000243E0100283E01002C3E0100303E010070
:106C8000343E0100F0B52B4E2B4FDFF8C4E0054633
:106C90000FCE87B06C460FC496E803003B68274AC6
:106CA000274F44F8040B40F6CC308342C8BF3A4625
:106CB000BEF800602180012E11889278ADF80D1089
:106CC0008DF80F202AD032D340F6CA02022E18BF08
:106CD00000229A4226DAA3F698031A491A4AC3EB0D
:106CE000031381FB03011944DB17C3EB6123243336
:106CF00082FB0321DA17C2EBA10202EB8201A3EBB4
:106D00004103303330328DF813308DF8112069464D
:106D1000284616220BF092FF07B0F0BD40F698020D
:106D20009A42D8DB094B1868CDF81100EFE740F61E
:106D3000FC02CEE74C3E0100549EFF1F403E010086
:106D40003C3E01003B773B9867666666443E010027
:106D5000EC9DFF1FF8B5174C174E2278174D33786E
:106D60002F888E46003218BF012201467046FFF779
:106D70002DFB002398423370237015DB14BF0120D4
:106D800000202B889F420ED040F23A72A3F5AF73D9
:106D90000B490C4C02FB03F381FB0312DB17A3EB43
:106DA000621332332360F8BD0749012218460A7086
:106DB0002270E6E7B88AFF1F059FFF1FB49EFF1FE2
:106DC000B5814E1BAC89FF1F949FFF1F014B1878A4
:106DD00002F078BB7C9FFF1F014B187802F08CBB40
:106DE000AC90FF1F134BB3F9003030B583EAE37466
:106DF000A4EBE374002BA0B218DB012300E01346E0
:106E000003EB830252009442F9DA0B4D90FBF3F24C
:106E100085FB03E403FB1200DB173032D3EBA40342
:106E200080B201F8012BF1D10B7030BD2D230B7016
:106E30000131E2E7AC90FF1F67666666144BB3F959
:106E4000003070B583EAE375A5EBE375002BACB2B7
:106E50001ADB012300E0034603EB83004000854278
:106E6000F9DA0C4E94FBF3F086FB03E503FB1044C8
:106E7000DB173030D3EBA503A4B201F8010BF1D13D
:106E800005480B70106070BD2D230B700131E0E7D9
:106E9000389CFF1F67666666643E0100134BB3F9BA
:106EA000003030B583EAE374A4EBE374002BA0B2A6
:106EB00018DB012300E0134603EB830252009442E7
:106EC000F9DA0B4D90FBF3F285FB03E403FB1200B0
:106ED000DB173032D3EBA40380B201F8012BF1D1E0
:106EE0000B7030BD2D230B700131E2E7A889FF1F25
:106EF00067666666134BB3F9003030B583EAE37416
:106F0000A4EBE374002BA0B218DB012300E01346CE
:106F100003EB830252009442F9DA0B4D90FBF3F23B
:106F200085FB03E403FB1200DB173032D3EBA40331
:106F300080B201F8012BF1D10B7030BD2D230B7005
:106F40000131E2E7809CFF1F67666666134BB3F969
:106F5000003030B583EAE374A4EBE374002BA0B2F5
:106F600018DB012300E0134603EB83025200944236
:106F7000F9DA0B4D90FBF3F285FB03E403FB1200FF
:106F8000DB173032D3EBA40380B201F8012BF1D12F
:106F90000B7030BD2D230B700131E2E7A29CFF1F67
:106FA00067666666134BB3F9003030B583EAE37465
:106FB000A4EBE374002BA0B218DB012300E013461E
:106FC00003EB830252009442F9DA0B4D90FBF3F28B
:106FD00085FB03E403FB1200DB173032D3EBA40381
:106FE00080B201F8012BF1D10B7030BD2D230B7055
:106FF0000131E2E7929EFF1F67666666134BB3F9A5
:10700000003030B583EAE374A4EBE374002BA0B244
:1070100018DB012300E0134603EB83025200944285
:10702000F9DA0B4D90FBF3F285FB03E403FB12004E
:10703000DB173032D3EBA40380B201F8012BF1D17E
:107040000B7030BD2D230B700131E2E74289FF1F29
:1070500067666666134BB3F9003030B583EAE374B4
:10706000A4EBE374002BA0B218DB012300E013466D
:1070700003EB830252009442F9DA0B4D90FBF3F2DA
:1070800085FB03E403FB1200DB173032D3EBA403D0
:1070900080B201F8012BF1D10B7030BD2D230B70A4
:1070A0000131E2E73689FF1F67666666134BB3F965
:1070B000003030B583EAE374A4EBE374002BA0B294
:1070C00018DB012300E0134603EB830252009442D5
:1070D000F9DA0B4D90FBF3F285FB03E403FB12009E
:1070E000DB173032D3EBA40380B201F8012BF1D1CE
:1070F0000B7030BD2D230B700131E2E7BC89FF1FFF
:1071000067666666134BB3F9003030B583EAE37403
:10711000A4EBE374002BA0B218DB012300E01346BC
:1071200003EB830252009442F9DA0B4D90FBF3F229
:1071300085FB03E403FB1200DB173032D3EBA4031F
:1071400080B201F8012BF1D10B7030BD2D230B70F3
:107150000131E2E7C089FF1F67666666134BB3F92A
:10716000003030B583EAE374A4EBE374002BA0B2E3
:1071700018DB012300E0134603EB83025200944224
:10718000F9DA0B4D90FBF3F285FB03E403FB1200ED
:10719000DB173032D3EBA40380B201F8012BF1D11D
:1071A0000B7030BD2D230B700131E2E74089FF1FCA
:1071B0006766666608B5702002F02EFA044B1988DF
:1071C000884204D07020BDE8084002F00BBA08BD28
:1071D000EC9DFF1F08B5742002F01EFA044B1988BD
:1071E000884204D07420BDE8084002F0FBB908BD15
:1071F000849EFF1F054B1B880846042213B90449CF
:107200000BF01CBD03490BF019BD00BF889CFF1F8C
:107210006C3E0100683E01000E4B1B88032B17D803
:10722000DFE803F0110C0702084604220A490BF0BC
:1072300005BD0846042209490BF000BD084604229A
:1072400007490BF0FBBC0846042206490BF0F6BCCC
:10725000704700BFFC9DFF1F783E0100743E010097
:10726000703E0100103F010010B40A4B0A4C0A4660
:1072700093E8030083B0238802AC04E9030004EB25
:107280008303104653F8081C052203B010BC0BF012
:10729000D5BC00BF683A0100609EFF1F30B40A4BA6
:1072A0000A4D0C4693E8070084B02B8804AD05E92D
:1072B000070005EB8303204653F80C1C042204B09E
:1072C00030BC0BF0BBBC00BF703A0100EC9DFF1F4F
:1072D000F0B40C4D0C4F0E460FCD8CB001AC0FC46A
:1072E0000FCD0FC495E807003B8884E807000CAA7F
:1072F00002EB8303304653F82C1C04220CB0F0BC84
:107300000BF09CBC7C3A0100429EFF1F30B50A4B3B
:107310000A4D0C460FCB85B00DF1100E0EE90F0093
:107320002B880EEB8303204653F8101C042205B073
:10733000BDE830400BF082BCB83A0100629EFF1FEE
:1073400030B50A4B0A4D0C460FCB85B00DF1100E2F
:107350000EE90F002B880EEB8303204653F8101C18
:10736000042205B0BDE830400BF068BCB83A01001B
:10737000F09DFF1FF0B40B4D0B4F0E460FCD86B0A6
:107380006C460FC495E803003B8884E8030006AA16
:1073900002EB8303304653F8181C042206B0F0BCFD
:1073A0000BF04CBCC83A0100FA9CFF1FF0B40A4D28
:1073B0000A4F0E460FCD86B001AC0FC42A683B8839
:1073C000226006AA02EB8303304653F8141C0C22F9
:1073D00006B0F0BC0BF032BCE03A01008A9CFF1F03
:1073E000F0B40B4D0B4F0E460FCD86B06C460FC45C
:1073F00095E803003B8884E8030006AA02EB8303B8
:10740000304653F8181C042206B0F0BC0BF016BC32
:10741000F43A0100849EFF1F164B1B880BB31BB26E
:1074200083EAE370A0EBE370002B30B584B21DDB80
:10743000012300E0134603EB830252009042F9DA85
:107440000D4894FBF3F280FB03E503FB1244DB17CA
:107450003032D3EBA503A4B201F8012BF1D10B70AC
:1074600030BD0846042205490BF0E8BB2D230B7004
:107470000131DDE7C89CFF1F676666667C3E010040
:1074800030B50A4B0A4D0C460FCB85B00DF1100EEE
:107490000EE90F002B880EEB8303204653F8101CD7
:1074A000042205B0BDE830400BF0C8BB0C3B010026
:1074B0002C9CFF1F054B1B881BB9054B18680860E7
:1074C00070470846042203490BF0B8BB709EFF1FAB
:1074D000103E01000C3E0100164B1B880BB31BB283
:1074E00030B583EAE374A4EBE374002BA0B21CDB99
:1074F000012300E0134603EB830252009442F9DAC1
:107500000D4D90FBF3F285FB03E403FB1200DB1748
:107510003032D3EBA40380B201F8012BF1D10B7010
:1075200030BD064B1868086070472D230B70013181
:10753000DEE700BF749CFF1F67666666103E0100B1
:10754000164B1B880BB31BB230B583EAE374A4EB74
:10755000E374002BA0B21CDB012300E0134603EB15
:10756000830252009442F9DA0D4D90FBF3F285FB51
:1075700003E403FB1200DB173032D3EBA40380B229
:1075800001F8012BF1D10B7030BD064B1868086073
:1075900070472D230B700131DEE700BF529EFF1FA5
:1075A00067666666103E0100164B1B880BB31BB264
:1075B00030B583EAE374A4EBE374002BA0B21CDBC8
:1075C000012300E0134603EB830252009442F9DAF0
:1075D0000D4D90FBF3F285FB03E403FB1200DB1778
:1075E0003032D3EBA40380B201F8012BF1D10B7040
:1075F00030BD064B1868086070472D230B700131B1
:10760000DEE700BF429CFF1F67666666803E0100A2
:10761000174B1B881BB31BB270B583EAE375A5EB50
:10762000E375002BACB21EDB012300E0034603EB45
:10763000830040008542F9DA0E4E94FBF3F086FB9E
:1076400003E503FB1044DB173030D3EBA503A4B2F2
:1076500001F8010BF1D108480B70106070BD074BA9
:107660001868086070472D230B700131DCE700BFFC
:10767000DC9CFF1F67666666843E0100103E0100C9
:10768000164B1B880BB31BB230B583EAE374A4EB33
:10769000E374002BA0B21CDB012300E0134603EBD4
:1076A000830252009442F9DA0D4D90FBF3F285FB10
:1076B00003E403FB1200DB173032D3EBA40380B2E8
:1076C00001F8012BF1D10B7030BD064B1868086032
:1076D00070472D230B700131DEE700BFC89EFF1FEE
:1076E00067666666103E0100164B1B880BB31BB223
:1076F00030B583EAE374A4EBE374002BA0B21CDB87
:10770000012300E0134603EB830252009442F9DAAE
:107710000D4D90FBF3F285FB03E403FB1200DB1736
:107720003032D3EBA40380B201F8012BF1D10B70FE
:1077300030BD064B1868086070472D230B7001316F
:10774000DEE700BFA09EFF1F67666666103E010071
:10775000164B1B880BB31BB230B583EAE374A4EB62
:10776000E374002BA0B21CDB012300E0134603EB03
:10777000830252009442F9DA0D4D90FBF3F285FB3F
:1077800003E403FB1200DB173032D3EBA40380B217
:1077900001F8012BF1D10B7030BD064B1868086061
:1077A00070472D230B700131DEE700BFC49EFF1F21
:1077B00067666666103E0100174B1B881BB31BB241
:1077C00070B583EAE375A5EBE375002BACB21EDB65
:1077D000012300E0034603EB830040008542F9DA11
:1077E0000E4E94FBF3F086FB03E503FB1044DB171E
:1077F0003030D3EBA503A4B201F8010BF1D1084856
:107800000B70106070BD074B1868086070472D231F
:107810000B700131DCE700BF9E9EFF1F6766666646
:10782000843E0100103E0100054B1B881BB1054B37
:10783000186808607047044B18680860704700BFFC
:10784000CA9CFF1F983E0100943E010070B5FAF7F4
:10785000EBFB164B1B7813B1154C237833B9154B42
:107860001020198801F0BEFE012070BD124D134E8C
:107870002B783288B3FA83F382F008025B09114651
:1078800042202B70328001F0ADFE23780BB12B78B3
:107890002BB90021212006F003FC002070BD01213E
:1078A000212006F0FDFB002070BD00BF409EFF1FA1
:1078B000F29DFF1F0A9EFF1F089EFF1FBE9EFF1F17
:1078C000184B1A8852B3184A128830B50A80B3F997
:1078D0000030002B83EAE374A4EBE374BCBF2D23D8
:1078E0008B70A0B2ACBF02310331012300E013461C
:1078F00003EB830252009442F9DA0C4D90FBF3F251
:1079000085FB03E403FB1200DB173032D3EBA40347
:1079100080B201F8012BF1D10B7030BD044B186817
:1079200008607047909CFF1F9C3E0100676666667A
:10793000103E010070B53C4D2B780646002B35D12A
:107940001C4673780BB9204670BDFAF76DFB374AB9
:10795000374B3848127831781B78007802EB4303B4
:107960004A1E03EB80030E2AEDD801A050F822F046
:10797000D9790000FB79000047790000D97900002F
:10798000477900004779000047790000C779000077
:1079900047790000477900004779000047790000E7
:1079A0004779000047790000C3790000AE212248E2
:1079B00004F012FC204804F05BFE00232B7001242D
:1079C000BFE707F0DBFBAF211B4804F005FC1B4AB7
:1079D000012313702B70B6E783B919480388042973
:1079E0004FF6FF7103F1FF320CBF01230B46134426
:1079F00003F07F03013303800FE073B1013B114AB1
:107A000032F813304BB10E4E0F481049104A3380F4
:107A10000123002606700B701370084A022101230F
:107A200011702B70204670BDB88AFF1FE59EFF1FA6
:107A3000E69EFF1F949EFF1F149FFF1F949FFF1F32
:107A4000909EFF1FCC9DFF1FC09CFF1F489CFF1FE7
:107A5000979FFF1F10B5064B064C1A882046012140
:107A600001F0AEFD21884220BDE8104001F0BABD12
:107A7000A89CFF1FBE9EFF1F10B5064B064C1A8820
:107A80002046022101F09CFD21884220BDE81040E3
:107A900001F0A8BDDE9CFF1FBE9EFF1F10B5064B68
:107AA000064C1A882046042101F08AFD21884220D4
:107AB000BDE8104001F096BD009EFF1FBE9EFF1F57
:107AC00010B5064B064C1A882046062101F078FDB9
:107AD00021884220BDE8104001F084BD149EFF1FA4
:107AE000BE9EFF1F10B5064B064C1A88204600218B
:107AF00001F066FD21884220BDE8104001F072BD12
:107B00004E9EFF1FBE9EFF1F08B5122001F084FD90
:107B1000054B1988884206D0122001F063FDBDE8AC
:107B2000084001F001BC08BD429EFF1F08B5582067
:107B300001F072FD054B1988884206D0582001F0EB
:107B400051FDBDE8084001F0EFBB08BD529EFF1F8C
:107B500008B5142001F060FD054B1988884206D055
:107B6000142001F03FFDBDE8084001F0DDBB08BD79
:107B7000EA9CFF1FF0B480EAE075A5EBE0750028F1
:107B8000ACB21FDB1DBF2B230B704E1C0E46012316
:107B900000E0134603EB830252009542F9DA0B4FE3
:107BA00094FBF3F287FB030503FB1244DB1730322F
:107BB000D3EBA503A4B206F8012BF1D1337008462C
:107BC000F0BC70472D230B704E1CE0E767666666BD
:107BD000174B18880C2813D0192815D01A2817D03D
:107BE0001B2819D01C281BD01D281DD01E2803D0EF
:107BF0000C3800B2FFF7BEBF0E4A1068086070472D
:107C00000D4A1068086070470C4A10680860704799
:107C10000B4A1068086070470A4A1068086070478D
:107C2000094A106808607047084A10680860704781
:107C30008E9EFF1FBC3E0100A43E0100A83E010035
:107C4000AC3E0100B03E0100B43E0100B83E010070
:107C5000034B1888A0EB8000400000B2FFF78ABFFA
:107C60007C9FFF1F024BB3F90000FFF783BF00BFEB
:107C7000989CFF1F024B1888033800B2FFF77ABFA9
:107C8000669EFF1F024B18880C3800B2FFF772BFC8
:107C90003E9CFF1F024B1888183800B2FFF76ABFDE
:107CA000709CFF1F024B1888183800B2FFF762BFA4
:107CB0006E9CFF1F024B1888183800B2FFF75ABF9E
:107CC000649CFF1FC3681888183800B2FFF752BFC2
:107CD000054B1B881BB9054B1868086070470846A0
:107CE000042203490AF0AABF769CFF1F103E010040
:107CF0000C3E0100054B1B881BB9054B186808603A
:107D000070470846042203490AF098BFD49CFF1F1D
:107D1000103E01000C3E010030B5134C85B001252A
:107D20002B463C2202212046009504F0CBFA204647
:107D300004F09EFC00224021802320460191009304
:107D400011460A4B029505F041F9204604F09CFDCE
:107D500007480849084A0023036083800B608B8032
:107D60001360938005B030BD149FFF1F3C45010098
:107D7000F89EFF1F0C9FFF1F849FFF1F10B500EB95
:107D8000C00000F10F02D2B293B284B09C1E981CC6
:107D90003D2303918DE819003921024805F07AF856
:107DA00004B010BD149FFF1F014B01221A707047D1
:107DB000059FFF1FF0B5734B734C744D744F754E98
:107DC00085B004228DE80C0002932046724B4022BD
:107DD000802104F07FF82046704A7149714C09F007
:107DE000C5F8AF61704FEF61704FA7617048714F78
:107DF000E761714F87617149714FC761714F8F6141
:107E0000714A724FCF61724F9761724B724FD76157
:107E1000724F9F61724FDF61724FB761724D734F46
:107E2000F761734FAF61734C734FEF61734FA7618D
:107E30007348744FE761744F74498761744FC76129
:107E4000744F754A8F61754FCF61754F754B976150
:107E5000754FD761754F764E9F61764FDF61764FD4
:107E6000764DB761764FF761764F774CAF61774FBC
:107E7000EF61774F7748A761774FE761774F876169
:107E80007749784FC761784F8F61784A784FCF61D3
:107E9000784F9761784B794FD761794F9F61794ED1
:107EA000794FDF61794FB761794D7A4FF7617A4F3A
:107EB000AF617A4C7A4FEF617A4FA7617A487B4F76
:107EC000E7617B4F87617B497B4FC7617B4F8F6148
:107ED0007B4A7C4FCF617C4F97617C4B7C4FD76155
:107EE0007C4F7D4E9F617D4FDF617D4F7D4DB76142
:107EF0007D4FF7617D4F7E4CAF617E4FEF617E4FCE
:107F00007E48A7617E4FE7617E4F7F4987617F4F43
:107F1000C7617F4F7F4A8F617F4FCF617F4F804B1B
:107F20009761804FD761804F9F61804E804FDF61A6
:107F3000804F814DB761814FF761814F814CAF61B7
:107F4000814F82488249EF61824F834DA761E5618D
:107F5000824F834D834CDFF830E2834A834B876145
:107F6000C5618C61824E834F834D844CC1F81CE007
:107F7000834884499761D5619C61D861B16005B03F
:107F8000F0BD00BF40420F00149FFF1F288AFF1F53
:107F9000857C0000D08CFF1FE090FF1F1C89FF1F15
:107FA0002DBF0000048FFF1F61680000757C00007A
:107FB000508EFF1F6D680000F56A0000408CFF1FA7
:107FC000557A00001D6B0000288FFF1F797A000092
:107FD000456B00004C8AFF1F9D7A0000657C000005
:107FE0007D6800006D6B0000608DFF1FC17A00008E
:107FF00069720000AC8CFF1F8D680000956B00005B
:108000003C8DFF1FE57A0000517C0000188DFF1F9A
:10801000CD6D0000E56D0000E08EFF1FD96D000002
:108020009D720000D48BFF1FB5710000D17200005B
:10803000948FFF1F097B000041750000888CFF1F93
:108040002D7B00003D6E0000948BFF1F9D6800009B
:10805000BD6B00002490FF1F517B0000A97500003C
:10806000648CFF1FAD68000011760000848DFF1F37
:10807000BD680000817600001C8CFF1FCD680000E9
:108080009D6E00004C8BFF1FDD6800000D7300002B
:10809000DC8FFF1FED680000F56E0000988EFF1F5B
:1080A000FD68000041730000288BFF1F0D69000070
:1080B0004D6F0000E089FF1F1D690000757300000F
:1080C000708AFF1F2D690000A56F0000F48CFF1F50
:1080D0003D690000C1780000BC8EFF1F4D690000A3
:1080E000AD730000BC90FF1F5D690000E9760000E1
:1080F0002C8EFF1F6D69000051770000048BFF1F5D
:108100007D690000E1730000B88FFF1FD57100008A
:10811000B9770000748EFF1F8D690000D17B0000CD
:10812000E08AFF1F9D69000019740000BC8AFF1FD0
:10813000AD690000817400008890FF1FBD690000D8
:10814000FD6F0000F88BFF1FCD690000948AFF1FB0
:10815000708BFF1F55700000DD690000AD700000DE
:10816000ED690000057100004C8FFF1F048AFF1F9E
:10817000B090FF1F5D7100000D6A000029780000BB
:108180001D6A000045870000FD690000F0B5461C2F
:1081900083B00D460127032336B22AB20446314686
:1081A0008DE888002348ADB204F00AFE0C23AA1C17
:1081B00012B200930197052321B21E4804F000FE7D
:1081C0001D4A1E4B12881B68BA422AD023D3022AAA
:1081D00010D11B4CA3F6CA0384FB03241C44DB17F9
:1081E000C3EB24140A2CA8BF0A2424EAE474A2B224
:1081F00023B202E000231A461C460D35AA1A0120BC
:108200000093019012B2314603230A4804F056FD50
:10821000204603B0F0BD0B4CA3F6FC0384FB032403
:10822000DDE7094CA3F6980384FB0324DB17C3EBBB
:10823000A404D7E7149FFF1FEC9DFF1F549EFF1F50
:10824000898888881F85EB51398EE3382DE9F04302
:108250008FB283B0DFF84C80BD1D461D2DB204B235
:1082600036B24FF001090AB2234631464046009526
:10827000CDF8049004F054FD2A463346214640468A
:108280008DE8200204F04CFD07F10C020095334606
:1082900012B22146CDF80490404604F041FD03B0EF
:1082A000BDE8F083149FFF1F2DE9F04F804685B095
:1082B000002959D10121314805F0BCF8304998F81E
:1082C000062098F8083011F80290994525DADFF871
:1082D000ACB04FEA89064D460C244FF0000AD8F89E
:1082E0000C309B595F68ABF810403846ABF80EA0D5
:1082F0000AF0E6FB39460246204808F0C9FA1F4852
:1083000008F0DCFA98F8083001350934AB42A4B221
:1083100006F1040601DD422CE1D1B9F1000F13D1C1
:1083200009F1060999450CDA3C2301213B2203910E
:1083300002930093019239233F223A210F4804F01F
:10834000A9FD05B0BDE8F08F0F2301213B22039169
:1083500002930093019239230C223A21074804F03A
:1083600099FD98F80830DBE7002134230093019150
:108370003F230C22014804F0A1FC9BE7149FFF1F40
:108380000C9FFF1F38B50F4C012320461946A382CE
:108390006382552505F04EF83423204602220A490F
:1083A0002382E58108F074FA20460522074908F087
:1083B0006FFA204608F082FA2046BDE8384004F003
:1083C00063BA00BF149FFF1F083F01000C3F01006C
:1083D000F8B50F4606460AF073FB00EB4000840038
:1083E000AFB338460AF06CFB00EB400040002318A6
:1083F0005B10194D03F16002121A4FF0280E012193
:108400002846C3F16004EA81A5F810E005F012F8EF
:1084100038460AF055FB39460246284608F038FA35
:10842000284608F04BFA02210B4805F003F82123F7
:1084300030462B82EC810AF043FB31460246064867
:1084400008F026FA0448BDE8F84008F037BA64108E
:10845000C4F16004004DE6E7149FFF1F10B50D4BFB
:108460001B5C51F82340237884B013B1012004B081
:1084700010BD04AA01A942F8103D2046A3699847FF
:10848000A38A9B07F2D401A80099FFF7A1FF01205E
:1084900004B010BDF89EFF1F2DE9F04F304DDFF8FE
:1084A000D0B0DFF8C8A00FCD91B003AC0FC40FCD92
:1084B0000FC40FCD0FC42B6823600025A8462F469C
:1084C0002E4600E09846BAF8003026495BF8232093
:1084D000DFF8A09011232846F8F76EF900EBC003EF
:1084E00000EB8300204B83FB00340444C017C0EB37
:1084F0006434C4F13C00C6F13C0207F1410101269D
:1085000000B208F1410300901BB2019612B209B209
:10851000484604F005FC08EB060305F211153C2B58
:108520002646ADB24746CDD16B22342300214846C2
:10853000A9F80E20A9F8103004F07CFF0B4B1B8823
:1085400010AA02EB830353F8344C20460AF0B8FA21
:1085500021460246484611B0BDE8F04F08F098B9F0
:108560001C3B0100FC340100090002805A9CFF1FE3
:1085700060330100149FFF1F234B70B5B3F9003027
:1085800083EAE374A4EBE374002B82B0A1B234DB82
:1085900068466D46012300E0134603EB8302520058
:1085A0009442F9DA194E91FBF3F286FB03E403FBE4
:1085B0001211DB173032D3EBA40389B205F8012B7B
:1085C000F1D119462B70FFF703FF114B1B7813B144
:1085D000104B1B780BB902B070BD0F4C0121204627
:1085E00004F028FF64253323204604220B49E5814B
:1085F000238208F04DF902B070BD2D238DF80030B4
:108600000DF101056846C5E70A9EFF1F67666666AD
:10861000F29DFF1F089EFF1F149FFF1F143F0100C4
:1086200070B5404E404D82B0304604F021F82B78B2
:10863000D3B93C4C0621204604F0FCFE2B78012BDC
:1086400038D9022B4FF003024FF00A030CBF374911
:108650003749E3812046238208F01AF9204602B008
:10866000BDE8704008F02AB9324B1A780121052381
:10867000002A33D1019100931146304604F0A0FB4B
:108680002D4B1A78002A34D0052301220192009341
:1086900000220A21234804F011FB284B1A78002AF3
:1086A00033D1012105230191009314211D4804F0C9
:1086B00087FBBEE7224B1988092930D963298CBF73
:1086C0000A221F220A231748F281338208F046F952
:1086D000144802B0BDE8704008F0F0B800220191E3
:1086E00000931146304604F0E9FA134B1A78002A39
:1086F000CAD105230121019100930A21094804F000
:108700005FFB0E4B1A78002ACBD001220523019281
:10871000009300221421034804F0D0FA89E73022A4
:10872000D0E700BF149FFF1F979FFF1F1C3F010052
:10873000203F0100E59EFF1FE69EFF1F949EFF1F46
:10874000909EFF1F2DE9F047714E307848B9714B6C
:108750001B6899425FD3704A012313703370BDE8E0
:10876000F0876E4D6B4F0C46284603F081FF04F6F0
:10877000AC5331240022EC810124114628462A8280
:10878000AC826C823B60327004F054FE0522644976
:10879000644E284608F07CF8102728464FF00C0855
:1087A00008F08CF80B226049EF812846A5F810806C
:1087B00008F06EF85D490522284608F069F8284659
:1087C00008F07CF85A4BEF811A68A2F69803C3EBC5
:1087D000031386FB03161E44DB17C3EB662640F625
:1087E000CC3320219A42298206F124064FF022013F
:1087F0004FF0040011DCFFF7C9FC4E4BB3F80090BA
:108800008246B9F1000F30D0B9F1010F4DD0B9F166
:10881000020F47D02046BDE8F087FFF717FD464915
:108820000922284608F034F84449EF8181FB0637D5
:10883000F317C3EBA7072A23394628462B8208F0F3
:108840008DF822463E49284608F022F807EB8701BA
:10885000A6EB4101284608F081F82246284639490E
:1088600008F016F82046BDE8F08737493A46284612
:1088700008F00EF8284608F021F82A232B825146EA
:10888000EF8128462D4F08F069F807222F49284626
:1088900007F0FEFFF31787FB0627C3EBA707394650
:1088A0002846CCE742462A49E1E742462949234C7B
:1088B000284607F0EDFF284608F000F82A232B820F
:1088C00051462846EF8108F049F807221F492846FB
:1088D00007F0DEFFF31784FB0624C3EBA404214654
:1088E000284608F03BF84A461549284607F0D0FFCD
:1088F00004EB8401A6EB4101284608F02FF84A4614
:108900002846104907F0C4FF4846BDE8F08700BF7D
:10891000B88AFF1F789FFF1F949FFF1F149FFF1FA0
:10892000243F01003B773B982C3F01000C3F0100A6
:10893000549EFF1FEC9DFF1F383F0100676666666F
:10894000244B01009C4A0100443F0100583F0100B4
:10895000703F0100603F01002DE9F041744C227826
:10896000002A05460F4614BF4FF001084FF00008DB
:108970004ED1704E3368CB1AB3F5FA6F04D86B78CA
:10898000A3B94046BDE8F0816B4B6C486C49DFF8F9
:10899000CCE11A70012303700988237026208EF819
:1089A000002000F01FFE6B78002BEAD03760F9F74B
:1089B0003BFB644A644B6549127828781B78097838
:1089C00002EB4303421E03EB81030E2AD9D801A117
:1089D00051F822F0C18A00008D8A000083890000CE
:1089E000C18A000083890000838900008389000018
:1089F000758A0000838900002B8A000083890000AB
:108A0000838900008389000083890000278A000091
:108A1000AF214F48474E03F0DFFBFFF701FE002375
:108A200037602370ABE706F0A9FB494C204603F002
:108A30001FFE2046022104F0FDFC23250F23238284
:108A400005224449E581204607F022FF204607F031
:108A500035FF1E230522404923822046E58107F089
:108A600017FF204607F02AFF204603F00DFF00F015
:108A7000ABFC86E7394D2B78012B50D9304B2620A3
:108A8000198800F0AFFD00232B707AE7002B3FF42C
:108A900078AF013B324A32F81330002B3FF471AF0C
:108AA000274C304825492D4A23804FF001080023E8
:108AB000037081F8008082F80080FFF7B1FD60E765
:108AC00093B1013B264A32F8131019B31C4B254DC4
:108AD0001A4C224A19800026012326202E7023706A
:108AE000137000F07FFD15E0154C1E4922880B70B5
:108AF00004284FF6FF7002F1FF310CBF012202463D
:108B00000A440E4E154D02F07F02013201212280EF
:108B100031702B70FFF784FD4FF0010831E70649F3
:108B2000064A01230020087013702370A6E700BFD7
:108B3000B88AFF1F909FFF1F949FFF1F489CFF1F35
:108B4000909EFF1FE59EFF1FE69EFF1F949EFF1F46
:108B5000149FFF1F803F0100883F0100979FFF1F68
:108B6000CC9DFF1FC09CFF1F2DE9F04FAE4E4FF074
:108B70000109A6F81490A6F81290838813EA090454
:108B80008BB005460F46934640F0AB80DFF8C482B9
:108B900098F80030002B7BD1AA79A44CA35CA3B930
:108BA000DFF8B4A279781AF8029039B33B78013B28
:108BB000072B00F2B280DFE813F0EF005101B000A4
:108BC0006B01B000B000B000E7007E78002E00F02E
:108BD000C580013BE868397850F82360F0684B1E87
:108BE0000788072B00F2A380DFE813F0700159011A
:108BF000A1006A01A100A100A1009B008C4E336876
:108C0000C3EB0B03B3F5967F72D98A4B1878012812
:108C10001ABF012018701970874B18BF0146985C65
:108C2000C0EB0900C0B2FFF7A9F80124C6F800B0F4
:108C3000AB889B076DD57B78002B6AD0F9F7F4F9E8
:108C40007E4B7F4A7F481B7812783978007802255E
:108C500015FB02330A2903EB800300F049810C293C
:108C600057D1002B55D003F11900774E774A013BBD
:108C70000021400080B226F813100123157088F8F7
:108C8000003000F0AFFC724B032220461A702CE03B
:108C9000304603F0EDFC3046494604F0CBFBF4814E
:108CA0003482AB88580725D42C68204609F008FF89
:108CB00021460246304607F0EBFD304607F0FEFD48
:108CC000092201238DE80C0000217F23564804F07F
:108CD00027F800212846FFF7E7FA002388F800303C
:108CE0005AE783681146384698470BB0BDE8F08FC5
:108CF0000846FAE72B6804A8984704A809F0E0FEA4
:108D000004A90246304607F0C3FD304607F0D6FD01
:108D1000D6E720460BB0BDE8F08F00240AF8029099
:108D200086E70023A3543046F3699847F06807802C
:108D3000002425223C238DE81400412118223A48C2
:108D400003F0BCFFE968A879FFF788FB394A384B84
:108D50001470C3F800B00BB0BDE8F08F34490B6855
:108D6000C3EB0B03B3F5967F40F2E080314FC1F8BF
:108D700000B03C78012C00F0AF800123E9683B7023
:108D80001046FFF76BFBB0E7304BE9791970012310
:108D900088F800300024C1E72B7A013B4B45BCDD4D
:108DA00009F10104E4B2A145B7D0234E16F802B090
:108DB000CBEB0900C0B20021FEF7E0FF2B7A052BB8
:108DC000D9461BD9CBEB0402042A40F3A980A4F1B5
:108DD000040BBBF1000FC0F2AD80063B5B45A8BFA2
:108DE0005B465FFA83F9AA791348B15C994205D0D2
:108DF00000F8029001212846FFF756FAC9EB04005B
:108E0000C0B201210B4EFEF7B9FF002134230191BE
:108E100000930B223170044840233F21A14603F008
:108E20004DFF0124AA7979E7149FFF1F849FFF1F3C
:108E3000809FFF1F959FFF1F0C9FFF1FE59EFF1F39
:108E4000E69EFF1F949EFF1FCC9DFF1F949FFF1F58
:108E5000979FFF1FB88AFF1FF89EFF1F0FFA89F325
:108E6000E9685D4851F823B0036804935B499BF8B7
:108E7000003004980860002B6CD0012B7FF44DAFBC
:108E800057499BF8080088F800300870002445E72F
:108E9000B9F1000F4CD009F1FF34E4B283E7B38A93
:108EA00003F004039BB2002B3FF43CAF336A9847B6
:108EB00000283FF43BAFAB79F0680022E25436E77C
:108EC000738ABB4240D90137BFB230E7338ABB4215
:108ED00034D2013FBFB22AE725238DE8480041483C
:108EE0003E703C231822412103F0E8FE2046FCE6B8
:108EF000002B3FF40EAF3C4A3C4E1188384A03F138
:108F00001900013B400080B226F81310012388F8B5
:108F10000030157000F066FB354B20461D70E4E60E
:108F2000002A3FF75AAF04F1FF3B52E73046DCE638
:108F30004C46F3E64FF000094B4654E7B38AD90795
:108F40007FF5F5AE778AF2E6B38ADA077FF5EFAE02
:108F5000378AECE627490393885CC0EB090009F1E6
:108F6000010EC0B2012104F802E0FEF707FF039BE7
:108F7000DBF808B0019334231A4800930B224023F6
:108F80003F2103F09BFE012434230B228DE81800BF
:108F90003F214023134803F013FF2146114804F0FA
:108FA00049FA584609F08CFDA0EB800000F15F0300
:108FB0000F22F3813282584609F082FD594602465B
:108FC000084807F065FC074807F078FCE968A879CD
:108FD000FFF744FAAA79A1E6B49FFF1F809FFF1F05
:108FE000949FFF1F149FFF1F909EFF1FCC9DFF1F8C
:108FF000979FFF1F0C9FFF1F2DE9F047DFF8089296
:109000006D4B99F800601B68DFF800A282B0003653
:1090100001934FF0030018BF0126019F9AF80080CA
:1090200005F044F80546042005F040F80446052004
:1090300005F03CF8800040EA4404062005F036F8CC
:109040002C4364B25D4944EAC0000A7880F00F0303
:10905000DBB29A425A4A3CD01760002259480B7042
:1090600003788DF800808DF8012053B3564A1268BA
:109070004EF66021BA1A8A4219D8022B59D0012B18
:109080005FD0062B48D0032B63D0042B69D0052B6F
:1090900077D0072B7DD0082B00F08380092B68D078
:1090A00016B14A4803F0F0FB02B0BDE8F087484A29
:1090B000484C00230121237003701360938089F8CA
:1090C00000103A4669464448FFF74EFD3043C6B2A9
:1090D000E6E71268BA1A1E2A6BD99AF80020934262
:1090E00022D0394C3D488AF80030012B276082EAB3
:1090F000030207609846B1D0042BAFD1374800680F
:10910000381AB0F5C87FA9D9354C2068381A3228EA
:10911000A4D927601A46A1E73A4669463148FFF7C5
:1091200023FD3043C6B2BBE7012B4FF00002E3D171
:10913000E4E73A4669462C48FFF716FD3043C6B2CD
:10914000AEE73A4669462948FFF70EFD3043C6B2FE
:10915000A6E73A4669462648FFF706FD3043C6B201
:109160009EE73A4669462348FFF7FEFC3043C6B205
:1091700096E73A4669462048FFF7F6FC3043C6B208
:109180008EE73A4669461D48FFF7EEFC3043C6B20B
:1091900086E73A4669461A48FFF7E6FC3043C6B20E
:1091A0007EE73A4669461748FFF7DEFC3043C6B211
:1091B00076E7002252E700BFB49FFF1F989FFF1F72
:1091C000009FFF1F949FFF1F8C9FFF1F149FFF1F77
:1091D000849FFF1F969FFF1F483D01009C9FFF1F1C
:1091E000089FFF1F783D0100C43C0100D83B0100EF
:1091F000E0490100D0490100C83B0100303C0100BA
:109200001C4A0100B090FF1FB88AFF1F049FFF1F78
:1092100028B11028044BA8BF102018607047024BDB
:1092200001201860704700BFA09FFF1F08B50020F5
:1092300006F09CFE0028FAD108BD00BF70B50D46AF
:109240001446064605F062FD284605F05FFD2046FF
:1092500005F05CFD084B1B7813B1084B1B7803B974
:1092600070BD304605F0E0F9284605F0DDF92046EE
:10927000BDE8704005F0D8B9F29DFF1F089EFF1FA2
:1092800038B5164D2B78044641F6FF72A0F5005014
:10929000824203F1FF33A8BF02461B0202F50052CF
:1092A00003F47063100443F4604343F00E0300F4CE
:1092B000FE005204184302F0FE42104306F08CFDFB
:1092C0002868013860F01F00C4F3C61204F07F0163
:1092D000C0B2BDE83840FFF7B1BF00BFA09FFF1F7D
:1092E00070B5104E3378013B1B0203F470630446E3
:1092F00043F430430806220400F0FE4043F00B0321
:10930000034302F4FE0018430D4606F065FD306885
:10931000013860F04F002A462146C0B2BDE87040D7
:10932000FFF78CBFA09FFF1F08B564210720FFF740
:10933000D7FF7F210B20BDE80840FFF7D1BF00BF5A
:1093400070B5104E3378013B1B0203F47063044682
:1093500043F410430806220400F0FE4043F00903E2
:10936000034302F4FE0018430D4606F035FD306855
:10937000013860F06F002A462146C0B2BDE8704057
:10938000FFF75CBFA09FFF1F38B50E4D2B78013B48
:109390001B0203F47063044643F41043000443F0DB
:1093A000090300F4FE00184306F016FD2868013892
:1093B00060F06F002146C0B20022BDE83840FFF7E0
:1093C0003DBF00BFA09FFF1F10B500217B20FFF70E
:1093D00087FF0024E0B2FFF7D7FF0134022004F03A
:1093E0009BFE802CF6D110BD38B50C46054605F025
:1093F0008DFC204605F08AFC074B1B7813B1074B08
:109400001B7803B938BD284605F00EF92046BDE8A3
:10941000384005F009B900BFF29DFF1F089EFF1FED
:1094200038B50D4D2B78013B1B0203F470630446E5
:1094300043F45043000443F00D0300F4FE001843CE
:1094400006F0CAFC2868013860F02F002146C0B23F
:10945000BDE83840FFF7C8BFA09FFF1F38B50E4DCD
:109460002B78013B01381B02C4B203F47063200463
:1094700043F4404343F00C0300F4FE00184306F0AD
:10948000ABFC2868013860F03F002146C0B2BDE85F
:109490003840FFF7A9BF00BFA09FFF1F38B50446A3
:1094A0000D46F02005F032FC35B1254414F8010BCF
:1094B00005F02CFCAC42F9D1F720BDE8384005F0AE
:1094C00025BC00BF00B50B4B83B0024699881868D5
:1094D0000090032AADF8041002D903B05DF804FB34
:1094E000684606218DF80520FFF7D8FF03B05DF828
:1094F00004FB00BF5C4A010000B50B4B024683B081
:10950000186899880090131F4C2BADF8041002D9ED
:1095100003B05DF804FB684606218DF80520FFF7CF
:10952000BDFF03B05DF804FB644A0100030203F4CD
:10953000FE43C0F3C6101843704700BF037840785D
:10954000DB0103F47E5300F07F001843704700BF37
:1095500082B002AA114642F8040D002012F8013B25
:1095600003F07F03914243EA0020F7D102B0704735
:1095700010B547F6122104460D4807F043F805F0F0
:10958000E5FB0C4B1B7833B974B1102C0A4BA8BF08
:1095900010241C6010BD47F61221084806F082FF17
:1095A00005F0FEF8002CF0D1034B01241C6010BD27
:1095B000BC92FF1FF29DFF1FA09FFF1FA892FF1FDD
:1095C000003210B403884FF0010404FA01F418BF0C
:1095D000012202FA01F123EA04020A43028010BCCC
:1095E000704700BF70B5CEB20C46054604F0EEF9E8
:1095F000864203D03146284604F002FA0135284657
:1096000004F0E4F9240A844205D021462846BDE846
:10961000704004F0F5B970BD38B5054604F0D6F9D0
:109620004FF0000460F30704681C04F0CFF960F306
:109630000F24A0B238BD00BFF8B504460020FFF7E4
:10964000EBFF002C00F077814FF4AF610220FFF7B1
:10965000C9FF04204FF47A61FFF7C4FF0B2004F028
:1096600025FD002840F02E874FF496610620FFF775
:10967000B9FF4FF4FA610820FFF7B4FF4FF4FA6125
:109680000A20FFF7AFFF40F6B8310C20FFF7AAFF22
:109690004FF42F612220FFF7A5FF40F6AC512420A4
:1096A000FFF7A0FF7D212A20FFF79CFF0C210E2051
:1096B000FFF798FF01211020FFF794FF02211220ED
:1096C000FFF790FF00211420FFF78CFF00211620E8
:1096D000FFF788FF02211820FFF784FF01211A20DD
:1096E000FFF780FF01211C20FFF77CFF04211E20D3
:1096F000FFF778FF14212020FFF774FF01212620B7
:10970000FFF770FF03212820FFF76CFF04212C20B6
:10971000FFF768FF14212E20FFF764FF002130209F
:10972000FFF760FF0C213220FFF75CFF002134209F
:10973000FFF758FF00213620FFF754FF00213820A3
:10974000FFF750FF00213A20FFF74CFF00213C209B
:10975000FFF748FF00213E20FFF744FF0021402093
:10976000FFF740FF00214220FFF73CFF1F2144206C
:10977000FFF738FF13214620FFF734FF0E21482062
:10978000FFF730FF11214A20FFF72CFF0A214C2060
:10979000FFF728FF00214E20FFF724FF062150206D
:1097A000FFF720FF02215220FFF71CFF0C2154205D
:1097B000FFF718FF00215620FFF714FF0021582063
:1097C000FFF710FF01215A20FFF70CFF08215C2052
:1097D000FFF708FF0A215E20FFF704FF0021602049
:1097E000FFF700FF04216220FFF7FCFE0121642047
:1097F000FFF7F8FE00216620FFF7F4FE0B2168203A
:10980000FFF7F0FE7F216A20FFF7ECFE00216C20BD
:10981000FFF7E8FE00216E20FFF7E4FE0021702034
:10982000FFF7E0FE00217220FFF7DCFE002174202C
:10983000FFF7D8FE1F217620FFF7D4FE13217820F2
:10984000FFF7D0FE0E217A20FFF7CCFE11217C20FD
:10985000FFF7C8FE0A217E20FFF7C4FE1F218020EB
:10986000FFF7C0FE13218220FFF7BCFE0E218420EB
:10987000FFF7B8FE11218620FFF7B4FE0A218820E9
:10988000FFF7B0FE00218A20FFF7ACFE00218C20FC
:10989000FFF7A8FE00219620FFF7A4FE00219820E4
:1098A000FFF7A0FE00219A20FFF79CFE05219C20D7
:1098B000FFF798FE06219E20FFF794FE0021A020CE
:1098C000FFF790FE7F21A220FFF78CFE40F2A461FB
:1098D000A420FFF787FE4FF4E161A620FFF782FE88
:1098E0000021A820FFF77EFE0021AA20FFF77AFEC4
:1098F0000221AC20FFF776FE0121AE20FFF772FEB9
:109900000121B020FFF76EFE0B21B220FFF76AFEA7
:109910002A210020FFF766FE0220FFF77DFEB0F54A
:10992000805F034616D34FF4AF610220FFF75AFE63
:109930004FF4AF630EE04FF6FF7398423FF484AEEE
:109940002A2840F0CB850220FFF766FEB0F5805F45
:109950000346E8D2D24A04201380FFF75DFEB0F53B
:10996000805F034680F06285CE4A06201380FFF7B1
:1099700053FEA0F52F739BB2B3F57A6F024606D95A
:1099800040F628210620FFF72DFE40F62822C64B80
:1099900008201A80FFF740FEA0F52F739BB2B3F5A5
:1099A0007A6F024606D940F6E4410820FFF71AFE16
:1099B00040F6E442BD4B0A201A80FFF72DFEA0F5C9
:1099C000FA739BB240F6AC518B42024606D94FF473
:1099D000FA610A20FFF706FE4FF4FA62B44B0C203E
:1099E0001A80FFF719FEA0F5FA739BB240F6AC514E
:1099F0008B42024606D940F6B8310C20FFF7F2FD43
:109A000040F6B832AB4B0E201A80FFF705FE18283F
:109A1000034600F20A84A84A10201380FFF7FCFDD9
:109A2000431E9BB20F2B024604D901211020FFF7E1
:109A3000D9FD0122A14B12201A80FFF7EDFD0A2863
:109A4000034600F2EC839E4A14201380FFF7E4FDE6
:109A50000128034604D900211420FFF7C3FD002389
:109A6000984A16201380FFF7D7FD7F28034600F29F
:109A7000D083954A18201380FFF7CEFD05280346B2
:109A800000F2C183914A1A201380FFF7C5FD0C280C
:109A9000034600F2C4848E4A1C201380FFF7BCFDED
:109AA0000428034600F2B4848A4A1E201380FFF77C
:109AB000B3FD0928034600F2A484874A20201380BE
:109AC000FFF7AAFD4628034600F29484834A222029
:109AD0001380FFF7A1FDA0F5FA739BB240F6AC51DD
:109AE0008B42024606D94FF42F612220FFF77AFD00
:109AF0004FF42F627A4B24201A80FFF78DFDA0F5DA
:109B0000FA739BB240F6AC54A342024604D92146F4
:109B10002420FFF767FD2246724B26201A80FFF7AC
:109B20007BFD7F28034600F25E846F4A2820138065
:109B3000FFF772FD0628034600F24E846B4A2A2086
:109B40001380FFF769FDA0F132039BB2B3F5967F56
:109B5000024604D97D212A20FFF744FD7D22644B73
:109B60002C201A80FFF758FD0C28034600F22D84A4
:109B7000604A2E201380FFF74FFD1E28034600F297
:109B80001D845D4A30201380FFF746FD09280346F7
:109B900000F20D84594A32201380FFF73DFD1E2844
:109BA000034600F2FD83564A34201380FFF734FD4C
:109BB0007F28034600F2EE83524C36202380FFF7C5
:109BC0002BFD7F28034600F2DF8338206380FFF7F8
:109BD00023FD7F28034600F2D1833A20A380FFF7BC
:109BE0001BFD7F28034600F2C3833C20E380FFF780
:109BF00013FD7F28034600F2B5833E202381FFF743
:109C00000BFD7F28034600F2A78340206381FFF706
:109C100003FD7F28034600F299834220A381FFF7CA
:109C2000FBFC394D28804420FFF7F6FC3028034622
:109C300000F28683354A46201380FFF7EDFC30287A
:109C4000034600F27783324C48202380FFF7E4FC80
:109C50003028034600F268834A206380FFF7DCFC6B
:109C60003028034600F25A834C20A380FFF7D4FC2F
:109C70003028034600F24C834E20E380FFF7CCFCF3
:109C80000128034604D900214E20FFF7ABFC002336
:109C9000204A50201380FFF7BFFC431E3CE000BF6A
:109CA000F49CFF1FBC9EFF1FAA9CFF1F8C9EFF1FE2
:109CB000589EFF1F6C9CFF1F3E9CFF1F0A9EFF1FAC
:109CC000429EFF1FEA9CFF1F429CFF1FFA9CFF1F42
:109CD000909CFF1F8A9CFF1F749CFF1F9E9EFF1F6E
:109CE000069EFF1F029EFF1F909EFF1F669EFF1F86
:109CF000B49EFF1F5A9CFF1FDC9CFF1FC89EFF1FC6
:109D00008E9EFF1FCC9DFF1FBE9EFF1F649CFF1FEA
:109D1000689EFF1F889CFF1F9BB20B2B024604D935
:109D200006215020FFF75EFC0622CF4B52201A80FE
:109D3000FFF772FC0428034600F2E482CB4A542069
:109D40001380FFF769FC431E9BB21D2B024604D90A
:109D50000C215420FFF746FC0C22C54B56201A80DC
:109D6000FFF75AFC0128034604D900215620FFF7CB
:109D700039FC0023BF4A58201380FFF74DFC7F2891
:109D8000034600F2B982BC4A5A201380FFF744FC14
:109D9000431E9BB2092B024604D901215A20FFF72A
:109DA00021FC0122B54B5C201A80FFF735FC431ED5
:109DB0009BB2102B024604D908215C20FFF712FC4D
:109DC0000822AF4B5E201A80FFF726FC431E9BB291
:109DD0001D2B024604D90A215E20FFF703FC0A224C
:109DE000A84B60201A80FFF717FC0228034600F2F8
:109DF0007D82A54A64201380FFF70EFC01280346EC
:109E000004D901216420FFF7EDFB01239F4A622062
:109E10001380FFF701FCC31E9BB2012B024604D93D
:109E200004216220FFF7DEFB0422994B66201A8092
:109E3000FFF7F2FB7F28034600F25282954A682022
:109E40001380FFF7E9FB7F28034600F24382924A22
:109E50006A201380FFF7E0FB7F28034600F234827C
:109E60008E4A6C201380FFF7D7FB0328034600F2CD
:109E700025828B4A6E201380FFF7CEFB19280346FC
:109E800000F21682874A70201380FFF7C5FB022874
:109E9000034600F20782844A72201380FFF7BCFB5E
:109EA0000628034600F2F881804A74201380FFF7E9
:109EB000B3FB0528034600F2E9817D4A8A2013801E
:109EC000FFF7AAFB0A28034600F2DA81794A8C20C0
:109ED0001380FFF7A1FB0428034600F2CB81764AEA
:109EE00098201380FFF798FB0128034604D900212E
:109EF0009820FFF777FB0023704A9A201380FFF722
:109F00008BFB0128034604D900219A20FFF76AFB46
:109F100000236B4A96201380FFF77EFB0B28034635
:109F200000F2A281674A9C201380FFF775FB831E15
:109F30009BB2032B024604D905219C20FFF752FB5C
:109F40000522614B76201A80FFF766FB3028034616
:109F500000F284815D4A78201380FFF75DFB302892
:109F6000034600F275815A4C7A202380FFF754FB98
:109F70003028034600F266817C206380FFF74CFBAB
:109F80003028034600F258817E20A380FFF744FB6F
:109F90003028034600F231818020E380FFF73CFB4C
:109FA0003028034600F223814A4A82201380FFF7BB
:109FB00033FB3028034600F21481474C8420238071
:109FC000FFF72AFB3028034600F2058186206380D4
:109FD000FFF722FB3028034600F2F7808820A38099
:109FE000FFF71AFB3028034600F2E980A020E38047
:109FF000FFF712FB0128034604D90021A020FFF738
:10A00000F1FA0023354A9E201380FFF705FBC31E9B
:10A010009BB20C2B024604D906219E20FFF7E2FAE0
:10A0200006222F4BA2201A80FFF7F6FA431E9BB29E
:10A030007E2B024604D97F21A220FFF7D3FA7F228C
:10A04000284BA4201A80FFF7E7FAA0F5AF639BB274
:10A05000B3F5167F024647D940F2A461A420FFF76A
:10A06000C1FA40F2A4623FE03689FF1F4289FF1F18
:10A07000BC89FF1FCA9CFF1F529EFF1F389CFF1FF9
:10A08000C089FF1F4089FF1FFE9DFF1F609EFF1FAD
:10A09000989CFF1FA09EFF1FC89CFF1F789CFF1F5E
:10A0A0002C9CFF1FE89EFF1FEC9DFF1FC49EFF1FFF
:10A0B000849EFF1F0C9EFF1FFC9DFF1F769CFF1FB1
:10A0C000D49CFF1F4C9EFF1F5C9CFF1F6E9CFF1FBC
:10A0D000DC9DFF1F709CFF1FE49DFF1F709EFF1FF4
:10A0E000A889FF1F929EFF1FD84BA6201A80FFF75A
:10A0F00093FAA0F5AF639BB2B3F5167F024606D97B
:10A100004FF4E161A620FFF76DFA4FF4E162D04B06
:10A11000A8201A80FFF780FA0628034600F2CC81B7
:10A12000CC4AAA201380FFF777FA0328034600F2EF
:10A13000BD81C94AAC201380FFF76EFA032803469D
:10A1400000F2AE81C54AB0201380FFF765FA0328FC
:10A15000034600F29F81C24AAE201380FFF75CFAEB
:10A160007F28034600F29081BE4AB2201380FFF799
:10A1700053FA7F2800F263812B88DFF808E3BA4F97
:10A18000BA4ABB4DBB4EBC4CBC4903F0010CAEF807
:10A1900000C0C3F3400EA7F800E0C3F380071780A8
:10A1A000C3F3C007B64A2F70C3F30017C3F34015BB
:10A1B000C3F38013378025800B801080F8BD0A21FF
:10A1C0008820FFF70FFA0A2310E711218620FFF7F6
:10A1D00009FA112302E70E218420FFF703FA0E2368
:10A1E000F4E613218220FFF7FDF91323E5E61F2192
:10A1F0008020FFF7F7F91F23D6E60A217E20FFF71C
:10A20000F1F90A23C8E602211820FFF7EBF902232F
:10A2100038E400211620FFF7E5F9002329E40221A4
:10A220001220FFF7DFF902230DE40C210E20FFF7C7
:10A23000D9F90C23FFF7EFBB11217C20FFF7D2F9EE
:10A240001123A1E60E217A20FFF7CCF90E2393E625
:10A2500013217820FFF7C6F9132384E61F21762007
:10A26000FFF7C0F91F2375E600219620FFF7BAF922
:10A27000002357E600218C20FFF7B4F900232EE6D7
:10A2800000218A20FFF7AEF900231FE60021742089
:10A29000FFF7A8F9002310E600217220FFF7A2F9CA
:10A2A000002301E600217020FFF79CF90023F2E56E
:10A2B00000216E20FFF796F90023E3E500216C20D2
:10A2C000FFF790F90023D4E57F216A20FFF78AF990
:10A2D0007F23C5E50B216820FFF784F90B23B6E542
:10A2E00000216620FFF77EF90023A7E5002160200A
:10A2F000FFF778F900237CE500215820FFF772F979
:10A30000002340E502215220FFF76CF9022315E5F6
:10A310000A214C20FFF766F90A23ADE411214A20F7
:10A32000FFF760F911239FE40E214820FFF75AF947
:10A330000E2391E413214620FFF754F9132382E4FE
:10A340001F214420FFF74EF91F2373E40021402012
:10A35000FFF748F9002360E400213E20FFF742F9AF
:10A36000002352E400213C20FFF73CF9002344E4A1
:10A3700000213A20FFF736F9002336E40021382087
:10A38000FFF730F9002328E400213620FFF72AF9EF
:10A3900000231AE400213420FFF724F900230BE402
:10A3A0000C213220FFF71EF90C23FFF7FCBB002124
:10A3B0003020FFF717F90023FFF7ECBB14212E2004
:10A3C000FFF710F91423FFF7DCBB04212C20FFF763
:10A3D00009F90423FFF7CCBB03212820FFF702F97A
:10A3E0000323FFF7ABBB01212620FFF7FBF8012376
:10A3F000FFF79BBB14212020FFF7F4F81423FFF78D
:10A4000065BB04211E20FFF7EDF80423FFF755BBC1
:10A4100001211C20FFF7E6F80123FFF745BB0121CE
:10A420001A20FFF7DFF80123FFF735BB4FF47A61FD
:10A430000420FFF7D7F84FF47A63FFF795BAB220FC
:10A440000B21FFF7CFF80B2096E600BFF89CFF1F0B
:10A45000789EFF1F3A9CFF1FAE9CFF1F629EFF1F4E
:10A46000F09DFF1F809CFF1FA89CFF1FDE9CFF1F0D
:10A47000089EFF1F009EFF1F649EFF1F149EFF1F6C
:10A48000A29CFF1F4E9EFF1F0121AE20FFF7AAF8DE
:10A49000012369E60121B020FFF7A4F801235AE661
:10A4A0000221AC20FFF79EF802234BE60021AA20F0
:10A4B000FFF798F800233CE60021A820FFF792F868
:10A4C00000232DE640F628210620FFF78BF840F602
:10A4D000E4410820FFF786F8FFF7D0B817287FF689
:10A4E000B3A819287FF622A91B287FF63FA91C28AC
:10A4F0003FF454A91E287FF659A91F283FF45EA9EE
:10A5000020283FF477A921283FF480A922283FF48E
:10A5100085A923283FF48EA924283FF4BFA9252824
:10A520003FF4C4A926283FF4C5A927283FF4CAA9A7
:10A5300028283FF4D5A929287FF4EAA9FFF7D8B93C
:10A54000F8B5C52007F030FD204B214A054603CB66
:10A550001368C5F803001A0CB420C5F807102B8047
:10A56000AA70FEF7E3FF2E46002426F80B0FA0B2D8
:10A57000FFF752F8FEF7DAFF0234B42C26F8020F88
:10A58000F5D16C1E05F1C0064FF0FF3014F8013F05
:10A59000082758400F4B40F300017A1E0B4012F081
:10A5A000FF0783EA5000F5D1B442EFD1C043FEF774
:10A5B000CFFF3A46C5F8C100C521284605F05AFC30
:10A5C0002846BDE8F84007F0F7BC00BF704A01001C
:10A5D0006C4A01002083B8EDF0B50E4B0E4C0546D9
:10A5E00093E8070085B024682E88AD7801AB83E836
:10A5F0000700270C184600220B21ADF804408DF807
:10A600000670ADF80C608DF80E5005F033FC05B007
:10A61000F0BD00BF7C4A01006C4A0100F0B5124B4E
:10A62000124D1E68124F0FCD87B06C460FC495E8CF
:10A63000030044F8040B38683B79CDF80D00320C68
:10A640002A2021808DF802208DF81130ADF80060AD
:10A65000FEF76CFF0022ADF80B001221684605F0F2
:10A6600009FC07B0F0BD00BF6C4A0100884A010038
:10A670000C3F0100002005F079BC00BF03F05EB97B
:10A6800070B5104C82B0002540230646294620466E
:10A69000009301958023202202F010FB0123202249
:10A6A00030462282A3826382E58108F009FA3146AE
:10A6B0000246204606F0ECF8204602B0BDE87040A5
:10A6C00002F0E2B8149FFF1FF0B5C42983B075D91A
:10A6D0000546441E00F1C0064FF0FF3014F8012F6C
:10A6E00008275040404A40F300017B1E0A4013F007
:10A6F000FF0782EA5000F5D1B442EFD1C043FEF724
:10A7000027FF0146D5F8C1000190019A914202D07D
:10A71000B2F17F2F0BD105F10B00FEF70FFFB4282C
:10A720000BD03248FFF7ACFF002003B0F0BD30483B
:10A73000FFF7A6FF384603B0F0BD05F10D00FEF7A8
:10A74000FDFE2A2840D1002440F6AC5613E0042830
:10A750001AD0062821D008281FD00A2828D00C2873
:10A7600022D1A1F5FA7292B2B24201D8FEF73AFFB5
:10A770000234B42C0ED004F10D002844FEF7DEFEA6
:10A78000022C0146A0B2E2D1B1F5805FEED30234D3
:10A79000B42CF0D1012003B0F0BDA1F52F7292B21C
:10A7A000B2F57A6FE4D8E1E7222801D0242811D14C
:10A7B000A1F5FA7292B2B242DAD8D7E70D48FFF7A4
:10A7C0005FFF002003B0F0BD0B48FFF759FF0020EA
:10A7D00003B0F0BD2A28C9D1A1F1320292B2B2F57C
:10A7E000967FC5D8C2E700BF2083B8EDCC4A0100F0
:10A7F000B84A0100A04A0100E04A010003290CD92F
:10A8000070B5461C82B005460C46304603222A49E4
:10A8100008F0C4F910B102B070BD70470B2C05D917
:10A8200005222649281D08F0B9F940B12448FFF750
:10A8300027FF244802B0BDE87040FFF7CDBE05F108
:10A840000901032201A808F0F9F901A803221E4911
:10A8500008F0A4F9D8B103221C4901A808F09EF918
:10A8600008B301A803221A4908F098F9B0B91948A9
:10A87000FFF706FFA11E89B23046FFF725FF00282B
:10A88000C9D0154802B0BDE87040FFF7F9BE1348C3
:10A89000FFF7F6FEFFF754FE1148F3E71148FFF704
:10A8A000EFFE1148C6E71148FFF7EAFE02B0BDE827
:10A8B0007040FFF7B3BE00BF6C4A0100243F0100A7
:10A8C000F84A01000C4B0100104B0100384B01000D
:10A8D000504B0100544B0100684B0100144B010028
:10A8E000284B01007C4B0100904B01003C4B0100C8
:10A8F0002DE9F043174D2B6883B081460F469046F3
:10A90000F3B1154E34880A1992B2184611463280B6
:10A9100007F0C8FE28603A464946204402F092FDFE
:10A92000B8F1000F09D031882868FFF767FF286861
:10A9300007F042FB00232B60338003B0BDE8F083B7
:10A94000054E01930846318007F02EFB019B2860DD
:10A950001C46E0E7A89FFF1FA49FFF1F10B51D4CDA
:10A960004FF4FA70FBF718FE204601F081FE002339
:10A97000194601222046E3812382A282628202F0EC
:10A9800059FD0B221449204605F082FF204605F0B0
:10A9900095FF0F221149204605F07AFF204605F069
:10A9A0008DFF0F490722204605F072FF204605F073
:10A9B00085FF204601F068FF0A4B0B4A1A604FF4EE
:10A9C000FA70FBF7E9FDFFF729FE0848BDE81040E3
:10A9D000FFF756BE149FFF1F944B0100A04B0100D0
:10A9E000B04B0100BCA1FF1FF1A80000B84B010053
:10A9F0000020704790F8392090F83800101A7047FE
:10AA000090F8383090F839209A4205D95A1C0344FE
:10AA100080F83820187E70474FF0FF30704700BF35
:10AA200090F8383090F839209A4286BF1B18187E6B
:10AA30004FF0FF30704700BF704700BF38B5054684
:10AA4000B0F85E0090B195F85D301446C3F1210274
:10AA500094420CD805F13B001844224602F0F2FC67
:10AA600095F85D30234485F85D30204638BD0120DF
:10AA700014462871EEE700BFB0F85E306BB190F875
:10AA80005D30202B07D8C218013380F85D300120DB
:10AA900082F83B107047012303710020704700BF0C
:10AAA0000023426980F8383080F8393080F85C3013
:10AAB00080F85D3080F85E3080F85F3006CA30B4D0
:10AAC0000D68046943662A4383660A60A37042697D
:10AAD00090F861301649146813441D7A5B7B01EBD2
:10AAE000C5051B026D6803F4E06343F064032B604B
:10AAF00090F8623013449D7CDB7D01EBC5011B02A5
:10AB0000496803F4E06343F064030B602168536811
:10AB1000194205D0036927225A70036904229A71E9
:10AB2000036920225A71036980229A7030BC7047F1
:10AB3000DC56010043690CCB12681A420CD0094B59
:10AB400099420AD9084B9942036994BF1A220D22EF
:10AB50005A70036904229A717047036927225A7058
:10AB6000F7E700BF7F1A06003F420F0010B50269E9
:10AB7000D378DBB2D90604463DD510215806D170F2
:10AB800038D503F0040303F0FF02002B51D03D49F8
:10AB9000626E00230B7084F85D30002A5BD0904712
:10ABA00094F85D30002B56D02369D0229A70236927
:10ABB00094F83B201A712369012284F85C20022258
:10ABC000DA7010BD304B84F860009C424AD02F4BA5
:10ABD0009C4252D094F8391013791F29DBB207D860
:10ABE0002848007820B16018013184F839100376C4
:10ABF0000223D37010BD5906C3D4917801F010011F
:10AC000001F0FF000029DDD013F001031ED194F8FC
:10AC10005C1094F85D00884281BF4B1C091984F8D0
:10AC20005C3091F83B3013712369D0229A7022690D
:10AC3000DEE7236984F83920C0229A702369114A1B
:10AC40001979012111700222DA7010BDC0239370AE
:10AC500022691379CCE70122002384F85D2084F86F
:10AC60003B30A1E7626994F861300949134403223B
:10AC7000187A02F0B3FF2269ACE7626994F8613098
:10AC80000449F3E7AC9FFF1FE090FF1F4C91FF1FAB
:10AC9000F5AC000001AD00000369DB7803F0200390
:10ACA00073B190F860300133DBB2012B80F8603073
:10ACB0001AD9426990F861301344187A03F00AB83F
:10ACC00070B5426903F0FF0590F861301344044603
:10ACD000187A02F0FFFFA36E5BB184F8385094F845
:10ACE0003900BDE87040184790F85F30002BE0D085
:10ACF000704770BD0148FFF7CFBF00BFE090FF1F56
:10AD00000148FFF7C9BF00BF4C91FF1F2DE9F04775
:10AD1000374FDFF8E0903B68026982B00646009347
:10AD2000DDF800800021A025D3789B065BD53B6829
:10AD30000193019BC8EB03030F2BF5D949B1102BED
:10AD4000F2D000209070336980229A7002B0BDE882
:10AD5000F087726996F8613013440521187A03F080
:10AD6000B3F9726996F861301344012193F812A087
:10AD7000504603F0A9F909240021504603F090F948
:10AD80002B46013BFDD10121504603F089F92B46AA
:10AD9000013BFDD1013CEFD1706996F8611001448F
:10ADA0004FF4A0720C7A4B7B09EBC4011B0249687B
:10ADB00003F4E06343F064030B6096F862300344ED
:10ADC000997CDB7D09EBC1011B02496803F4E06358
:10ADD00043F064030B60013AFDD13269D3789B06DE
:10ADE0004FF00101A3D4012002B0BDE8F08700BFFD
:10ADF000B49FFF1FDC560100F0B503691222DA7020
:10AE00000269937803F0200385B004460D46002BB9
:10AE10005ED0B42393703C4922690B680093009E76
:10AE200005E00B680193019B9B1B042B42D8D37850
:10AE300003F0200303F0FF00002BF2D094F85D3004
:10AE4000002B31D04FF0000E4FF0020C04EB0E033C
:10AE500093F83B3013710B680393039F206907E05D
:10AE60009B060DD50B680293029BDB1B052B28D894
:10AE7000C378DBB203F0020202F0FF06002AEFD033
:10AE800080F803C02669F378DBB2DF0632462DD4A2
:10AE90009F062BD5DB0731D40EF1010E94F85D30FF
:10AEA0005FFA8EFE7345D1D800201DBB002384F8C5
:10AEB0005E3004E09070236980229A70042005B00F
:10AEC000F0BD86702369802204209A7005B0F0BD21
:10AED00003F0FF06FFF71AFF10B9042005B0F0BD1C
:10AEE000236984F85F60B0229A7094E78023B3707E
:10AEF0000420DAE726698023B370D7E7BEF1000F9C
:10AF00000CBF02200320F6E7B49FFF1F2DE9F0419C
:10AF100006690025122780F8385080F83950F770FC
:10AF2000D0F810C09CF802E00EF0200E88B0044665
:10AF3000884615461E46BEF1000F49D0B4238CF852
:10AF40000230784B21691A680092DDF800E006E0D3
:10AF50001A6801920198CEEB0000042830D8C87816
:10AF600000F0200000F0FF070028F1D04FEA48026F
:10AF700042F00102D2B20A711A680292DDF808E0CA
:10AF8000206906E01A6803920399CEEB01010529B6
:10AF90002AD8C17801F0020101F0FF070029F1D0A1
:10AFA0004FF0020C80F803C02269D17811F011072C
:10AFB00022D12DBB002E0CBFA0238023937003E071
:10AFC0008F70236980229A70384608B0BDE8F081FE
:10AFD0000EF0FF07FFF79AFE0028F5D0236984F8EA
:10AFE0005F70B0229A70ACE7877023698022384680
:10AFF0009A7008B0BDE8F081802393700027E3E7E2
:10B00000012D75D0A021917021690A79BE4667464D
:10B010004FF0A80C1A680492049805E01A6805928B
:10B02000059A121A052A4AD8CA7802F0020202F0DA
:10B03000FF08002AF2D0CF702169CA78D2B212F08C
:10B04000100F08465AD1920658D5013DEDB2012D98
:10B0500049D0BEF11F0F3BD90A79012DDAD11A6808
:10B060000692069D05E01A680792079A521B052A68
:10B0700046D8C27802F0020202F0FF01002AF2D0A4
:10B080000223C3702269D378DBB2D9063AD49B0677
:10B0900034D5B023BEF11F0F93703FD8226904EB63
:10B0A0000E0312791A760EF1010E5FFA8EFE16B1BA
:10B0B000236980229A7084F839E0774684E781F822
:10B0C0000280236980229A70774684F839E07BE712
:10B0D00004EB0E0291F8048082F818800EF1010E44
:10B0E0005FFA8EFEB9E781F802C021690846B0E731
:10B0F000A82191702069BE460279B0E7774663E7E0
:10B100008170DEE71021A023D170013BFDD12269BF
:10B11000937803F0F7037746937055E723691B791B
:10B12000C5E700BFB49FFF1F0148FFF71FBD00BF69
:10B13000E090FF1F0148FFF719BD00BF4C91FF1FB2
:10B1400000220260704700BF30B5056889B0012356
:10B1500000240A460193294602A8009400F006F94B
:10B1600002A800F0ADF9C0B209B030BD30B5056835
:10B1700089B0012400230A468DE8180029460223DD
:10B1800002A800F0F3F802A800F09AF980B209B022
:10B1900030BD00BF0C2901D90020704702314900A1
:10B1A00001F0FE01FFF7E2BF2DE9F04303688FB025
:10B1B000012600240D4607461946904633465E2276
:10B1C00002A80196009400F0D1F802A800F078F9E6
:10B1D0005E2D03D0A5F17303072B10D801230024A3
:10B1E000396801932A4608A8009400F0BFF8224667
:10B1F000414608A800F006F90FB0BDE8F08381468B
:10B200002246214602A800F0FDF8396833462A4656
:10B210008DE8500008A800F0A9F82246414608A889
:10B2200000F0F0F822465FFA89F102A800F0EAF88F
:10B230000FB0BDE8F08300BFF8B505460F461646CF
:10B24000412421463A462846FFF7AEFF611C0234EE
:10B25000C9B232462846E4B2FFF7A6FF592CF0D116
:10B26000F8BD00BF2DE9F843044600689DF8209022
:10B270000E461746984610B1102105F081FB1020AC
:10B2800005F07CFB3A460546314600F057F925604B
:10B290002846012100F078F9054618B9002528460E
:10B2A000BDE8F883632280212046FFF77DFF01205F
:10B2B00002F032FF00225E212046FFF775FF5D217C
:10B2C0002046FFF741FF2428E8D14A464146204660
:10B2D000FFF7B2FF204601222B21FFF765FF204632
:10B2E00001222C21FFF760FF20460E222D21FFF7BF
:10B2F0005BFF204600222E21FFF756FF2046012249
:10B300002F21FFF751FF204605223021FFF74CFF88
:10B31000204601223121FFF747FF2046002232213B
:10B32000FFF742FF204600223321FFF73DFF204672
:10B3300000223421FFF738FF204600223521FFF795
:10B3400033FF204600225B21FFF72EFF204610220C
:10B350005C21FFF729FF204620225D21FFF724FF13
:10B3600020468C225E21FFF71FFF98E770B49DF8FE
:10B3700010609DF80C500160002146738573428176
:10B3800003734161416070BC704700BFF0B54389F1
:10B39000056885B0DCB21B128DF80C408DF80D30BD
:10B3A0004DB1437B019303AB00932846012300F08A
:10B3B000FBF805B0F0BD43680BB31746027A0E46A2
:10B3C0006AB904F07F048DF80C40427B009231464C
:10B3D0003A46184603AB00F055FA05B0F0BD022A14
:10B3E00004D164F07F048DF80C40EEE7012AECD123
:10B3F00004F07F0444F040048DF80C40E5E7184663
:10B40000D7E700BF02B9027B042A1AD8F0B4416121
:10B4100000F10F077AB102F10E03867B3C4603442C
:10B4200000F10E055EB92170013BAB424FEA1121DC
:10B4300004F10104F6D13946F0BCFFF7A7BF19703B
:10B44000F2E70020704700BF70B54489066884B0F9
:10B45000E5B224128DF80C508DF80D405EB1437B9F
:10B46000009200241A4630460B46019403A900F0CE
:10B470000BF904B070BD4468FCB1037A7BB965F088
:10B480007F058DF80C50437B0092FF251A4620461D
:10B490000B46019503A900F08BFA04B070BD022B96
:10B4A00004D105F07F058DF80C50ECE7012B04BFAB
:10B4B00065F03F058DF80C50E5E72046D9E700BF61
:10B4C00038B500F10F042146027B0546FFF7BCFFAB
:10B4D00010B94FF0FF3038BD287B0028FBD00E306C
:10B4E0002B18AA7B21460E35002007E01C78013B73
:10B4F000AB4240EA040001F101010AD00002002A37
:10B50000F4D00C78013BAB4240EA040001F10101A8
:10B51000F4D138BD70B5044640681E4603685B68C8
:10B5200015469847854201D0002070BD31466068BD
:10B53000FFF762FCB0FA80F0400970BD30B400251E
:10B5400020240572C4600170426030BC704700BFA7
:10B55000037A10B5044683B1227863680121520052
:10B5600083F83B2083F85E1083F85D106068FFF776
:10B5700043FCB0FA80F0400910BD012100F004F84E
:10B580000028E9D110BD00BF38B5044640680D461B
:10B59000FFF786FA0120207205B938BD2046BDE8C4
:10B5A0003840FFF7D5BF00BF2DE9F041079EC468C2
:10B5B000DDF818E09519A54219D815460278984685
:10B5C00043680F4652000121044683F83B2083F86C
:10B5D0005E1083F85D106EB1BEF1000F0AD04068B6
:10B5E000036871465B6832469847864202D0002065
:10B5F000BDE8F08143462A4639462046BDE8F04181
:10B60000FFF788BF2DE9F843C468A24202D90020A1
:10B61000BDE8F88316468846074601784068D2B2EE
:10B62000FFF774FC8642F2D136B30023DFF8549062
:10B630001C4612E090F8383090F839209A4203F115
:10B64000010E00EB03011AD980F838E0087E28705B
:10B650000134A4B2A64223460ED978680268526922
:10B660004A4508EB0305E5D090470134A4B2C0B2C7
:10B67000A64228702346F0D80120BDE8F883FF20B9
:10B68000E5E700BF01AA00002DE9F041C568069F6B
:10B690009DF81C60AA4202D90020BDE8F08190F814
:10B6A00000C0D0F804E04FF001084FEA4C0C1D46F2
:10B6B0008EF83BC033468EF85E808EF85D8004467F
:10B6C000FFF728FF0028E7D043463A4629462046A0
:10B6D000BDE8F041FFF796BF2DE9F0470468134637
:10B6E0000A4624B12046BDE8F04700F035BB057B93
:10B6F0000C7886686249B1FBF6F1002D0CBF4FF063
:10B7000001094FF0800919EA040F0CBF4FF0010C3A
:10B710004FF0000CCDB2002B00F0AF804F0107F4CA
:10B72000FF57114602EB030811F801EB4B460026C8
:10B73000002D50D0002F4ED03A46013AFDD1427B29
:10B7400012F0F70F40F08D8090F91020013212D0E6
:10B750001EEA030214BF0124002464450BD0002A12
:10B760006CD0446990F8242094F800C04CEA02029E
:10B7700022704FF0010C846990F8262094F800A004
:10B780004AEA020222701DB117B13A46013AFDD1D0
:10B7900090F91120013206D0C26990F82540127844
:10B7A000224218BF1E43826990F826A0147824EA2A
:10B7B0000A04147090F91120013201D001F8016CD3
:10B7C000027B002A35D15B00DBB2002BB0D188456B
:10B7D000AAD1BDE8F087427B12F0F70FB4D084699C
:10B7E00090F8262094F800A04AEA0202227090F90C
:10B7F000102001320AD01EEA030F44692AD090F8C3
:10B80000242094F800A04AEA02022270846990F889
:10B8100026A0227822EA0A02227090F91120013231
:10B82000CED0C26990F825401278224218BF1E433C
:10B83000C4E75B08002B7FF47BAFC8E7D0F814A007
:10B8400090F824C09AF8004024EA0C048AF80040DA
:10B85000944690E790F824A0227822EA0A02227007
:10B86000D4E7846990F8262094F800A04AEA0202FE
:10B8700022703A46013AFDD1B9E7BDE8F08700BF32
:10B8800020A107002DE9F0430C4683B001680A9F10
:10B89000064690461D4681B14268CB7A1268002B5D
:10B8A0004ED10B68D968914207D0394818603949A0
:10B8B000DA6042F08040186119600021B07B02F02C
:10B8C000EFFB77B105EB07090DF1070715F8013B11
:10B8D0008DF80730012239463046FFF7FDFEA945B5
:10B8E000F4D1B8F1000F0ED004EB08050DF10707F5
:10B8F00014F8013B8DF80730012239463046FFF736
:10B90000EBFEA542F4D10121B07B02F0C9FB336804
:10B9100093B1DA7A82B1D00703D51F4A99691160D1
:10B92000DA7A910703D51D4AD9691160DA7A52078C
:10B9300002D51B4A1B6A1360012003B0BDE8F083E7
:10B9400072B6CB7AD80709D5DFF858E0C868DEF8B8
:10B95000003003408B61CEF80030CB7A980709D5D0
:10B96000DFF844E00869DEF800300340CB61CEF830
:10B970000030CB7A5B0708D5DFF830E04869DEF8A5
:10B98000003003400B62CEF8003062B689E700BF9A
:10B9900001403F0000003F8000E100E004E100E0E2
:10B9A00008E100E080E100E084E100E088E100E0FF
:10B9B0002DE9F0470D4682B00168DDF828909DF82A
:10B9C0002C80064617461C4681B14268CB7A126825
:10B9D000002B4FD10B68D968914207D039481860C5
:10B9E0003949DA6042F08040186119600021B07B6B
:10B9F00002F056FB77B105EB070A0DF1070715F8C2
:10BA0000013B8DF80730012239463046FFF764FECE
:10BA1000AA45F4D1B9F1000F0FD0A1440DF10707E9
:10BA20000122394630468DF80780FFF755FE9DF814
:10BA3000073004F8013BA145F2D10121B07B02F0AF
:10BA40002FFB336893B1DA7A82B1D00703D51F4A4E
:10BA500099691160DA7A910703D51D4AD969116095
:10BA6000DA7A520702D51B4A1B6A1360012002B022
:10BA7000BDE8F08772B6CB7AD80709D5DFF858E071
:10BA8000C868DEF8003003408B61CEF80030CB7A16
:10BA9000980709D5DFF844E00869DEF80030034074
:10BAA000CB61CEF80030CB7A5B0708D5DFF830E009
:10BAB0004869DEF8003003400B62CEF8003062B611
:10BAC00088E700BF01403F0000003F8000E100E048
:10BAD00004E100E008E100E080E100E084E100E052
:10BAE00088E100E02DE9F0410468E56815F0807F09
:10BAF000794D256052D1DF0740F1B380002900F075
:10BB0000E3800D78012B18BF45F0004565630131D6
:10BB100090F8248003F1FF3C48EA0828BCF1000FAC
:10BB200000F0A88021B14D7811F8028B45EA082871
:10BB300045682E7ABCF1020F06F1FF364FEA063651
:10BB40000CBF48F0805548F01045B6B26563ACF1C3
:10BB5000020C08E00AB114700132013B05F4704593
:10BB6000B54216D90468E56A15F0F00FF6D0A46B5B
:10BB700013F0010F17464FEA242EEBD11AB107F844
:10BB800002EB54703A4605F47045B542A3F1020346
:10BB9000E8D8BCF1000F6DD00468C3E7DD074CD5D1
:10BBA000002900F089800D78012B18BF45F0004571
:10BBB0006563013103F1FF3E90F824C0BEF1000F30
:10BBC00041D029B191F801C00D78023145EA0C2C21
:10BBD00045682E7ABEF1020F06F1FF364FEA0636AF
:10BBE0000CBF4CF080554CF01045B6B26563AEF119
:10BBF000020E08E00AB114700132013B05F47045F1
:10BC0000B54215D90468E56A15F0F00FF6D013F0C7
:10BC1000010F1746A46BEDD122B107F8024B241295
:10BC200054703A4605F47045B542A3F10203E9D8D1
:10BC3000BEF1000F07D00468C3E79E4690F824C009
:10BC4000BEF1000FBDD11BB30468E16A11F0F00F23
:10BC5000FBD0A16BDC071DD50AB111700132013B8D
:10BC6000F1E790F824809C4648EA0828BCF1000FD0
:10BC70007FF458AF63B10468E16A11F0F00FFBD0B4
:10BC8000DE07A16B0FD50AB111700132013BF1E75C
:10BC9000BDE8F0812AB114460D1204F8021B55705C
:10BCA0002246023BCFE72AB114460D1204F8025B8C
:10BCB00051702246023BDDE790F82450012B18BF5B
:10BCC00045F00045656375E790F82450012B18BFD7
:10BCD00045F0004565631BE700041F8090E80C00F9
:10BCE000F0B41C6859682568164F174E2943216027
:10BCF000164D17491760D66015611160417A154AD3
:10BD00005C180A3194F8244053F8215002EBC40126
:10BD100049680D60017A5C1803EB8101247ECD69CE
:10BD200002EBC40149680D60817A581803EB810366
:10BD300090F83000596B02EBC002F0BC53681960F8
:10BD4000704700BF01401F0001100038011000784B
:10BD500000001F80DC5601000BB1FFF7C3BE704727
:10BD6000704700BFF0B50C1EBDF8146034DBB0F9AD
:10BD700006701919B942C4BF3B1B1BB2002BA64663
:10BD80001CDD002A1146B8BFD11D02F00705CC10FA
:10BD9000826A012007FB04E1A840012E0A44C0B2D8
:10BDA0001ED00CD3022E09D1013B12FA83F3013AC3
:10BDB00012F8011F41409A421170F9D1F0BDC04301
:10BDC000013B12FA83F3C0B2013A12F8011F01409D
:10BDD00093421170F9D1F0BD23441BB20024C6E791
:10BDE000013B12FA83F3013A12F8011F01439A4210
:10BDF0001170F9D1F0BD00BF00291EDB30B4B0F9DD
:10BE00000A408C4218DD002A16DBB0F90C4094423F
:10BE100012DD047E022C54D0032C4CD0012C06D110
:10BE20005140C4884A405140013C611A09B2012B7B
:10BE30002DD017D3022B01D030BC7047002AB0F9A7
:10BE40000630856A1446B8BFD41D44F3CF0404FB02
:10BE5000031102F007026B5C012000FA02F25A4063
:10BE60006A54E9E7002AB0F90630856A1446B8BF7B
:10BE7000D41D44F3CF0404FB031102F007026B5CF2
:10BE8000012000FA02F223EA02026A54D4E7002AEF
:10BE9000B0F90630856A1446B8BFD41D44F3CF0408
:10BEA00004FB031102F007026B5C012000FA02F2AE
:10BEB0001A436A54C0E70489013C641A114622B24D
:10BEC000B5E7C5880489013D013C691AA21A09B287
:10BED00012B2ACE72DE9F041079E9DF91880089D4C
:10BEE00004461F4600F0BCFF0D4B0E480E4984F877
:10BEF0003380FF22002F08BF1F4684F82F20002325
:10BF000084F8302084F8312084F83220206066657F
:10BF1000A565676221662362A3622046BDE8F081C1
:10BF2000E090FF1F444C01000110013810B5044699
:10BF3000806A034B236008B106F03EF8204610BD2E
:10BF4000444C0100F8B5436ADBB190F82C20012580
:10BF5000AA4083F83B2083F85E5083F85D50044686
:10BF6000406A03680E461B6800219847606A0368B0
:10BF700031461B6898472946606ABDE8F840FEF7DD
:10BF80003BBFC26BC56C1368046A23EA05031360E8
:10BF90004CB122684FF00043D3625163D36A002B47
:10BFA000FCDA936BF8BD836B466B0825802410E0A8
:10BFB0003768426C3A4332601F68826C3A431A60B9
:10BFC0001A68876C013D22EA07024FEA54041A609E
:10BFD00007D02142ECD13268476C22EA0702326076
:10BFE000EAE7F8BD70B50446406A0D4600282BD03C
:10BFF000616DFEF79FFD002D20460CBFA621A721F5
:10C00000FFF7A0FF606A20B1A16DBDE87040FEF7A8
:10C0100091BD216C226D0868236A02430A6093B1C6
:10C02000DA7A82B1D00703D5224A99691160DA7AA7
:10C03000910703D5204AD9691160DA7A520702D5EF
:10C040001E4A1B6A136070BD236A002B2BD0D97A5D
:10C05000226EE1B172B6D97ACE0706D51848D968F2
:10C060000668314099610160D97A880706D515487C
:10C07000196906683140D9610160D97A4E0705D542
:10C0800011485969066831401962016062B61B683F
:10C09000D968914207D00D4818600D49DA6042F026
:10C0A000804018611960226C216D136823EA010336
:10C0B0001360A0E700E100E004E100E008E100E037
:10C0C00080E100E084E100E088E100E001403F0021
:10C0D00000003F80436A2DE9F04105460E46904638
:10C0E000002B3ED090F82C100124A14083F83B1087
:10C0F00083F85E4083F85D40406A036800211B6856
:10C1000008F1FF379847FFB2B8F1000F23D037444A
:10C11000A046013E686A16F8011F03681B6898472D
:10C120000134B742A4B216D01F2CF3D90121686A9A
:10C13000FEF762FE95F82C206B6A520083F83B20D4
:10C1400083F85E8083F85D80686A036800211B685D
:10C1500098470124DEE7686A0121BDE8F041FEF757
:10C160004BBEC26BC16C136823EA010306EB0804E3
:10C1700013604FF00048A6420ED02B6A16F801EB70
:10C1800063B11A68C2F82C80C2F834E0D36A002B7D
:10C19000FCDAA642936BF0D1BDE8F081AB6BD5F829
:10C1A00034C008208021DCF800206F6C1EEA010FEB
:10C1B00014BF3A43BA43CCF800201A68AF6C3A4334
:10C1C0001A601A68AF6C013822EA07024FEA51017F
:10C1D0001A60E8D1CFE700BF70B50446406A0D464B
:10C1E000002828D0616DFEF7A5FC20462946FFF700
:10C1F000A9FE606A20B1A16DBDE87040FEF79ABC4F
:10C20000216C226D0868236A02430A6093B1DA7ACE
:10C2100082B1D00703D5234A99691160DA7A910770
:10C2200003D5214AD9691160DA7A520702D51F4A2B
:10C230001B6A136070BD236A002B2BD0D97A226E43
:10C24000E1B172B6D97ACE0706D51948D968066821
:10C25000314099610160D97A880706D51548196976
:10C2600006683140D9610160D97A4E0705D5124878
:10C270005969066831401962016062B61B68D96865
:10C28000914207D00D4818600D49DA6042F08040B5
:10C2900018611960226C216D136823EA0103136091
:10C2A000A3E700BF00E100E004E100E008E100E0F6
:10C2B00080E100E084E100E088E100E001403F002F
:10C2C00000003F802DE9F041044686B0806A9DF869
:10C2D00030801E460F461546B4F90830002800F09D
:10C2E0004B81DA1D48BF03F10E02B4F90630D210BB
:10C2F00003FB02F2002106F083F9B4F90820202A9A
:10C3000000F3A780B4F90610A74B0120203A733937
:10C3100002EBD27201EBD1714FF0200E029073202C
:10C320008DE8014042F34F0241F34F01204600F0F7
:10C330004DFE606A84F82D70002800F05181002DB8
:10C3400040F09F80B4F90830202B14BF3D253C25D8
:10C3500084F82C50B8F1000F40F09A8006B394F99D
:10C360003300002818DBC0B2012101F0ADFE01212D
:10C3700094F8330001F094FE012001F0CDFE00217D
:10C3800094F8330001F08CFE0A2001F0C5FE012173
:10C3900094F8330001F084FE606A002800F0988071
:10C3A000616DFEF7C7FB042280492046FFF792FE2D
:10C3B000217A0139C9B22046FFF7C4FD7C49042225
:10C3C0002046FFF787FE94F92D30012B14BF14216E
:10C3D00010212046FFF7B6FD042276492046FFF7DC
:10C3E00079FEB4F906308F22802B84F85C2000F0AF
:10C3F000A580602B00F0B1800225DA212046FFF7EE
:10C40000A1FD29462046FFF79DFD81212046FFF72B
:10C4100099FD94F85C102046FFF794FDD921204641
:10C42000FFF790FD94F92D30012B14BFF12122214B
:10C430002046FFF787FD204606225F49FFF74AFEA8
:10C44000606A58B3A16DFEF775FB012006B0BDE828
:10C45000F081B4F90610594B0120403A52394FF09F
:10C46000400E029002EBD272522001EBD1718DE8A6
:10C47000014042F34F0241F34F01204600F0A6FD78
:10C4800057E76DB284F82C50B8F1000F3FF466AF57
:10C49000FEF706FB002E3FF47FAF60E7216C226DB4
:10C4A0000868236A02430A6073B1DA7A62B1D0077E
:10C4B00003D5434A99691160DA7A91076FD452071C
:10C4C00002D5404A1B6A1360012006B0BDE8F08126
:10C4D000236A002B2BD0D97A226EE1B172B6D97AB9
:10C4E000CF0706D53848D9680568294099610160A9
:10C4F000D97A8E0706D53548196905682940D9616A
:10C500000160D97A4D0705D5314859690568294038
:10C510001962016062B61B68D968914207D02D4844
:10C5200018602D49DA6042F0804018611960226C71
:10C53000216D136823EA0103136034E7B4F908306E
:10C54000402B7FF459AF94F92D30012B14BFCF232A
:10C550009F2384F85C3012254FE7B4F90830102B84
:10C560007FF44AAF94F92D30012B14BFAF23102371
:10C5700084F85C30022540E7DA1D48BF03F10E0263
:10C58000B4F90630D21003FB02F21046059205F012
:10C590000BFDA06200283FF459AF059AAAE60F4AA6
:10C5A000D9691160DA7A8AE7944C0100744E01006F
:10C5B000784E01007C4E0100804E0100884E010043
:10C5C00000E100E008E100E080E100E084E100E05B
:10C5D00088E100E001403F0000003F8004E100E00E
:10C5E000012194F83100214F01F06EFD94F83200E2
:10C5F000012101F069FD94F9312094F9323057F8A6
:10C600003220E26357F83330206A23640125E56461
:10C6100025651A682A431A6048B1B8F1000F3FF443
:10C6200039AFFFF75BFB002E3FF4B6AE97E6294625
:10C6300094F82F0001F048FD294694F8300001F0ED
:10C6400043FD94F92F2094F9303057F8322062637B
:10C6500057F833306564A5641A68A36322F00102B9
:10C660001A60002E3FF498AE79E600BFDC56010058
:10C67000B0F90820D31D48BF02F10E03B0F906201F
:10C68000806ADB1002FB03F2002105F0B9BF00BF96
:10C69000F0B50029BDF814502EDBB0F90660B142A8
:10C6A0002ADA002A59DBB0F9087014461C44BC424F
:10C6B000C4BFBB1A1BB2002B1EDDD2B2D408D0F807
:10C6C00028E016FB041112F00702DBB20EEB0104A6
:10C6D00021D0C2F10807FAB2374F9342BF5C0CD2A7
:10C6E000C3EB020CFF2646FA0CF6012D07EA0607FB
:10C6F0003FD005D3022D36D0F0BD012D39D030D238
:10C700001EF8016026EA07070EF801709342F3D382
:10C71000B0F906100C449A1AD2B2072A10D9022D89
:10C7200036D0002D14BFFF26002613462670083B86
:10C73000B0F90610DBB2072B0C44F7D802F0070261
:10C74000002AD9D01D4B012D9B5C1DD017D3022D83
:10C75000D2D1227853402370F0BD13441BB2002283
:10C76000A1E7022D25D11EF8016077400EF8017077
:10C77000CCE71EF8016037430EF80170C6E7227857
:10C7800022EA03032370F0BD227813432370F0BD27
:10C7900011462378DB4323700839B0F90630C9B25B
:10C7A00007291C44F5D812F00702A5D0034B9B5C67
:10C7B000CFE73444AFE700BF344C0100244C010004
:10C7C00070B4047EBDF80C50022C18D0032C1FD07E
:10C7D000012C0BD0002A03DBB0F90840944201DCA5
:10C7E00070BC7047039570BCFFF7BCBAC488039552
:10C7F000013CA41A0A4621B270BCFFF749BF068962
:10C80000C488013E641AB21AE41A12B221B2E1E7F6
:10C8100004890395E41A641A114622B270BCFFF72A
:10C8200037BF00BF70B4057EBDF80C60022D1AD072
:10C83000032D12D0012D03D0039670BCFFF728BF43
:10C84000C488E41AA41A0A4621B2002A03DBB0F90C
:10C850000840944213DC70BC70470489013C641AA0
:10C86000114622B2F1E7C48805890396013CAD1A4E
:10C87000ED1A621A11B22AB270BCFFF709BF039613
:10C8800070BCFFF76FBA00BF2DE9F8430446406A59
:10C89000002863D0616DFEF74DF9052274492046EA
:10C8A000FFF718FCA1790139C9B22046FFF74AFB0E
:10C8B000B4F90820E588A66AD31D48BF02F10E032B
:10C8C000DB10626A15FB03F51FFA85F8002A7BD09E
:10C8D00094F82C300125AB4082F83B3082F85E5052
:10C8E00082F85D50606A036840211B6808F1FF37D9
:10C8F0009847BFB2B8F1000F23D03744A846013E95
:10C90000606A16F8011F03681B6898470135B74233
:10C91000ADB216D01F2DF3D90121606AFEF76CFA73
:10C9200094F82C20636A520083F83B2083F85E80E1
:10C9300083F85D80606A036840211B689847012581
:10C94000DEE70121606AFEF757FA606A002800F00E
:10C950008D80A16DBDE8F843FEF7ECB8236A002B8B
:10C960002BD0D97A226EE1B172B6D97ACE0706D52C
:10C970004048D9680568294099610160D97A8D07D6
:10C9800006D53D48196905682940D9610160D97A01
:10C99000480705D539485969056829401962016079
:10C9A00062B61B68D968914207D03548186035498E
:10C9B000DA6042F0804018611960226C216D1368C2
:10C9C00023EA0103136068E7E26BE36C1168276AEE
:10C9D0000B4306EB080913604FF0004E4E450DD097
:10C9E00016F801CB2FB33A68C2F82CE0C2F834C075
:10C9F000D36A002BFCDA4E45936BF1D1226C236D88
:10CA000011680B43136097B1FB7A83B1D90703D543
:10CA10001D4BBA691A60FB7A9A0703D51B4BFA695A
:10CA20001A60FB7A5B0702D5194B3A6A1A60BDE8B7
:10CA3000F883A36BD4F8348008208021D8F8002034
:10CA4000656C1CEA010F14BF2A43AA43C8F80020F2
:10CA50001A68A56C2A431A601A68A56C013822EA84
:10CA600005024FEA51011A60E8D1B7E7276AC5E726
:10CA70002C4C010080E100E084E100E088E100E06E
:10CA800001403F0000003F8000E100E004E100E0E1
:10CA900008E100E02DE9F04F85B09946BDF9387006
:10CAA000BDF83CA0BB1AC1EB090B002BB8BF5B4221
:10CAB000BBF1000FB8BFCBF1000B5B450D4616462E
:10CAC0000093804648DC4D453A4633464CDC1946D7
:10CAD00013460A46C5EB09019B1A89B2002B0CB21A
:10CAE000B8BF5B4204EBD474BE42ACBF4FF0FF3220
:10CAF00001224D45039102924FEA640429DC9BB266
:10CB000001930DE0D8F80070BF69B847019BE41AA3
:10CB1000A3B21CB20135002C2DB211DBA94518DBE4
:10CB2000009B5B452A46534631464046EADCD8F82E
:10CB3000002053469769294632464046B847E5E704
:10CB4000029A1644039AA94502EB030436B224B2B2
:10CB5000E6DA05B0BDE8F08F4A462B46B9463546C1
:10CB60004D4517461E46B2DD304629463E464D46E7
:10CB700007468946AEE700BF10B404682469A4469E
:10CB800010BC604730B40468BDF808500295A46B2F
:10CB9000A44630BC604700BF30B40468BDF80850FC
:10CBA0000295E46BA44630BC604700BF70B40468D3
:10CBB000BDF90C60BDF8105003960495246CA44692
:10CBC00070BC6047704700BF10B582B0B0F90C2050
:10CBD00001910168009200220C6CB0F90A301146F4
:10CBE000A04702B010BD00BF704700BF01F00301B5
:10CBF0000129017606D0032904D0C2880389428125
:10CC0000838170470289C38842818381704700BF56
:10CC10002DE9F0410568134E6F6986B0B7420446AE
:10CC2000BDF8308010D1013B13441BB20093CDF806
:10CC300004800B46AD6A2046A8472368DB6AB342EE
:10CC40000AD106B0BDE8F081059304920391B8477C
:10CC500003A925680EC9E6E7204606B0BDE8F04105
:10CC6000184700BFC5CB00002DE9F0410568124E02
:10CC70006F6986B0B7420446BDF830800FD1013BE2
:10CC8000CDF804800B4400921BB2AD6A2046A84741
:10CC90002368DB6AB3420AD106B0BDE8F081059390
:10CCA00004920391B84703A925680EC9E7E7204617
:10CCB00006B0BDE8F0411847C5CB00002DE9F04FA4
:10CCC0000568DFF858B06F6985B05F450646BDF965
:10CCD0003890BDF83CA00C46904615D11F19BC42B7
:10CCE0000CDACDF800A0214601342D6A4B464246AD
:10CCF000304624B2A847BC423568F2DBEB6A5B459C
:10CD000007D105B0BDE8F08F0393B8473568039BA2
:10CD1000E4E7304605B0BDE8F04F1847C5CB00004A
:10CD20002DE9F04387B099420546BDF93840BDF87A
:10CD30003C6025D0A24212D00768DFF88080D7F887
:10CD40001490C14532D18DE850002846BC6AA047F6
:10CD50002B68DB6A434524D107B0BDE8F0839942D4
:10CD600002DD08461946034628680E96C46B013357
:10CD70005B1A1BB22846A44607B0BDE8F0436047E3
:10CD8000A24202DD134622461C4628680E96631C0A
:10CD9000846B9B1A1BB22846A44607B0BDE8F0433B
:10CDA0006047284607B0BDE8F04318470593049252
:10CDB0000391C84703A92F680EC9C4E7C5CB00007B
:10CDC0002DE9F04FD0F800E0DFF89090DEF814B0D5
:10CDD00083B0CB450446BDF93080BDF834A00D4684
:10CDE00017461E4631D1CDF800A0DEF824B0294602
:10CDF00033463A462046D8472368CDF800A008F1CC
:10CE0000FF323A44D3F824B0294612B233462046C2
:10CE1000D8472368CDF800A02946D3F820B03A4679
:10CE200043462046D8472068CDF800A0711E29440B
:10CE30004346056A09B23A462046A8472368DB6A9A
:10CE40004B4506D103B0BDE8F08FD847D4F800E0D9
:10CE5000C9E7204603B0BDE8F04F1847C5CB000036
:10CE6000F0B4002401254FF6FF76094F07600471E6
:10CE70000476C48104828476C461C575857545765F
:10CE800086824682C180028141818281F0BC7047E6
:10CE9000505101002DE9F04F85B00668BDF84450AF
:10CEA000BDF93880CDF8008004460195D6F848B029
:10CEB0000392BDF93C60BDF9407089469A46D84757
:10CEC00023680195009742465146D3F84880204692
:10CED0003346C0472068039B0E930F95856C4B46E5
:10CEE0003A4631462046AC4605B0BDE8F04F6047B3
:10CEF0002DE9F04F87B01746BDF940400091254617
:10CF0000E91D059344BF2B4603F10E010268BDF8ED
:10CF1000486053690294C91003912B49BDF94440FC
:10CF200001968B42824645D1002C3CDD029B3C445D
:10CF30005E1EB6B24FF0000923B2049301364D468F
:10CF4000029B002B28DD059B002403EB090806E06B
:10CF5000EDB22B0604F1010411D4A6421CD0A1B2FB
:10CF600011F0070F23B24FEA4505F1D1002BB8BFEE
:10CF70000733DB10013418F803502B06EDD5009B66
:10CF8000D2F818B019443A4609B2019B5046D84726
:10CF9000A642DAF80020E2D1039B01379944049BB2
:10CFA0003FB2BB42CCD1D36A074A934206D107B005
:10CFB000BDE8F08F9847DAF80020B5E7504607B093
:10CFC000BDE8F04F184700BFC5CB000070B4BDF9F5
:10CFD0000C60BDF91050BDF81440039604950594FB
:10CFE00070BCFFF785BF00BF2DE9F04F91B08346BD
:10CFF0000591C169BDF8680006909DF87400BDF800
:10D000006C709DF870A0039002929946002900F080
:10D01000CC800B7A48680A68C3EB0903DBB215467B
:10D0200000EBC30230F83360D3780993BAF1010FF3
:10D0300092F9053092F802800E9392F9064079D960
:10D04000BDF93830089323B20B93A94BDBF80020CD
:10D050000F93194653698B4240F0A280099B002B25
:10D0600053D0BDF808300C930021234407910D9351
:10D070000F460C46A946B8F1000F3FD0BDF81C1072
:10D080000B9BBDF80C000297CB1813FB00F30C9818
:10D0900003440D981BB2014404930BB20A9300257C
:10D0A00005E00135EBB264009845E4B223D9029B58
:10D0B0002B44590703D1731C19F806409EB223066E
:10D0C000EFD5089BE918059B11FB0AF1BAF1010F96
:10D0D000194402D1039B012B1ED0069B0193039B95
:10D0E0000093D369049A1F4609B253465846B8477D
:10D0F000DBF80020D5E7029F4744FFB2079B099960
:10D1000001330793DBB29942B5D8D36A0F9A9342A1
:10D1100041D111B0BDE8F08F0E9B05995918936964
:10D120000A9A29441F4609B2069B5846B847DBF8BD
:10D130000020B6E7039B012B82D800230B930893B2
:10D1400083E70799099A0131013A49B212F0FF02C7
:10D150000791099260D1069A4A454F4617D0BAF115
:10D16000010F03D1039A012A00F0B5800A9A0898AA
:10D1700002EB8201039AD2008DE88400084401B2D8
:10D18000DC69029A53465846A047DBF80030DB6A58
:10D190000F9A9342BDD0584611B0BDE8F04F1847E2
:10D1A00058469847DBF8002058E7BBF90A30059944
:10D1B0008B42AEDDBBF90C3002988342A9DD062319
:10D1C00013FB0A13002BA4DD039B00EBC303002B0E
:10D1D0009FDD9BF81A3033B9B9F1AF0F84BF09F165
:10D1E00001035FFA83F9424ADBF800300F921146DF
:10D1F0005A698A426AD1BDF8142008920522099220
:10D20000002207921FFA8AF20A92CDF830900FFAA4
:10D210008AF2B946039F05920799BDF83040089DF0
:10D220000522104610FB04120A98324C06460846A6
:10D2300001FB0651A65C15FA80F209B212B2049104
:10D240000B92082400251CE0BAF1010F01D1012F37
:10D2500024D0069A0192029A009705FB0722D3F880
:10D260001C800499059B12B25846C047DBF8003079
:10D27000013C013514F0FF046DB24FEA56063FF44D
:10D2800060AFF007E0D4069A4A45F1D0BAF1010F39
:10D2900001D1012F0ED0CDF80490DCE7029AD3F82B
:10D2A00018800B99069BAA1812B25846C047DBF8A3
:10D2B0000030DDE7029AD3F818800B99AA184B4684
:10D2C00012B25846C047DBF80030D1E758469047C5
:10D2D000DBF800308FE70899CDF8009005311C6A23
:10D2E000029A082309B25846A047DBF800304EE7FF
:10D2F000C5CB0000A0510100F0B5C36985B004465C
:10D300003BB30A296FD00D294FD01A7A91424CD3E2
:10D31000987A884249D38A1A5D68D2B205EBC20571
:10D32000AA78002A56D0E878002853D0607E0028DA
:10D330003ED095F905E0B4F90E00A67DB4F90A7067
:10D34000724406FB0202BA4269DCE77DB4F91020A0
:10D3500034E00A295CD00D2927D0427E002A50D023
:10D36000B0F90E00A57DB4F90A60062212FB050291
:10D37000B242E67D42DD228AE38102EBC60212B2AE
:10D3800018462282B4F814E0678A03960B46029589
:10D3900001468DE880402046FFF726FEA37DE28906
:10D3A00003EB430302EB4303E381012005B0F0BD2F
:10D3B000A67DE77DB4F90E00B4F91020B4F814E0AE
:10D3C0000397678A02960B468DE880400146204607
:10D3D000FFF70AFE2979E389A27D012001FB0233D0
:10D3E000E38105B0F0BD0022C2811A7BC17D038AB2
:10D3F00001FB02330382012005B0F0BDB4F9102017
:10D40000C0E7857DC67DB4F91020B0F90E00B9E7FC
:10D41000028AC17DC38102EBC1030382C5E70020FC
:10D42000E0811B7B228AE77D03FB072212B2228266
:10D43000C4E700BF11B18175C175704701218175C5
:10D44000C1757047844641EA000313F003036DD1B0
:10D45000403A41D351F8043B40F8043B51F8043BB7
:10D4600040F8043B51F8043B40F8043B51F8043BBE
:10D4700040F8043B51F8043B40F8043B51F8043BAE
:10D4800040F8043B51F8043B40F8043B51F8043B9E
:10D4900040F8043B51F8043B40F8043B51F8043B8E
:10D4A00040F8043B51F8043B40F8043B51F8043B7E
:10D4B00040F8043B51F8043B40F8043B51F8043B6E
:10D4C00040F8043B51F8043B40F8043B51F8043B5E
:10D4D00040F8043B403ABDD2303211D351F8043BFE
:10D4E00040F8043B51F8043B40F8043B51F8043B3E
:10D4F00040F8043B51F8043B40F8043B103AEDD2AD
:10D500000C3205D351F8043B40F8043B043AF9D2FD
:10D51000043208D0D2071CBF11F8013B00F8013BD0
:10D5200001D30B8803806046704700BF082A13D3DD
:10D530008B078DD010F003038AD0C3F10403D21AF5
:10D54000DB071CBF11F8013B00F8013B80D331F829
:10D55000023B20F8023B7BE7043AD9D3013A11F8A9
:10D56000013B00F8013BF9D20B7803704B78437014
:10D570008B78837060467047374A384913681B06BA
:10D58000FCD40B6813F08003F8D172B634490A78E2
:10D59000002A5FD0334A3448F0B4344C1768066828
:10D5A0002568D4680C303E44143200681268304F4D
:10D5B00035442C4420440244C2F34E022D4E2E48E2
:10D5C0002E4D2F4C42F400423A60376806682D68B1
:10D5D0002C4A24680C303E44006812682A4F3544B7
:10D5E0002C4420440244C2F34E02284E2848294DC0
:10D5F000294C42F400423A60376806682D68274A91
:10D6000024680C303E4400681268254F35442C4491
:10D6100020440244C2F34E02224E2348234D244CA0
:10D6200042F400423A60376806682D68214A24684F
:10D630000C303E440068126835442C4420440244B7
:10D64000C2F34E021C4842F4004202600B7062B604
:10D65000F0BC704762B6704724B0034024B00B4062
:10D66000AE9FFF1F38B003403CB0034040B00340C2
:10D670002CB0034058B003405CB0034060B003409E
:10D6800064B003406CB0034030B0034038B00B408E
:10D690003CB00B4040B00B4044B00B404CB00B4092
:10D6A0002CB00B4058B00B405CB00B4060B00B404E
:10D6B00064B00B406CB00B4030B00B4030B4294824
:10D6C000294A2A4B2A4D6024E121047011701B78ED
:10D6D000284C082B30D00A2B2748284937D00C2B50
:10D6E0000CBF35223D2212232A60236002600B60AA
:10D6F000234B24491B78244ABBB101230B601360E0
:10D70000224B23491B78234A012B26D9042B0FD9FE
:10D71000082B1ED9102B94BF862387230B60136020
:10D720001D4B01221A7030BC70470B601360E7E795
:10D7300084230B601360F3E700F58E200F49083057
:10D74000012213232A60236002600B60D0E7392294
:10D75000F7E785230B601360E2E780230B6013601B
:10D76000DEE700BF0040074001400740B891FF1FBF
:10D7700008B003400CB0034008B00B400CB00B40A5
:10D78000B19FFF1F20B0034020B00B40B991FF1F95
:10D7900024B0034024B00B40AE9FFF1F0C2830B4D0
:10D7A00017D91023984228BF18461C46104A114D1D
:10D7B0001178181A8C42287018D00F4913700B7802
:10D7C00023B10E490E4A00230B60136030BCFFF7F3
:10D7D00075BF0A2802D90C231C46E7E7082802D99E
:10D7E0000A231C46E2E708231C46DFE730BC7047EB
:10D7F000B891FF1FAD9FFF1FAE9FFF1F24B00340D6
:10D8000024B00B4028282FD8334B2DE9F0411E5C63
:10D81000FF2E2BD0314B1B78002B2AD132062CD473
:10D8200072B62F4D2F4C2F46012326602B7062B607
:10D8300072B623681B060CD43B781BB9F4E72B782F
:10D84000002BF1D062B603F0A1F872B62368180677
:10D85000F5D5254B1B6800222A7062B6234A107842
:10D8600043FA00F0BDE8F081002070470020BDE8D9
:10D87000F081FFF781FE3206D2D572B61C4DDFF87B
:10D880007C801C4C06F04007FFB206F03F06D8F83B
:10D890000030DFB123F01003C8F800300123266008
:10D8A000134A2B7062B672B6236819060CD413782B
:10D8B0001BB9ECE72B78002BE9D062B603F066F8D1
:10D8C00072B623681B06F5D50B4BC3E743F0100374
:10D8D000C8F80030E2E700BFA0560100AE9FFF1F6E
:10D8E000B09FFF1F00B0034010B00340AD9FFF1F6B
:10D8F000AF9FFF1F00B00B4010B00B400CB00B40AF
:10D900000A4A0B49136843F4805313600B7843B9F8
:10D91000084BC0221A70084B80F30C0000B218802C
:10D920007047044B80221A70F5E700BF2C8004403A
:10D93000B19FFF1F21C00C4000C00C40F0B51B4B35
:10D940001B4E596818689A68DB6885B06C460FC42E
:10D95000337899071DD5174A174C1378174913F0D8
:10D96000700318BF1370164A164B802717700026D5
:10D970003320032226706D4608701A7072B6043C7C
:10D9800045F001052046A84762B6237813F07003DE
:10D9900009D10D4B064901E0013B02D00A78D207BC
:10D9A000FAD505B0F0BD237005B0F0BDCC5601002E
:10D9B0000100024000000240040002400B0002404F
:10D9C000070002400A000240410D0300B0F5006F5D
:10D9D0000AD210B5094B1B78DB07044606D504F1C3
:10D9E000A0500078C0B210BD00207047FFF7A6FF1E
:10D9F00004F1A0500078C0B210BD00BF0100024089
:10DA0000B0F5006F17D238B50F4B1B78DA070D460B
:10DA1000044611D504F1A0500378AB420AD00B4A5A
:10DA2000137813F0700318BF1370074A057013784A
:10DA3000DB07FCD538BD7047FFF780FF04F1A0502D
:10DA40000378AB42EBD1F5E7010002400000024051
:10DA500008B5104C08E0236859050DD423681A0551
:10DA60000FD42368DB0411D423685803F3D501F0E5
:10DA700087FB23685905F1D500F00EF823681A05D5
:10DA8000EFD500F02DFF2368DB04EDD501F0EAF9B6
:10DA9000EAE700BF3480044008B5FFF7D9FF00BFB4
:10DAA000014B10221A80704700200540704700BFCC
:10DAB000094908B50B6830B16A461844A2F580528E
:10DAC000904202D20860184608BD04F03FFA0C23C9
:10DAD00003604FF0FF3008BDBC91FF1FFEE700BFA1
:10DAE000EFF3138070B9EFF310836BB9EFF3058296
:10DAF0005AB94FF48070EFF311832BB1984228BFCD
:10DB0000184670474FF0FF3070470F2A01D818466B
:10DB1000F1E7014BD05CEEE7F0E300E0704700BFB7
:10DB200010B40F4B53F8302092F880422CB10123EF
:10DB300069B182F8803010BC704703EBC0035B68AA
:10DB40001A6841B922F002021A6010BC704782F8CC
:10DB5000003110BC704742F003021A6010BC7047DD
:10DB6000DC5601001C4A02EBC00301295B6811D09E
:10DB700004291BD052F83000002280F8802229B1FD
:10DB8000022920D0032922D01A6070474FF48072F6
:10DB90001A60704752F830004FF4A27280F8801279
:10DBA0001A601A6822F020021A60704752F830108A
:10DBB0004FF4A272012081F880021A601A6842F0C4
:10DBC00020021A60704740F203121A6070474FF447
:10DBD00081721A60704700BFDC560100212848D8C6
:10DBE000F8B5042A44D8DFE802F0484B4E0345005C
:10DBF0004FF410262B4B03EBC0030D465C682168E5
:10DC000011F4E06148D0284B284A2949C3F89C21E7
:10DC100004F140422748C3F8A411A2F59221264FEF
:10DC2000C3F8A0017C292548C3F8A871C3F8AC014A
:10DC30002CD9A2F594237C2B2AD9A2F596237C2BF0
:10DC400028D9A2F598237C2B29D9A2F59A227C2ADF
:10DC500027D81B4872B6236823F4702343F08072E0
:10DC6000C4F384011643236040F82150266062B655
:10DC7000F8BD70474FF43026BCE74FF40026B9E7F3
:10DC80004FF44026B6E74FF42026B3E70D48E1E70E
:10DC90000D48DFE70D48DDE7FFF764FFB3E70C4809
:10DCA000D8E7F8BDDC5601000082FF1FF188FF1F96
:10DCB0009988FF1FC588FF1F6D88FF1F4188FF1FC0
:10DCC0009892FF1FC091FF1FF891FF1F4892FF1FFE
:10DCD0007892FF1F1A4B03EBC00010B4426802F1A8
:10DCE0004043A3F592217C2923D9A3F594217C29D3
:10DCF0000DD9A3F596217C291FD9A3F598217C295C
:10DD000019D9A3F59A237C2B11D80E4C00E00E4CA8
:10DD100072B613680D4823F08773C2F3840123F4AD
:10DD2000803343F08073136044F8210062B610BC66
:10DD30007047074CECE7074CEAE7074CE8E700BF01
:10DD4000DC5601009892FF1FF891FF1F1DDB0000B9
:10DD5000C091FF1F7892FF1F4892FF1F30B4054B00
:10DD6000054D064C002210211A602A6020601960BF
:10DD700030BC704714D0034004D0034000D00340AF
:10DD8000282838B52ED0002904464FDD5F4B1B787C
:10DD9000012505FA03F28A4202D8212837D938BD75
:10DDA0000338C2B2012A3AD9202C4AD0192C48D0C3
:10DDB000574A126802FB011222FA03F31D2800F2EF
:10DDC0009B80DFE800F0928B847D9999766F99991A
:10DDD0009999999999999968615A53994C999999EE
:10DDE00099999945494B1B780B2B08D90C2B1CBFD3
:10DDF0000C3B19410846BDE83840FFF781BDC3F12F
:10DE00000C0399400846BDE83840FFF779BD294624
:10DE1000FFF786FE2946BDE83840FFF7A3BE3D4A1E
:10DE2000126802FB011222FA03F3C7E72128B6D8D1
:10DE30000021FFF775FE20460121BDE83840FFF7BD
:10DE400091BE354A126802FB011222FA03F3B5E7CC
:10DE50003249334A0B604FF45173136038BD314976
:10DE6000314A0B604FF45173136038BD2F49304A6B
:10DE70000B6040F24443136038BD2E492E4A0B60BC
:10DE800040F24443136038BD2C492D4A0B6040F2E8
:10DE90004443136038BD2B492B4A0B6040F2444386
:10DEA000136038BD29492A4A0B6040F2444313608D
:10DEB00038BD2849284A0B6040F24443136038BDFE
:10DEC0002649274A0B6040F24443136038BD254978
:10DED000254A0B6040F24443136038BD2349244A6D
:10DEE0000B604FF45173136038BD2249224A0B6016
:10DEF0004FF45173136038BD212C3FF650AF7F298A
:10DF0000D4BF00210121204693E700BFA092FF1F4C
:10DF1000088003400890034008800B4010800B40AD
:10DF200048A0044018800B404CA0044018800340D7
:10DF300008B004401080034004B004404080034017
:10DF400018C004403880034014C0044028800340B7
:10DF500010B00440208003400CB0044030800340E7
:10DF600010C00440488003401CC004401890034087
:10DF700034900440109003403090044038B1102891
:10DF800028BF1020044AC3B2107813707047024AA9
:10DF90000123107813707047A092FF1F2DE9F843FA
:10DFA0000E4680463249334D304603F05BFF47F65C
:10DFB000122300281ABF1D464FF002094FF0010935
:10DFC000002425FA04F003F057FD4FF05E51074698
:10DFD00003F0AAFD0146304603F058FF30B9013482
:10DFE000072CEED1E80903F047FD074631463846D5
:10DFF00003F04EFE4FF07C5103F08CFC03F080FFE9
:10E000004FF6FF729042A8F1030328BF1046012B80
:10E0100029D9B8F1170F17D8174B23FA08F303F0D3
:10E02000010383F0010223B9B8F1190F0FD0BDE845
:10E03000F883124B124D13491A6044EAC9042A604E
:10E0400008601C60BDE8F883B8F1200FECD10E4BDE
:10E050000E4D0F49002244EAC9041A602A60086084
:10E060001C60BDE8F8830B4B0B4D0C49F2E700BF79
:10E07000001BB740006CDC026006F000008003402B
:10E08000048003400880034000800B4004800B4064
:10E0900008800B4000900340049003400890034028
:10E0A000212801D8FFF73CBD704700BF212806D8C2
:10E0B000044B53F8303093F80002C0B27047002090
:10E0C000704700BFDC560100212801D8FFF74ABD88
:10E0D000704700BF72B60C490C4B0D4A1B680868AC
:10E0E000126862B6520102D5322B88BF013009494D
:10E0F000C3F5BB334FF47A72FF33A1FB031302FB6A
:10E1000000F000EB93107047B49FFF1F18E000E091
:10E1100004ED00E0ABAAAAAA2DE9F843054672B6C1
:10E12000204F214B214A1B683C68126862B652019D
:10E1300002D5322B88BF013495B3C3F5BB331C4ED7
:10E14000DFF86490DFF86480FF334FF47A72A6FB47
:10E15000031302FB04F404EB931472B6D9F8001015
:10E160003A68D8F800E062B6C1F5BB33FF33A6FBCE
:10E1700003031EF0806FC4EB93134FF47A7002D048
:10E18000322988BF013200FB0233B3F57A7F04D312
:10E19000013D05D004F57A74DFE702F0F7FBDCE718
:10E1A000BDE8F883B49FFF1F18E000E004ED00E035
:10E1B000ABAAAAAAF8B52D4B2D49DFF8D0E0DFF8BD
:10E1C000D0C02C4E2C4D2D4C2D4A2E4F4FF400001C
:10E1D00018604FF0807018604FF0007018604FF0BA
:10E1E000806018604FF000601860002008602823ED
:10E1F0004BF6FF71CCF80010CEF80030336013609E
:10E200002B6023603B60B3629362092245F8242CA3
:10E21000C4F8D80F05F57F65C7F8D41F07F5FF27A9
:10E2200007F5FA67C6F8F83F2B6006F5FF26C4F835
:10E23000D42F05F5FD2504F5FF24386006F2F476A9
:10E240001148316005F5FF6504F5FD642B6023601E
:10E250000260FFF733FA1920FFF75EFF01F0F6FCCA
:10E2600040F21310BDE8F840FFF756BF08E100E0A8
:10E270000480034014800340248003402C8003402A
:10E280001C8003403480034000800B400C8003401E
:10E29000088003402B4A2C491368F0B543F400630F
:10E2A00013600A78294F2A4E2A4D2B4C2B49002304
:10E2B000092A3B7033702B7023700B703DD01A2AE3
:10E2C00021D0274B1B780A2B25D01F2B30D01F289D
:10E2D00027D8002002460125224B234C1A702349DF
:10E2E0005D7004224FF0020E88273C26402598726C
:10E2F0009A704FF4004083F813E05A751F74DE7073
:10E3000025700860F0BD1A4B40F213321A60144BAE
:10E310001B780A2BD9D1174B4FF451721F281A6062
:10E32000D7D9C0F34432C0F3471500F01F00D3E73C
:10E33000114B4FF451721A60C9E7104B40F213327F
:10E340001A60BEE734800440A192FF1F28A0FF1F7F
:10E35000BD9FFF1F30A0FF1F29A0FF1FBC9FFF1FF5
:10E36000A292FF1F00B006402FE400E004E100E0AD
:10E3700004D0044010B0044000D004400CB004406D
:10E38000144B14499B7803F0EC0200F00303134391
:10E39000420700F00F0248BF43F01003042A8B70BD
:10E3A00013D00C4B0B4A5B79C10603F0EF0348BF57
:10E3B00043F0100353719379820603F0EF03054A8B
:10E3C00048BF43F01003937170478B7943F04003CB
:10E3D0008B71E6E700B00640234B1B681B0542D556
:10E3E00010B5224C237823B102F0D0FA2378002B09
:10E3F000FAD11F481F4A204B4FF40044002104600B
:10E40000D1701B78092B1FD01A2B03D11B4B40F264
:10E4100003121A601A4B1B7803F07F030A2B1DD0DE
:10E420001F2B03D1174B40F203121A60164A114BEF
:10E430001648174912681C79DB79002303700B70AA
:10E440000AB10123137010BD124B40F203121A607F
:10E450000B4B1B7803F07F030A2BE1D10E4B40F2EC
:10E4600003121A60E2E7704734800440BC9FFF1F2C
:10E4700084E100E000B00640A192FF1F04D00440F8
:10E48000A292FF1F00D00440B89FFF1F28A0FF1FCB
:10E49000BD9FFF1F0CB0044010B004400A4A38B5BD
:10E4A0000546137803F0FF04002BFAD1012128461A
:10E4B000FFF70AFE21462846FFF7F2FD034A044B08
:10E4C00052F835201A6038BDBC9FFF1FDC56010092
:10E4D0002CA0FF1F09B140F08000174A1378984222
:10E4E00016D010B4154C246824050FD503F07F0313
:10E4F0000A2B1CD01F2B11D0002900F07F0114BF64
:10E50000602344230A290DD01F2902D0107010BCAB
:10E5100070470B4943F440730B60F7E7084B002446
:10E520001C60E9E7074943F440730B60EEE7054BD5
:10E5300000241C60E0E700BFA292FF1F348004406B
:10E5400000D0044010B00440124B1A7882420CD024
:10E5500011490968090507D5092A16D01A2A0AD0CF
:10E5600009280DD01A2801D0187070470B4A40F2C4
:10E5700013311160F8E7094A002109281160F1D12F
:10E58000074A40F213311160EEE7054A002111609D
:10E59000E6E700BFA192FF1F3480044004D004408E
:10E5A0000CB004400D4B1B6813F4006305D0212808
:10E5B00005D90B4B00201860704718467047094B6F
:10E5C00010B5074C53F8303023600121FFF77CFD74
:10E5D000236800221A70012010BD00BF348004405F
:10E5E000B89FFF1FDC5601000C4B1B6813F400633F
:10E5F00006D0172806D00A4A537B03F0FE03537354
:10E6000000207047074B064A40F202311960537BE5
:10E6100043F0010353730120704700BF348004406E
:10E6200000B0064008B004402DE9F84F234B1B68AA
:10E630001A053BD5224B1B680BB101221A70DFF87B
:10E640009090204D99F80040DFF888801E4E0134EC
:10E65000272C8ABF4FF0000A5FFA84FA5446074617
:10E66000AB462B789C4216D1FFF73AFA40281FDCC4
:10E6700033791B06F5D59BF800300133272B86BF75
:10E6800000221346DAB218F80330DBB2F3712A70B5
:10E690002B789C42E8D00D490B4BFFB20120BC22E5
:10E6A00008F80470087089F800A0DA70BDE8F88FE7
:10E6B000FF28D6DD02F06AF9D3E700BF34800440BA
:10E6C0002CA0FF1F29A0FF1F00B00640BC9FFF1F0A
:10E6D00030A0FF1FC09FFF1F2DE9F84F294B1B687B
:10E6E0001A0548D5284B1B6805460BB101221A7044
:10E6F00005EB010A554540D2DFF89C80234CDFF83A
:10E700009C90234F0AE015F8012B09F80B20214AB1
:10E710000123AA45137088F800602ED098F80030C5
:10E72000227803F1010BBBF1270F86BF0026B34609
:10E730005FFA8BF69345E6D1BC22FA7005E03A7990
:10E7400013060BD422789345DDD1FFF7C9F9402891
:10E75000F5DDFF28F6DD02F019F9F3E72278013242
:10E76000272A86BF00210A46D1B219F80220D2B268
:10E77000FA712170E6E7BDE8F88F054BBC22DA702C
:10E78000BDE8F88F348004402CA0FF1F29A0FF1F94
:10E7900000B00640BC9FFF1F30A0FF1FC09FFF1F9F
:10E7A00010B5044C237823B102F0F0F82378002B45
:10E7B000FAD110BDBC9FFF1F064A074B1B7810788B
:10E7C000DBB2C0B283422CBF273000F1FF30C01A49
:10E7D000704700BF29A0FF1F30A0FF1F054A064B4E
:10E7E00010781B78C0B2DBB2984238BF4030C01AF4
:10E7F000704700BF28A0FF1FBD9FFF1F30B4154BFF
:10E80000154C1A782378D2B2DBB29A421ED001336B
:10E810003F2B0ED91149124B087819680023C0B25A
:10E82000237021B1D31A1A2B01DC00230B7030BCEA
:10E8300070470A480A49C05C0968DDB2C0B2257059
:10E840000029F4D09A4238BF4032EBE74FF0FF3056
:10E85000EDE700BF28A0FF1FBD9FFF1FE89FFF1F20
:10E86000B89FFF1F084A094B12781B78DBB29A4207
:10E8700007D00133402B28BF0023054AD05CC0B22B
:10E8800070474FF0FF30704728A0FF1FBD9FFF1F4C
:10E89000E89FFF1F0D4B1B681B0516D530B40C4BB2
:10E8A0000C4CDA780C480D4902F0CB024025DA70A6
:10E8B0005D74DA7842F03402DA7023780268DBB2F1
:10E8C0000B700AB10023137030BC704734800440D1
:10E8D00000B00640BD9FFF1FB89FFF1F28A0FF1F6D
:10E8E000F0B4384B1A7912F0300F2CD072B6997DF3
:10E8F00001F0FF0200293DD062B6334F334938782A
:10E900000D78334E1C46C0B2EDB2431C402BE1796A
:10E9100028BF0023AB4202F1FF32C9B21CBFF15441
:10E92000184612F0FF02F0D12A4B1B68C2B23A70AF
:10E930004BB1A84236BFC5F14005401B40192728FE
:10E94000C4BF01221A701F49CA78D2B2150616D464
:10E9500052060DD51B4B1B795B0609D51E4B1F4973
:10E960001B6800220A7003B11A70164B3C22DA7041
:10E97000F0BC70474022D9795A7462B6E3E70B794C
:10E980001C06E5D5164B174E1C783378E4B2DBB283
:10E990009C420ED0144D01E0A3420AD00133282B33
:10E9A00028BF00230879E85CC0B2C871087D072839
:10E9B000F2D9DBB2034933700B79180644BF7C23CC
:10E9C000CB70C5E700B0064028A0FF1FBD9FFF1F0A
:10E9D000E89FFF1FB89FFF1F2CA0FF1FBC9FFF1FBA
:10E9E00030A0FF1F29A0FF1FC09FFF1F2DE9F84F78
:10E9F000214B1B6807460BB101221A70DFF8889083
:10EA00001E4D99F80040DFF884801D4E0134272CFC
:10EA10008ABF4FF0000A5FFA84FA5446AB462B785F
:10EA2000A34216D1FFF75CF840281FDC33791B06A0
:10EA3000F5D59BF800300133272B86BF0022134603
:10EA4000DAB218F80330DBB2F3712A702B78A342E4
:10EA5000E8D00C490A4BFFB208F804700120AC2240
:10EA6000087089F800A0DA70BDE8F88FFF28D6DDBD
:10EA700001F08CFFD3E700BFA8A0FF1FA5A0FF1FD8
:10EA800000C00640A4A0FF1FACA0FF1F3CA0FF1FBA
:10EA90001C4BDFF894C01A681B49F0B542F4805251
:10EAA0001A4D1A60DFF884E0194F1A4E1A4C0023F1
:10EAB0008CF800304FF451722B701F2840F2133540
:10EAC0008EF800303B70337025600A6012D819460A
:10EAD0000124124A124D11701248547000212C2743
:10EAE000402693724FF4003491701174D7702E70D9
:10EAF0000460F0BDC0F34431C0F3471400F01F03BD
:10EB0000E7E700BF348004400CC0044039A0FF1F79
:10EB1000A5A0FF1FA4A0FF1F08C0044000C006401E
:10EB200031E400E004E100E038A0FF1FACA0FF1FCB
:10EB3000144B14499B7803F0EC0200F003031343D9
:10EB4000420700F00F0248BF43F01003042A8B7005
:10EB500013D00C4B0B4A5B79C10603F0EF0348BF9F
:10EB600043F0100353719379820603F0EF03054AD3
:10EB700048BF43F01003937170478B7943F0400313
:10EB80008B71E6E700C00640F8B5134B1B68DB0449
:10EB90001FD5124C237823B101F0F8FE2378002B07
:10EBA000FAD10F4B0F4A104D104F114E114C124815
:10EBB0004FF4003119600023D37040F20311396023
:10EBC000316029681579D2792370037011B101235E
:10EBD0000B70F8BDF8BD00BF34800440A4A0FF1F37
:10EBE00084E100E000C0064034A0FF1F08C00440DC
:10EBF0000CC0044038A0FF1F39A0FF1F0A4A38B5D7
:10EC00000546137803F0FF04002BFAD101212846B2
:10EC1000FFF75AFA21462846FFF742FA034A044B07
:10EC200052F835201A6038BDA4A0FF1FDC56010041
:10EC3000A8A0FF1F09B140F080000F4A1378984246
:10EC400019D010B40D4C2468E40412D503F07F03EE
:10EC5000082B02D10A4B00241C60002900F07F031E
:10EC600014BF60214421082B03D1054B41F44071AE
:10EC70001960107010BC7047A392FF1F34800440CD
:10EC80000CC00440704700BF0D4B1B6813F4805349
:10EC900005D0212805D90B4B002018607047184675
:10ECA0007047094B10B5074C53F8303023600121F1
:10ECB000FFF70AFA236800221A70012010BD00BF76
:10ECC0003480044034A0FF1FDC5601000C4B1B684D
:10ECD00013F4805306D00E2806D00A4A537B03F063
:10ECE000FE03537300207047074B064A40F202317F
:10ECF0001960537B43F0010353730120704700BF39
:10ED00003480044000C0064004C00440034B1B682C
:10ED1000DB0401D5FFF76ABE704700BF34800440B2
:10ED200070B5094E04464518AC4204F101040AD0FE
:10ED30003368DB04F8D514F8010CFFF757FEAC423A
:10ED400004F10104F4D170BD3480044010B5044CCA
:10ED5000237823B101F01AFE2378002BFAD110BDDD
:10ED6000A4A0FF1F064A074B1B781078DBB2C0B285
:10ED700083422CBF273000F1FF30C01A704700BF1C
:10ED8000A5A0FF1FACA0FF1F054A064B10781B78FB
:10ED9000C0B2DBB2984238BF4030C01A704700BFE3
:10EDA00038A0FF1F39A0FF1F30B4154B154C1A783F
:10EDB0002378D2B2DBB29A421ED001333F2B0ED958
:10EDC0001149124B087819680023C0B2237021B191
:10EDD000D31A1A2B01DC00230B7030BC70470A4891
:10EDE0000A49C05C0968DDB2C0B225700029F4D0C0
:10EDF0009A4238BF4032EBE74FF0FF30EDE700BFFB
:10EE000038A0FF1F39A0FF1F64A0FF1F34A0FF1F01
:10EE1000084A094B12781B78DBB29A4207D00133BB
:10EE2000402B28BF0023054AD05CC0B270474FF08A
:10EE3000FF30704738A0FF1F39A0FF1F64A0FF1FDD
:10EE4000054B064A1B7806491268DBB20B700AB103
:10EE500000231370704700BF39A0FF1F34A0FF1FAD
:10EE600038A0FF1F30B42B4B1A7994061FD52A48BF
:10EE7000DA790378294901333F2B0978C8BF002389
:10EE80008B42D2B203D0264CD9B2E2540170254A4B
:10EE9000116861B1244A1278D2B2934236BFC2F1EE
:10EEA00040029B1A9B18272BC4BF01230B70194AE1
:10EEB000D378DBB2180611D45A060DD5154B1B7941
:10EEC0005B0609D5194B1A491B6800220A7003B169
:10EED0001A70104B2C22DA7030BC70471179090679
:10EEE000EAD5144910480C780178C9B28C420DD08B
:10EEF0004A1C272A84BF00210A460F4D054C98BFA3
:10EF0000D1B2AA5CD2B2E2710170D5E76C21D170A6
:10EF1000D2E700BF00C0064038A0FF1F39A0FF1F86
:10EF200064A0FF1F34A0FF1FA5A0FF1FA8A0FF1F04
:10EF3000A4A0FF1FACA0FF1F3CA0FF1F21282FD8BB
:10EF4000184B195CFF292BD0174B184ADFF870C0FB
:10EF500003EBC000F0B54368DFF868E0144F154DCF
:10EF6000154E00241C60DEF80030012043F0200321
:10EF70008840CEF8003014604FF4A07338602E60E3
:10EF8000C2F800C0013BFDD113689B05FCD42023CF
:10EF9000013BFDD1094B09B233F8110080B2F0BD3D
:10EFA00000207047EC570100DC560100005004407F
:10EFB0000850044004500440000002030051044083
:10EFC00080014A0038800440431E032B14D872B6D7
:10EFD0000A4951F8230068B170B4094C058834F827
:10EFE0001320466841F82360521B24F8132062B6B0
:10EFF00070BC704762B670470020704708A1FF1FC1
:10F0000060A2FF1F013803280BD872B6074B53F8D4
:10F01000203043B100205B680130002BFBD162B689
:10F020007047002070471846F9E700BF5CA1FF1F3A
:10F0300030B472B62B4A13781D0706D52A4B196ACD
:10F04000002936D0996A002941D053781C0706D58B
:10F05000254B196C00293ED0996C002939D0937842
:10F06000190705D5204B196E002936D0996E89B144
:10F07000D3781B0707D51C4BD3F880207AB3D3F87D
:10F08000882011213AB162B6184B00221A7030BCA8
:10F0900000F058BE0D21154C154D227843F8315023
:10F0A00003EBC1030830013A5860227062B630BCED
:10F0B000704704220D4C0F4D217843F8325003EB7A
:10F0C000C20308304A1E5860227062B6EFE705217D
:10F0D000E1E70921DFE70822ECE70C22EAE710224A
:10F0E000E8E700BFD45801000080FF1F85A1FF1F83
:10F0F000C800400088004000431E032B1DD81B4A57
:10F10000400140F0100030B4104472B6184CE25C7C
:10F11000032A1BD8DFE802F00212151703220D881C
:10F12000E25410F0080F14BFC823882343EA0543B4
:10F1300008310360416062B630BC7047083002227B
:10F14000EDE70522EBE708300422E8E7094A52F828
:10F15000230038B1084A52F82300416042F82310D6
:10F1600062B6E9E742F82310034AF7E70080FF1F81
:10F1700094A1FF1F5CA1FF1F6CA1FF1F00BE00BF79
:10F180002DE9F04FDFF820B3DFF820A387B044E08B
:10F19000AF4F4FEA930807EBC809013ED9F80420A6
:10F1A00003F00803F6B2A2F1080003F0FF04002BFD
:10F1B00040F00B8157F838301B0C99B222F8081C2C
:10F1C000002B00F0F980A34B22F8064C42F8044CC7
:10F1D00053F82620002A00F075819F4D55F82630FF
:10F1E00058609E4C45F8260034F81630194424F82F
:10F1F000161000F087FD002800F05D81984A994BB9
:10F2000019F0080F00F1080018BF1346C9F80400F0
:10F2100047F8383008238BF800309BF80040E4B200
:10F2200065071DD5904B1B78BBB190490A7802F059
:10F23000FF032AB1013BDBB20B70002B00F001850C
:10F240008B490A7802F0FF032AB1013BDBB20B7055
:10F25000002B00F02D8100F073FE04238BF80030AA
:10F2600004F0080303F0FF02002B00F0DA809AF8A4
:10F270000030DBB21E098BD19A08DFF8D49159F81F
:10F28000321009EBC200C1F38301013940680C2937
:10F290007DD8DFE801F080807C7C7C7C7C7C467CB7
:10F2A0007C7C0700D0F800E0724C4168724F734ECE
:10F2B0006160C4F800E01FFA8EF140F2816E002513
:10F2C000674B49F83230012071453D60C9F8105054
:10F2D000C9F8185030705E4A00F20881B1F5D06F5D
:10F2E00080F08283B1F5817F00F0668300F28F8227
:10F2F000802900F07483822940F0A782A18801F060
:10F300007F01042900F2A1825D4B5E4A89000B4413
:10F310001570557019788D0740F1808310700220A8
:10F32000F2E2554F3A6842B3574B544E574918884A
:10F3300034780D784028864645F0020828BF4FF003
:10F34000400E002C84F001043470CEEB00000CBFA2
:10F350008824C82409EBC80680B285F0010544EA78
:10F360000E447260188049F8384072440D7018B924
:10F37000BEF1400F18BF00223A603E4B1A88B2F52A
:10F38000A06F04D100219A785970414B1A70414AFC
:10F39000012313703EE7374C258842F221018D424C
:10F3A00000F05A8224683C49324D8C4200F00082C1
:10F3B0002B4949F83210EAE7294A2A4B19F0080F7D
:10F3C00018BF134647F8383024E700F0BBFC334A37
:10F3D000334952F82630002B78D058688C5D42F8BB
:10F3E000260003F10802C9F80420032C05D8DFE841
:10F3F00004F0120F150204228A551A8819F0080F1A
:10F400000CBF8823C82343EA024347F8383001E79A
:10F4100002228A55F1E703228A55EEE705228A5532
:10F42000EBE7E00700F13082210600F15F82A207DE
:10F4300006D51C4A1C4913780220DBB213700870F1
:10F44000E30602D5184B10221A7007B0BDE8F08F02
:10F450000080FF1F08A1FF1FB4A0FF1F60A2FF1FB5
:10F46000C80040008800400090A1FF1F19A1FF1FA5
:10F4700004A2FF1F7CA1FF1FB0A0FF1F18A1FF1F48
:10F48000C020074088A1FF1FC4A0FF1F84A1FF1F49
:10F490009820074094200740210900035CA1FF1F2A
:10F4A00094A1FF1F8820074080200740902007403C
:10F4B00000F0ACFFCFE6AC4A47F8380013780133D0
:10F4C0001370A7E643F82600A84D8AE68B5D032B50
:10F4D00000F26B8201A252F823F000BF15F2000087
:10F4E00015F20000DDF80000D7F8000040F6211505
:10F4F000A94200F0358100F29F81B1F5086F00F05C
:10F50000FF81B1F5106F40F0A0819948116AA4788D
:10F5100004700C0600F19382D9F828209549100652
:10F5200000F18882D9F830209249120600F17D82DC
:10F53000D9F838208F49130600F17282D9F840209B
:10F540008C49150600F12E83D9F848208949140604
:10F5500000F12383D9F850208649100600F1188362
:10F56000D9F858208349120600F10D83D9F860209C
:10F570008049130600F12083D9F868207D491506DB
:10F5800000F11583D9F870207A49140600F1DE8263
:10F59000D9F878207749100600F1D382D9F8802075
:10F5A0007449120600F1E982D9F8882071491306DE
:10F5B00000F1DD82D9F890206E49150600F1D18264
:10F5C000D9F898206B49140600F1C5826A486B4A45
:10F5D0006B4901906B486C4C644D02940023049776
:10F5E000059680461C4617460E460395386828B196
:10F5F000456800F0A7FB2846002DF9D100233B60A9
:10F60000039B30681A46002342F8243028B145682D
:10F6100000F098FB2846002DF9D100223260019AB3
:10F6200098F800301146002241F8042B029A01910B
:10F63000023B4FF0000122F81410032B09D8DFE839
:10F6400013F050010400500104004FF0010388F84A
:10F6500000300134042C07F1040706F1040608F118
:10F660000108C3D1494C404D2278494B049F059E67
:10F670000021100729701A7000F14E824549627806
:10F680000A700021C9F83010C9F838101107DFF8E6
:10F69000E48000F12C82A2783F49DFF8D8800A701C
:10F6A00000211207C9F85010C9F8581000F108825B
:10F6B000E2783A492F4C0A7013074FF00001C9F85D
:10F6C0007010C9F8781000F1BF81337802930022DE
:10F6D00083F00105C9F89020C9F898200020019016
:10F6E0008046864602462E490C7844F0020C09EB0F
:10F6F000CC030393029B002B039B5A600CBF882210
:10F70000C82242EA080384F0010249F83C3035700F
:10F710000A70DFF860C0234BDFF88480002840F0D7
:10F720001681BEF1400F1BD142F0020C09EBCC0355
:10F73000019ADFF840E05A60002D40F01E81050478
:10F7400045F088059DF808304EF83C50024433706F
:10F750000C701346402803D10020134A3B601080F0
:10F76000124A0123137012E685A1FF1FB4A0FF1FE8
:10F7700090A1FF1F0080FF1F6CA1FF1F08A1FF1FAA
:10F780005CA1FF1F94A1FF1F60A2FF1FD4580100BE
:10F79000C4200740C8200740CC200740D0200740A5
:10F7A00084A1FF1F18A1FF1FC4A0FF1F94200740C2
:10F7B0006C68B1498C427FF4FBAD0178A9297FF4D4
:10F7C000F7AD417845297FF4F3AD8178C2297FF404
:10F7D000EFADC1786B297FF4EBADA849A84E08784E
:10F7E000347880F00105002C40F002000D700CBF51
:10F7F0008821C82184F0010449F8301009EBC000C9
:10F80000A04934700025052445600C70D0E540F215
:10F810000232914240F09480A28802F07F02042AD2
:10F8200013D865888DB998490290920011440A78DE
:10F8300042F002020A7051E740F62122914200F0A4
:10F84000828042F2212291427DD08F4A0F23137091
:10F850008E4A012313709AE58849894E0D783778CE
:10F8600085F0010E002F45F0020581F800E00CBF85
:10F870008821C82149F8351009EBC50587F0010733
:10F880000021377069608DE5814B80487B491A61A2
:10F890004FF0020E80F800E07B4F0A707D4919603E
:10F8A00099607D4E7D4D7E4C9A610D213970FF210E
:10F8B0003170DFF808E2297022707A4D7A4A8EF8AA
:10F8C00000109F27012406F8047C5D600470DA6054
:10F8D00007B0BDE8F08F01238B559BE400238B55C7
:10F8E00098E44FF0000388F80030B2E666496B4BAD
:10F8F00080220D2008701A70A2077FF5A1AD98E54F
:10F900006A496B4A09781170E588854280F08981DF
:10F910005A490C78402DAE4644F0020C28BF4FF0F7
:10F92000400E02EB0E0309EBCC0001930123426071
:10F930004FEA0E48CEEB050002930025C822E0E610
:10F94000B1F5A06F81D1012300250293C6E64028BE
:10F950007FF6EAAE42F002020CEBC201019E4E605D
:10F96000BDB19DF8085053491D703346403888F8A2
:10F97000004040334CF83210EFE69DF80830337009
:10F980000504019B0C7045F0C80503444EF83C503B
:10F99000E0E69DF808501D70019B3E4988F8004044
:10F9A000403840334CF83210D7E619F0080F0CBF3E
:10F9B000022303238B552DE4A28802F07F02042A40
:10F9C0003FF643AF6588002D7FF43FAF2E4902908C
:10F9D000920011440A7822F002020A707EE6344A4C
:10F9E0000220157055708FE733494A68002A3FF4AA
:10F9F0002CAF6588B4F804E004E00C314A68002AB2
:10FA00003FF423AF0B88AB42F7D14B887345F4D159
:10FA10002D0A032D0CBF1078088975E7022073E7C3
:10FA2000C86B083800F08EF988E5486B083800F09C
:10FA300089F97DE5C86A083800F084F972E5506AF2
:10FA4000083800F07FF967E500F05CF9002800F065
:10FA5000D68008300F4AC4F88400C4F8802000F033
:10FA600051F9002800F0C5800830124AC9F88C000E
:10FA7000C9F8882029E600BF0100040084A1FF1F07
:10FA800018A1FF1F19A1FF1FC020074094200740A5
:10FA90000080FF1F8800400088200740802007402A
:10FAA00098200740C8A0FF1F1CA1FF1F90A1FF1FA7
:10FAB00088A1FF1FC8004000D85801008C200740D3
:10FAC00000F020F9002800F0A68008305D4AC8F850
:10FAD0006400C8F8602000F015F9002800F0958057
:10FAE0000830594AC9F86C00C9F86820E0E500F010
:10FAF00009F9002877D00830524AC8F84400C8F8FD
:10FB0000402000F0FFF8002867D008304E4AC9F8BE
:10FB10004C00C9F84820BEE500F0F4F8002856D0A3
:10FB20000830484AC9F82400C9F8202000F0EAF853
:10FB3000002846D00830444AC9F82C00C9F82820CB
:10FB40009CE5C86F083800F0FDF827E5486F0838D5
:10FB500000F0F8F81CE5D1F89C00083800F0F2F845
:10FB600034E5D1F89400083800F0ECF828E5D1F835
:10FB70008C00083800F0E6F81CE5D1F8840008385D
:10FB800000F0E0F810E5C86D083800F0DBF8EDE4AF
:10FB9000486D083800F0D6F8E2E4C86C083800F088
:10FBA000D1F8D7E4486C083800F0CCF8CCE4C86E43
:10FBB000083800F0C7F8E5E4486E083800F0C2F8ED
:10FBC000DAE42A78C9F8280001322A7056E52A7842
:10FBD000C9F8200001322A70A8E72A78C9F848003D
:10FBE00001322A7057E52A78C8F8400001322A709D
:10FBF00087E72A78C9F8880001322A7065E52A78F3
:10FC0000C4F8800001322A7029E72A78C9F8680010
:10FC100001322A704CE52A78C8F8600001322A7057
:10FC200059E74028864628BF4FF0400E02EB0E03EE
:10FC300001930123CEEB00004FEA0E48002502930A
:10FC400051E500BE88004000C80040002DE9F8439F
:10FC5000204C00F037FF002204F1A00023461A6078
:10FC60005A60083383424FF00001F8D11A4A1B4F03
:10FC700013681B4D1B481C4EDFF87880DFF878C0F6
:10FC8000DFF87890DFF878E043F480231360C4F362
:10FC900007233B70C4F307432B70240EFF2302F5A8
:10FCA00028320470114D88F8003011488CF800306B
:10FCB000D4323370012389F8003070268EF800109A
:10FCC0004FF40074102107F8183C2E700460117076
:10FCD000BDE8F8830080FF1F348004409C2007406B
:10FCE000B0200740B42007401020074049E400E05E
:10FCF00008E100E08020074088200740942007406A
:10FD00000021074072B60D480268B2FA82F30F2B49
:10FD100010DC4FF00041D94022EA0102026062B6D5
:10FD2000074803EBC303DB00C2180021C150104693
:10FD30005160704762B60020704700BFA492FF1F59
:10FD4000BC83FF1F0D4B0E4AC31AA2FB03231B09E2
:10FD50000F2B0CD80B4A127852B972B60A484FF0E2
:10FD60000041026821FA03F31A43026062B6704749
:10FD7000064A1278002AF0D0FFF75AB9BC83FF1F59
:10FD8000398EE33885A1FF1FA492FF1F90A1FF1FAA
:10FD900038B50E4B0E4C1B68218805468BB1B1F56A
:10FDA000917F05D20B4A4B1C55549BB2238038BD22
:10FDB0000022084898470021064A55540123238011
:10FDC00038BDB1F5917FEDD338BD00BFBCA1FF1F99
:10FDD0006AA2FF1F70A2FF1F2DE9F843214E224F98
:10FDE0003168012380463B70B1B1204D4B8801EB57
:10FDF0008302013300240F2BC2F808802C7004D832
:10FE00004B8000233B70BDE8F88340230B80032028
:10FE1000FFF772F93460F4E7DFF8549099F8003096
:10FE2000002BF0D0114D45F6215408E0013C12D0D2
:10FE30002B7883B900F0AAFD99F800307BB103203C
:10FE4000FFF7E0F80528F1D8FFF75CFF01463060C6
:10FE50000028EBD0CAE701232B70BDE8F883BDE88A
:10FE6000F88300BFD8A1FF1FACA1FF1FDCA1FF1FBB
:10FE700090A1FF1F1201F8B5D5B2A1B3012943D05B
:10FE80004378044600781B0643EA004040F4704083
:10FE900045F004068F1E3043FFF79EFF022F04F14A
:10FEA000020314D9053414F8023C14F8032C14F896
:10FEB000010C1B0443EA0223334343EA0060033F7F
:10FEC000FFF78AFF022F234604F10304EBD8022F29
:10FED00023D0012F0DD045F4774040F00500BDE858
:10FEE000F840FFF779BF14482843BDE8F840FFF712
:10FEF00073BF187845F4770545F0060545EA0020FC
:10FF0000BDE8F840FFF768BF03780C4845EA0345B1
:10FF10002843BDE8F840FFF75FBF1A78587845F0EE
:10FF2000774545F0070545EA022545EA0040BDE86A
:10FF3000F840FFF751BF00BF06F0F70007F000F7E9
:10FF400038B5084B1C7824B9074D296809B14B888E
:10FF500003B938BD9B000B800320FFF7CDF82C6060
:10FF600038BD00BFACA1FF1FD8A1FF1F2DE9F04194
:10FF7000AD4E33680746002B00F092801D885A88EA
:10FF8000910803EB81010432AA428C6842D25A8064
:10FF900004F00F064FEA1428A449A6F1080208F05D
:10FFA0000F00C4F30313062A00F101050B701AD9E0
:10FFB000B31E012B5FFA88F04ED9052E48D0042ECF
:10FFC00000F0A481731F022B7FD90F2E0ED1F728CA
:10FFD00042D8F02802D0964B1B883BB1FFF7D8FEE1
:10FFE0000020BDE8F08127B1BD4202D00020BDE86D
:10FFF000F081082EC4F3033300F08780092E11D05E
:020000021000EC
:100000000A2E40F094800A2BF0D18A4B8A4A1B6852
:10001000A02181E01846FFF795FE0420FEF7D4FFEB
:100020003060B5E7092BE1D1270E00F07B81834BCF
:10003000814A1B689021C4F307461170EDB2FCB2EF
:10004000002B00F09D80224631462846984797E0D5
:10005000F02843D9F72841D0F1380E28C6D801A39B
:1000600053F820F01B020100FF010100ED01010027
:10007000EDFF0000EDFF0000DF010100EDFF0000DB
:10008000BF020100EDFF000089020100A302010090
:10009000C7010100EDFF0000AF0101009301010065
:1000A000674B1B78002BA1D00420FEF78DFF034681
:1000B000306000289AD00588002D7FF460AFFFF7EC
:1000C00041FE35602846BDE8F081FFF761FEC4F3CC
:1000D0000740FFF75DFE072E02D1200EFFF758FE06
:1000E000534B584A198858481468584D524A017061
:1000F00000270E0AF0201F802E7010700CB3012212
:100100005348A0470120BDE8F081082B7FF46EAF73
:10011000504B494A1B688021C4F307461170EDB269
:10012000240E6BB3284622463146984728E00B2E12
:1001300011D10B2B7FF45AAF474B3F4A1B68B021BC
:10014000EAE7464B1B68002B00F0FB8040489847CD
:100150000120BDE8F0810C2E40F000810C2B7FF4D3
:1001600045AF3F4B344A1B68C0211170EDB2C4F358
:100170000746002B00F0C88028463146240E9847D9
:100180003849314A314B0D7016701C700120BDE8A2
:10019000F081354B1B68002B00F0D6809847C4F3E4
:1001A0000746254BEDB2240E83F80080E8E72F4B7D
:1001B0001B68002BF2D12E4B1B68A3B1FE20984781
:1001C000C4F30746EDE72B4B1B68002BE6D1284B09
:1001D0001B6843B1FC209847C4F30746E1E7264B70
:1001E0001B68002BDAD1C4F30746DAE7234B1B6800
:1001F000C4F30746002BD4D030469847D1E7204BB4
:100200001A68002AEFD0260C630C06F07F0003F476
:100210007E531843F6B29047C3E71A4B1B68C4F3EA
:100220000746002BE8D1BCE7E4A1FF1F6EA2FF1F29
:100230006AA2FF1FC0A1FF1F68A2FF1FF4A1FF1F3A
:1002400090A1FF1FBCA1FF1F6CA2FF1F6DA2FF1F8B
:1002500070A2FF1FECA1FF1FF0A1FF1FD4A1FF1F81
:10026000B0A1FF1F6FA2FF1F9CA1FF1FA0A1FF1F36
:10027000A4A1FF1FE0A1FF1FD0A1FF1FE8A1FF1F46
:10028000B8A1FF1FCCA1FF1F3F4B1B68002B85D1DE
:100290003E4B1B68002BA6D0FA209847C4F30746B4
:1002A0007FE73B4B1B68002B7FF478AF374B1B6815
:1002B000002B98D0FB209847C4F3074671E7354BD5
:1002C0001B68002B7FF46AAF304B1B68002B8AD071
:1002D000F8209847C4F3074663E70E2B7FF486AEF9
:1002E0002D4A2E4B1268E0211970002A47D0260CA7
:1002F000610C06F07F0301F47E511943EDB2A1F5C4
:10030000005128469047F6B2240E39E7FFF740FD2A
:10031000C4F30740FFF73CFD200EFFF739FD002036
:10032000BDE8F0811E4B1D4A1B6880211170EDB2A3
:10033000C4F3074683B1314628463A4698473C46BF
:100340001EE70120BDE8F081104B1B68002B3FF435
:100350004AAFFF20984746E71C4611E70D2EBCD157
:100360000D2B7FF443AE0F4B0C4A1B68D02111704C
:10037000EDB2C4F30746002B7FF4FEAEC4E7C4F32E
:100380000746EDB2240EFBE6C8A1FF1FA4A1FF1F84
:10039000A8A1FF1F98A1FF1FB4A1FF1F68A2FF1F04
:1003A000ECA1FF1FC4A1FF1F38B5164D2868E0B1AE
:1003B00001884488A14213DD03191B7A83B104F13B
:1003C0000803C2180C1B002302E012F8011F21B120
:1003D0000133A342F9D1204638BD1C46204638BD22
:1003E000FFF7B0FC0020286038BD074B1B780BB925
:1003F000002038BD0220FEF7E7FD28600028D7D195
:10040000F6E700BF00A2FF1F90A1FF1F0D4B1B7856
:10041000BBB910B50C4C216803F0FF024B883F2B91
:1004200007DC07330B4401F1470003F8012F834237
:10043000FBD140230B800120FEF75EFE00232360EA
:1004400010BD7047F8A1FF1FFCA1FF1F70B5EFF3AF
:10045000108272B60C4C206880B10C4E00254369A6
:10046000236073B19D6102B962B64577836898478E
:10047000EFF3108272B620680028F0D102B962B69C
:1004800070BD3360EFE700BF08A2FF1F0CA2FF1F83
:10049000FFF7DCBF024A136801331360704700BFE7
:1004A000B49FFF1F4B0803F1376303F5D83310B532
:1004B0000446B3FBF1F0FDF7EDFE044B1B7803B1EE
:1004C00010BD2046BDE8104000F03EBBE092FF1F8B
:1004D00008B50846FEF7A8F8012008BD08B508468B
:1004E000FEF7A2F8012008BD38B508460D4602F017
:1004F000E7FA044601462846FEF7EEF8204638BDE6
:1005000010B5084614461146FEF7E6F8204610BD21
:10051000FEF7C0B908B50846FEF766F8003018BF08
:10052000012008BD08B50846FEF73CF8003018BFAA
:10053000012008BD08461146FDF7CCBF0846FEF76E
:1005400003B800BF0846FDF7A9BF00BFFDF744BFD1
:1005500010B54B0803F13760144600F5D830B0FBF6
:10056000F1F0FDF797FE2046BDE81040FDF708BF0B
:10057000FEF778B9FEF742B9FEF730B9FEF710B9C9
:10058000FEF71AB90368064A1B68934205D110B5F5
:10059000C8B2FEF749F8012010BDC9B2184700BF24
:1005A000DD0401000368064A1B68934205D110B5BB
:1005B000C8B2FEF739F8012010BDC9B2184700BF14
:1005C000DD0401000368064A1B68934205D110B59B
:1005D000C8B2FEF729F8012010BDC9B2184700BF04
:1005E000DD0401000368064A1B68934205D110B57B
:1005F000C8B2FEF719F8012010BDC9B2184700BFF4
:10060000DD0401004B0803F1B76303F5584310B54F
:100610000446B3FBF1F0FEF73BFA044B1B7803B141
:1006200010BD2046BDE8104000F08EBAE192FF1FD9
:1006300008B50846FEF76AFB012008BD08B5084664
:10064000FEF764FB012008BD38B508460D4602F0F0
:1006500037FA044601462846FEF762FB204638BDBD
:1006600010B5084614461146FEF75AFB204610BD49
:10067000FEF7E6BB08B50846FEF728FB003018BFBA
:10068000012008BD08B50846FEF7FEFA003018BF85
:10069000012008BD08461146FEF7CCBA0846FEF711
:1006A000F1BA00BF0846FEF7A9BA00BFFEF76CBA60
:1006B00010B54B0803F1B760144600F55840B0FB85
:1006C000F1F0FEF7E5F92046BDE81040FEF730BA3C
:1006D000FEF79EBBFEF768BBFEF756BBFEF736BBC8
:1006E000FEF740BB0368064A1B68934205D110B56C
:1006F000C8B2FEF70BFB012010BDC9B2184700BFFE
:100700003D0601000368064A1B68934205D110B5F7
:10071000C8B2FEF7FBFA012010BDC9B2184700BFEE
:100720003D0601000368064A1B68934205D110B5D7
:10073000C8B2FEF7EBFA012010BDC9B2184700BFDE
:100740003D0601000368064A1B68934205D110B5B7
:10075000C8B2FEF7DBFA012010BDC9B2184700BFCE
:100760003D060100704700BF0368F0B4FBB10025EF
:1007700001249D60DC601B4C1A601C44241104F1B0
:1007800044056A11032692009E60174F0679174BA5
:1007900047F8241002F1604202F5614205F01F059E
:1007A000012000FA05F5E6541560F0BC7047104CC6
:1007B000236843F40003236000BF0E4B0E4DA4F5E5
:1007C0008734A4F59E7401261E60234604609C684D
:1007D000002CD0D01033AB420360F8D1002303606B
:1007E0001846E2E7008FFCBFD092FF1F44E400E010
:1007F0003C80044000700340407103400168A9B18F
:100800000B4BF0B40B441B110A4E0B4F0B4D46F82B
:10081000237003F1440202F01F0401235211A3408C
:10082000002445F822308C600460F0BC704700BFA3
:10083000008FFCBFD092FF1F6507010080E100E040
:10084000024A034B012111601B6818470C710340D9
:10085000D092FF1F024A034B012111605B681847C9
:100860001C710340D092FF1F024A034B012111600B
:100870009B6818472C710340D092FF1F024A034B1C
:1008800001211160DB6818473C710340D092FF1FC3
:10089000F8B50E4671B17AB10746144600253B689B
:1008A00016F8011B1B6838469847013C0544F6D1F1
:1008B0002846F8BD0846F8BD1046F8BD00B5064A02
:1008C000036812885B6883B001A9ADF80420022296
:1008D000984703B05DF804FBD0580100F0B5074617
:1008E0008BB0002A33D0012A08BF0A2251B3212439
:1008F00000E0F4B2B1FBF2F502FB1511C8B2092910
:1009000000F1300198BFC8B20AA988BF373021442E
:1009100088BFC0B201F8240C661E2946002DE8D11C
:1009200033B1013CE4B20AAB23442D2203F8242C5A
:100930003B6801AA11195B683846C4F12202984746
:100940000BB0F0BD30228DF825202124E8E70368A4
:10095000C9B21B6898470BB0F0BD00BF0029BABFF1
:1009600049422D2300230A22FFF7B8BF08B5F1F74B
:1009700067F9F1F7D7FD00F009F8FAE701F014BBC9
:1009800001F01ABB704700BF704700BF2DE9F84364
:10099000314E337893B1314F3A787AB90122D90781
:1009A0003A7036D49A0719D400225B073A7005D5FD
:1009B0002B4B1A6812B1EFF305820AB1BDE8F88338
:1009C000EFF3108172B6186818B1264C2278002A0D
:1009D0002ED00029F2D162B6BDE8F883DFF890800E
:1009E00098F80020002ADFD0DFF88890002405E086
:1009F000013498F80030E4B2A34212D959F82450D7
:100A00002B6828461B6998470028F1D02B69984726
:100A1000EEE7FFF7C9FCC8B9134B1B781BB9337855
:100A2000C0E73378C0E7337803F0FE033370B9E7EB
:100A300045691D60012323705DB1AA6101B962B6E9
:100A400000254577836898472570B7E700F092F84E
:100A5000E2E7064B1D60F1E7E292FF1F19A2FF1FBC
:100A600014A2FF1F18A2FF1FC293FF1F10A2FF1F97
:100A700028A2FF1F1CA2FF1FF0B44D1E2E4600240B
:100A800000E00134B0FBF2F302FB1300092800F18F
:100A900030078ABF3730F8B2C0B206F8010F1846E7
:100AA000002BEED10A1953704CB1107815F8016F74
:100AB00028700133E01A834202F80169F5DB084629
:100AC000F0BC704770B584B072B6194B194D1A4816
:100AD000702241260F2480211A702E701A4604704D
:100AE000197013781B06FCD5144B186862B6144BAA
:100AF000144C984298BF00EB800001A998BF4000B9
:100B00000A22FFF7B9FF01A92046002311F8012BA3
:100B100001333AB10A2B20F8022FF7D116232370A4
:100B200004B070BD5B00DBB2237004B070BD00BFC9
:100B30000000024007000240060002400800024098
:100B40007F969800AC93FF1F30B40749074C0A7892
:100B50002378074D42F0020245F823000A70013362
:100B6000237030BC704700BFE292FF1F28A2FF1F16
:100B70001CA2FF1F704700BF2DE9F043DFF8EC8097
:100B80008BB006460F4600F073F898F90030013339
:100B900004460D4637D03046394600F0DFF90028CC
:100BA00031D02BA3D3E900233046394600F02CFE88
:100BB000814668BB28A3D3E900233046394600F0BC
:100BC00005FE00B398F90030254ACDF820900424A2
:100BD00000200021022BCDE90467CDE902670094D3
:100BE0000192CDE906012CD0684600F0BDF940B372
:100BF000089B1BB101F0AAF9089B0360DDE906011F
:100C00000BB0BDE8F083204629460BB0BDE8F08369
:100C1000134A98F90030019203210022CDE90467BC
:100C2000CDE90267009108922BB90E4B4FF060425C
:100C3000CDE90623D8E70C490020022BCDE90601B7
:100C4000D2D101F083F922230360D1E7AFF3008012
:100C5000EF39FAFE422E864051302DD5104987C01B
:100C600044590100FFFFEF470000F07FC393FF1FCF
:100C70002DE9F04FB04F21F00042BA4283B00C464C
:100C80004FEAD17605460DD9AC4FBA4225D9C1F30A
:100C90001303034340F0EF800EB10020014603B080
:100CA000BDE8F08FA64B9A4200F2CC80A54B9A4249
:100CB00000F2DE808AA3D3E9002300F063F900226A
:100CC000A14B00F0A1FD002800F005812846214637
:100CD00000229D4B00F056F9E1E783A3D3E90023FE
:100CE00000F092FD002840F0CB802846214680A3EA
:100CF000D3E9002300F06AFD0028CED1934B2846AB
:100D000003EBC60821467CA3D3E9002300F0ECFAEC
:100D1000D8E9002300F036F900F080FD804600F0AD
:100D20007DFA77A3D3E9002306460F4600F0DCFAEC
:100D300002460B462846214600F022F972A3D3E969
:100D40000023CDE900013046394600F0CDFA824655
:100D50008B4652465B46DDE9000100F011F905467D
:100D60000C462A4623462846214600F0BDFA68A3D1
:100D7000D3E9002306460F4600F0B6FA66A3D3E98E
:100D8000002300F0FDF832463B4600F0ADFA64A3C4
:100D9000D3E9002300F0F6F832463B4600F0A4FA0F
:100DA00061A3D3E9002300F0EBF832463B4600F0A4
:100DB0009BFA5FA3D3E9002300F0E4F832463B46F8
:100DC00000F092FA02460B462846214600F0D8F879
:100DD00006460F462846214632463B46B8F1000FEC
:100DE00056D000F081FA324604460D463B460020BC
:100DF0004FF0804100F0C4F802460B4620462946D9
:100E000000F09CFB02460B465046594600F0B8F8ED
:100E1000DDE9002300F0B4F80B4602464A49002001
:100E200000F0AEF86FF47F7398454FDA08F57A78E2
:100E300001EB085100224FF0B87300F055FA03B0EF
:100E4000BDE8F08F424B9A423FF658AF414BF40059
:100E50002344D3E9002300F093F83F4BC6F1010887
:100E60001C44CDE90001D4E900ABC6EB080870E7EB
:100E70004FF0000875E702460B4600F083F80EE7D6
:100E800017A3D3E900231046194600F02DFA06E710
:100E900000F02AFA0022804689464FF0804330460F
:100EA000394600F06DF802460B464046494600F0D0
:100EB00045FB2A46234600F063F802460B46002015
:100EC000214900F05DF803B0BDE8F08F01EB085157
:100ED00003B0BDE8F08F804643E700BFAFF300806A
:100EE0009C7500883CE4377EEF39FAFE422E86403E
:100EF00051302DD5104987C0FE822B654715F73F2D
:100F00000000E0FE422EE63F763C7935EF39EA3DBF
:100F1000D0A4BE726937663EF16BD2C541BDBB3EFF
:100F20002CDE25AF6A56113F93BDBE166CC1663FDD
:100F30003E5555555555C53F412E8640FFFFEF7F25
:100F4000422ED63FFFFF2F3E0000F03F48590100E0
:100F5000B1A2F03F685901005859010041F0004129
:100F600001F58010C00F7047002070470B46014606
:100F7000184600F0E5BF00BF81F0004102E000BF6D
:100F800083F0004330B54FEA41044FEA430594EA49
:100F9000050F08BF90EA020F1FBF54EA000C55EA84
:100FA000020C7FEA645C7FEA655C00F0E2804FEA55
:100FB0005454D4EB5555B8BF6D420CDD2C4480EA37
:100FC000020281EA030382EA000083EA010180EA67
:100FD000020281EA0303362D88BF30BD11F0004FB5
:100FE0004FEA01314FF4801C4CEA113102D04042EB
:100FF00061EB410113F0004F4FEA03334CEA133326
:1010000002D0524263EB430394EA050F00F0A7803D
:10101000A4F10104D5F1200E0DDB02FA0EFC22FA38
:1010200005F2801841F1000103FA0EF2801843FA2C
:1010300005F359410EE0A5F120050EF1200E012A1D
:1010400003FA0EFC28BF4CF0020C43FA05F3C0185B
:1010500051EBE37101F0004507D54FF0000EDCF1D4
:10106000000C7EEB00006EEB0101B1F5801F1BD37D
:10107000B1F5001F0CD349085FEA30004FEA3C0C81
:1010800004F101044FEA445212F5800F80F09A8077
:10109000BCF1004F08BF5FEA500C50F1000041EB7B
:1010A000045141EA050130BD5FEA4C0C404141EB7F
:1010B000010111F4801FA4F10104E9D191F0000FA6
:1010C00004BF01460020B1FA81F308BF2033A3F129
:1010D0000B03B3F120020CDA0C3208DD02F1140C20
:1010E000C2F10C0201FA0CF021FA02F10CE002F15B
:1010F0001402D8BFC2F1200C01FA02F120FA0CFC54
:10110000DCBF41EA0C019040E41AA2BF01EB04519C
:10111000294330BD6FEA04041F3C1CDA0C340EDC9A
:1011200004F11404C4F1200220FA04F001FA02F3DD
:1011300040EA030021FA04F345EA030130BDC4F19B
:101140000C04C4F1200220FA02F001FA04F340EA90
:101150000300294630BD21FA04F0294630BD94F041
:10116000000F83F4801306BF81F480110134013D28
:101170004EE77FEA645C18BF7FEA655C29D094EA99
:10118000050F08BF90EA020F05D054EA000C04BF17
:101190001946104630BD91EA030F1EBF0021002002
:1011A00030BD5FEA545C05D14000494128BF41F0A1
:1011B000004130BD14F580043CBF01F5801130BD05
:1011C00001F0004545F0FE4141F470014FF0000090
:1011D00030BD7FEA645C1ABF194610467FEA655C41
:1011E0001CBF0B46024650EA013406BF52EA0335E3
:1011F00091EA030F41F4002130BD00BF90F0000FD1
:1012000004BF0021704730B54FF4806404F132040C
:101210004FF000054FF0000150E700BF90F0000FC5
:1012200004BF0021704730B54FF4806404F13204EC
:1012300010F0004548BF40424FF000013EE700BFBC
:1012400042004FEAE2014FEA31014FEA02701FBF4C
:1012500012F07F4393F07F4F81F06051704792F01E
:10126000000F14BF93F07F4F704730B54FF4607498
:1012700001F0004521F0004120E700BF50EA0102E3
:1012800008BF704730B54FF000050AE050EA010290
:1012900008BF704730B511F0004502D5404261EB00
:1012A00041014FF4806404F132045FEA915C3FF441
:1012B000DCAE4FF003025FEADC0C18BF03325FEADA
:1012C000DC0C18BF033202EBDC02C2F1200300FA8F
:1012D00003FC20FA02F001FA03FE40EA0E0021FAB4
:1012E00002F11444C1E600BF70B54FF0FF0C4CF49E
:1012F000E06C1CEA11541DBF1CEA135594EA0C0F54
:1013000095EA0C0F00F0DEF82C4481EA030621EA8E
:101310004C5123EA4C5350EA013518BF52EA0335C9
:1013200041F4801143F4801338D0A0FB02CE4FF07B
:101330000005E1FB02E506F00042E0FB03E54FF0AB
:101340000006E1FB03569CF0000F18BF4EF0010EA3
:10135000A4F1FF04B6F5007F64F5407404D25FEA9F
:101360004E0E6D4146EB060642EAC62141EA555152
:101370004FEAC52040EA5E504FEACE2EB4F1FD0C94
:1013800088BFBCF5E06F1ED8BEF1004F08BF5FEA12
:10139000500E50F1000041EB045170BD06F00046C4
:1013A00046EA010140EA020081EA0301B4EB5C0471
:1013B000C2BFD4EB0C0541EA045170BD41F4801169
:1013C0004FF0000E013C00F3AB8014F1360FDEBF8E
:1013D000002001F0004170BDC4F10004203C35DA6A
:1013E0000C341BDC04F11404C4F1200500FA05F3ED
:1013F00020FA04F001FA05F240EA020001F000428E
:1014000021F0004110EBD37021FA04F642EB060103
:101410005EEA430E08BF20EAD37070BDC4F10C042D
:10142000C4F1200500FA04F320FA05F001FA04F2F1
:1014300040EA020001F0004110EBD37041F10001DD
:101440005EEA430E08BF20EAD37070BDC4F12005E8
:1014500000FA05F24EEA020E20FA04F301FA05F250
:1014600043EA020321FA04F001F0004121FA04F2F8
:1014700020EA020000EBD3705EEA430E08BF20EAC8
:10148000D37070BD94F0000F0FD101F00046400002
:1014900041EB010111F4801F08BF013CF7D041EA84
:1014A000060195F0000F18BF704703F00046520088
:1014B00043EB030313F4801F08BF013DF7D043EA59
:1014C0000603704794EA0C0F0CEA135518BF95EA0F
:1014D0000C0F0CD050EA410618BF52EA4306D1D196
:1014E00081EA030101F000414FF0000070BD50EAB5
:1014F000410606BF1046194652EA430619D094EA3F
:101500000C0F02D150EA013613D195EA0C0F05D128
:1015100052EA03361CBF104619460AD181EA03017C
:1015200001F0004141F0FE4141F470014FF0000034
:1015300070BD41F0FE4141F4780170BD70B54FF0CF
:10154000FF0C4CF4E06C1CEA11541DBF1CEA13554F
:1015500094EA0C0F95EA0C0F00F0A7F8A4EB050431
:1015600081EA030E52EA03354FEA013100F0888028
:101570004FEA03334FF0805545EA131343EA1263F1
:101580004FEA022245EA111545EA10654FEA0026A6
:101590000EF000419D4208BF964244F1FD0404F55F
:1015A000407402D25B084FEA3202B61A65EB0305BB
:1015B0005B084FEA32024FF480104FF4002CB6EB78
:1015C000020E75EB030E22BFB61A754640EA0C00F8
:1015D0005B084FEA3202B6EB020E75EB030E22BF38
:1015E000B61A754640EA5C005B084FEA3202B6EB79
:1015F000020E75EB030E22BFB61A754640EA9C0038
:101600005B084FEA3202B6EB020E75EB030E22BF07
:10161000B61A754640EADC0055EA060E18D04FEAC5
:10162000051545EA16754FEA06164FEAC30343EA65
:1016300052734FEAC2025FEA1C1CC0D111F4801F32
:101640000BD141EA00014FF000004FF0004CB6E72B
:1016500011F4801F04BF01430020B4F1FD0C88BFCA
:10166000BCF5E06F3FF6AFAEB5EB030C04BFB6EBD5
:10167000020C5FEA500C50F1000041EB045170BDC8
:101680000EF0004E4EEA113114EB5C04C2BFD4EBF5
:101690000C0541EA045170BD41F480114FF0000E79
:1016A000013C90E645EA060E8DE60CEA135594EAF5
:1016B0000C0F08BF95EA0C0F3FF43BAF94EA0C0FF8
:1016C0000AD150EA01347FF434AF95EA0C0F7FF46D
:1016D00025AF104619462CE795EA0C0F06D152EAC1
:1016E00003353FF4FDAE1046194622E750EA4106A5
:1016F00018BF52EA43067FF4C5AE50EA41047FF4B6
:101700000DAF52EA43057FF4EBAE12E74FF0FF3C1A
:1017100006E000BF4FF0010C02E000BF4FF0010CEB
:101720004DF804CD4FEA410C7FEA6C5C4FEA430C64
:1017300018BF7FEA6C5C1BD001B050EA410C0CBFB3
:1017400052EA430C91EA030F02BF90EA020F002015
:10175000704710F1000F91EA030F58BF994208BF7C
:1017600090422CBFD8176FEAE37040F00100704739
:101770004FEA410C7FEA6C5C02D150EA013C07D190
:101780004FEA430C7FEA6C5CD6D152EA033CD3D0DB
:101790005DF8040B704700BF8446104662468C46D5
:1017A0001946634600E000BF01B5FFF7B7FF002808
:1017B00048BF10F1000F01BD4DF808EDFFF7F4FF31
:1017C0000CBF012000205DF808FB00BF4DF808EDBC
:1017D000FFF7EAFF34BF012000205DF808FB00BFDF
:1017E0004DF808EDFFF7E0FF94BF012000205DF801
:1017F00008FB00BF4DF808EDFFF7CEFF94BF0120B6
:1018000000205DF808FB00BF4DF808EDFFF7C4FFAE
:1018100034BF012000205DF808FB00BF4FEA410201
:1018200012F5001215D211D56FF47873B3EB625232
:1018300012D94FEAC12343F0004343EA505311F059
:10184000004F23FA02F018BF404270474FF00000EB
:10185000704750EA013005D111F0004008BF6FF029
:10186000004070474FF00000704700BF4FEA410250
:10187000B2F1E04324BFB3F5001CDCF1FE5C0DD9EE
:1018800001F0004C4FEAC0024CEA5070B2F1004F38
:1018900040EB830008BF20F00100704711F0804F3B
:1018A00021D113F13872BCBF01F00040704741F400
:1018B00080114FEA5252C2F11802C2F1200C10FA04
:1018C0000CF320FA02F018BF40F001004FEAC123E8
:1018D0004FEAD32303FA0CFC40EA0C0023FA02F38C
:1018E0004FEA4303CCE77FEA625307D150EA013362
:1018F0001EBF4FF0FE4040F44000704701F0004032
:1019000040F0FE4040F40000704700BF80F000400F
:1019100002E000BF81F0004142001FBF5FEA4103C7
:1019200092EA030F7FEA226C7FEA236C6AD04FEAC7
:101930001262D2EB1363C1BFD2184140484041400C
:10194000B8BF5B42192B88BF704710F0004F40F4BE
:10195000000020F07F4018BF404211F0004F41F4DA
:10196000000121F07F4118BF494292EA030F3FD0A6
:10197000A2F1010241FA03FC10EB0C00C3F12003B9
:1019800001FA03F100F0004302D5494260EB400048
:10199000B0F5000F13D3B0F1807F06D340084FEAB3
:1019A000310102F10102FE2A51D2B1F1004F40EBA8
:1019B000C25008BF20F0010040EA03007047490010
:1019C00040EB000010F4000FA2F10102EDD1B0FADB
:1019D00080FCACF1080CB2EB0C0200FA0CF0AABFD0
:1019E00000EBC25052421843BCBFD040184370476E
:1019F00092F0000F81F4000106BF80F40000013274
:101A0000013BB5E74FEA41037FEA226C18BF7FEA4A
:101A1000236C21D092EA030F04D092F0000F08BF8C
:101A20000846704790EA010F1CBF0020704712F073
:101A30007F4F04D1400028BF40F00040704712F1B2
:101A400000723CBF00F50000704700F0004343F017
:101A5000FE4040F4000070477FEA226216BF08464D
:101A60007FEA23630146420206BF5FEA412390EA10
:101A7000010F40F4800070474FF0000304E000BF06
:101A800010F0004348BF40425FEA000C08BF7047B7
:101A900043F0964301464FF000001CE050EA01027B
:101AA00008BF70474FF000030AE000BF50EA010290
:101AB00008BF704711F0004302D5404261EB41017D
:101AC0005FEA010C02BF84460146002043F0B643A2
:101AD00008BFA3F18053A3F50003BCFA8CF2083AC7
:101AE000A3EBC25310DB01FA02FC634400FA02FCD0
:101AF000C2F12002BCF1004F20FA02F243EB0200D7
:101B000008BF20F00100704702F1200201FA02FC38
:101B1000C2F1200250EA4C0021FA02F243EB02002B
:101B200008BF20EADC7070474FF0FF0C1CEAD0526F
:101B30001EBF1CEAD15392EA0C0F93EA0C0F6FD030
:101B40001A4480EA010C400218BF5FEA41211ED00E
:101B50004FF0006343EA501043EA5111A0FB0131FA
:101B60000CF00040B1F5000F3EBF490041EAD371CF
:101B70005B0040EA010062F17F02FD2A1DD8B3F14B
:101B8000004F40EBC25008BF20F00100704790F0BA
:101B9000000F0CF0004C08BF49024CEA502040EA0C
:101BA00051207F3AC2BFD2F1FF0340EAC2507047D2
:101BB00040F400004FF00003013A5DDC12F1190F10
:101BC000DCBF00F000407047C2F10002410021FA82
:101BD00002F1C2F1200200FA02FC5FEA310040F19A
:101BE000000053EA4C0308BF20EADC70704792F013
:101BF000000F00F0004C02BF400010F4000F013A4B
:101C0000F9D040EA0C0093F0000F01F0004C02BF45
